:100000000C940D180C943E180C943E180C943E1849
:100010000C943E180C943E180C943E180C943E1808
:100020000C943E180C943E180C943E180C943E18F8
:100030000C943E180C9406C70C943E180C943E1871
:100040000C943E180C9437A50C943E180C943E1852
:100050000C943E180C943E180C94212F0C94CCC296
:100060000C943E180C9405A20C943E180C943E1867
:100070000C943E180C943E180C943E180C943E18A8
:100080000C943E180C943E180C943E180C943E1898
:100090000C943E180C943E180C943E180C94FEBF21
:1000A0000C943E180C943E180C943E180C943E1878
:1000B0000C943E180C943E180C943E180C943E1868
:1000C0000C943E180C943E180C943E180C943E1858
:1000D0000C943E180C943E180C943E180C943E1848
:1000E0000C943E186E2F7C2F982FA62FC02FCE2F4A
:1000F000E82FEC2FEE2FF22FFA2F50C155C15AC125
:1001000064C1DDC16EC176C17EC188C192C19CC18E
:10011000ABC1B5C1DDC1BFC1C9C1D3C1FBC1FEC146
:10012000F1C1F5C135C202C206C20CC210C214C26E
:100130001AC21EC222C235C228C22CC230C2084A0C
:10014000D73B3BCE016E84BCBFFDC12F3D6C7431EB
:100150009ABD56833DDA3D00C77F11BED9E4BB4C42
:100160003E916BAAAABE000000803F05A84CCDB20C
:10017000D44EB93836A9020C50B9918688083CA6ED
:10018000AAAA2ABE000000803F007C3C3E5E2B3DB8
:100190003F2F5B5D3B2C2A225C004572723A204D5A
:1001A000415854454D50204245440054656D70659A
:1001B000726174757265206865617465642062653A
:1001C00064207377697463686564206F66662E20A7
:1001D0004D415854454D502074726967676572658A
:1001E00064202121004572723A204D494E54454DFC
:1001F00050003A204578747275646572207377698F
:100200007463686564206F66662E204D494E5445C0
:100210004D502074726967676572656420210045DE
:1002200072723A204D415854454D50003A2045785D
:10023000747275646572207377697463686564208D
:100240006F66662E204D415854454D50207472699A
:10025000676765726564202100202D20496E7661F4
:100260006C6964206578747275646572206E756D52
:10027000626572202100504944204175746F747585
:100280006E652066696E69736865642120507574B7
:1002900020746865206C617374204B702C204B694E
:1002A00020616E64204B6420636F6E7374616E74A2
:1002B000732066726F6D2061626F766520696E745F
:1002C0006F20436F6E66696775726174696F6E2E19
:1002D0006800504944204175746F74756E652066DE
:1002E00061696C6564212074696D656F75740020A7
:1002F000403A006F6B20543A006F6B20423A005036
:100300004944204175746F74756E65206661696C2F
:100310006564212054656D70657261747572652025
:10032000746F6F206869676800204B643A20002072
:100330004B693A2000204B703A200020436C6173D7
:100340007369632050494420002054753A200020EE
:100350004B753A2000206D61783A2000206D696E5F
:100360003A200020643A200020626961733A20003C
:1003700070012C0190012701B0012201C0011D0173
:10038000F00118011002130130020E016002090190
:1003900090020401C002FF000003FA004003F500D0
:1003A0008003F000D003EB002004E6007004E100BD
:1003B000E004DC004005D700C005D2004006CD00B7
:1003C000D006C8008007C3003008BE00F008B9009E
:1003D000C009B400B00AAF00B00BAA00D00CA50051
:1003E000000EA000500F9B00C0109600501291000C
:1003F00000148C00C0158700B0178200B0197D0072
:10040000D01B7800001E730040206E00902269000F
:10041000F024640040275F0090295A00E02B55002B
:10042000102E500020304B0010324600E0334100C7
:1004300090353C001037370070383200A0392D005D
:10044000B03A2800A03B2300603C1E00103D19007C
:10045000903D1400103E0F00703E0A00C03E0500A3
:10046000003F0000686F77746F2E70727573613390
:10047000642E637A00686F77746F2E707275736183
:1004800033642E636F6D00666F72756D2E707275BA
:10049000736133642E637A00666F72756D2E7072AD
:1004A00075736133642E636F6D00707275736133A1
:1004B000642E637A00707275736133642E636F6D9E
:1004C000005679626572206A617A796B612020201A
:1004D00020202020200053656C656374206C616EC1
:1004E000677561676520202020200043657374696B
:1004F0006E6100456E676C697368004572726F7259
:1005000020696E206D656E752073747275637475E5
:100510007265004572726F7220696E206D656E752E
:100520002073747275637475726500446F737461BF
:10053000766F76616E69205A0041646A75737469DA
:100540006E67205A00426162797374657070696EDB
:1005500067205900426162797374657070696E67D3
:10056000205900426162797374657070696E67200A
:100570005800426162797374657070696E672058C3
:100580000020746F6F206C6F6E67206578747275D1
:1005900073696F6E2070726576656E746564002095
:1005A000746F6F206C6F6E672065787472757369F5
:1005B0006F6E2070726576656E7465640020636F7F
:1005C0006C6420657874727573696F6E20707265E3
:1005D00076656E7465640020636F6C642065787462
:1005E000727573696F6E2070726576656E7465647E
:1005F00000656E6473746F7073206869743A2000CC
:10060000656E6473746F7073206869743A20005368
:100610007465707261746520746F6F2068696768B3
:100620003A2000537465707261746520746F6F2096
:10063000686967683A200043616E6E6F7420656E6A
:10064000746572207375626469723A200043616E4A
:100650006E6F7420656E7465722073756264697262
:100660003A20006572726F722077726974696E67E2
:1006700020746F2066696C65006572726F722077F6
:10068000726974696E6720746F2066696C65004ECC
:100690006F74205344207072696E74696E67004EE7
:1006A0006F74205344207072696E74696E670053D2
:1006B00044207072696E74696E6720627974652077
:1006C000005344207072696E74696E672062797499
:1006D00065200057726974696E6720746F206669BF
:1006E0006C653A200057726974696E6720746F20D8
:1006F00066696C653A200046696C652073656C65B7
:10070000637465640046696C652073656C65637429
:100710006564002053697A653A20002053697A6540
:100720003A200046696C65206F70656E65643A20FA
:100730000046696C65206F70656E65643A20006FD5
:1007400070656E206661696C65642C2046696C6515
:100750003A20006F70656E206661696C65642C20BC
:1007600046696C653A2000776F726B446972206F3E
:1007700070656E206661696C656400776F726B44AA
:100780006972206F70656E206661696C65640053E4
:10079000442063617264206F6B0053442063617274
:1007A00064206F6B006F70656E526F6F74206661AE
:1007B000696C6564006F70656E526F6F742066615E
:1007C000696C656400766F6C756D652E696E697411
:1007D000206661696C656400766F6C756D652E6965
:1007E0006E6974206661696C656400534420696EAB
:1007F0006974206661696C00534420696E697420D5
:100800006661696C0043616E6E6F74206F70656E17
:10081000207375626469720043616E6E6F74206F3D
:1008200070656E2073756264697200486F74656EDE
:1008300064206F6666736574733A00486F74656E02
:1008400064206F6666736574733A006F70656E003E
:100850006F70656E005452494747455245440054F5
:100860005249474745524544005265706F7274695A
:100870006E6720656E6473746F7020737461747535
:1008800073005265706F7274696E6720656E647371
:10089000746F7020737461747573007A5F6D617822
:1008A0003A20007A5F6D61783A20007A5F6D696E58
:1008B0003A20007A5F6D696E3A2000795F6D617849
:1008C0003A2000795F6D61783A2000795F6D696E3A
:1008D0003A2000795F6D696E3A2000785F6D61782B
:1008E0003A2000785F6D61783A2000785F6D696E1C
:1008F0003A2000785F6D696E3A2000496E76616C2F
:10090000696420657874727564657200496E7661F9
:100910006C696420657874727564657200416374F3
:100920006976652045787472756465723A20004175
:1009300063746976652045787472756465723A20CF
:1009400000556E6B6E6F776E20636F6D6D616E64B8
:100950003A202200556E6B6E6F776E20636F6D6D5F
:10096000616E643A202200526573656E643A20001D
:10097000526573656E643A20005072696E746572D8
:100980002073746F707065642064756520746F20C7
:100990006572726F72732E204669782074686520C4
:1009A0006572726F7220616E6420757365204D39B7
:1009B000393920746F20726573746172742E202827
:1009C00054656D706572617475726520697320720B
:1009D000657365742E205365742069742061667494
:1009E00065722072657374617274696E6729005054
:1009F00072696E7465722073746F707065642064C0
:100A0000756520746F206572726F72732E2046694F
:100A10007820746865206572726F7220616E642040
:100A2000757365204D39393920746F207265737480
:100A30006172742E202854656D70657261747572D0
:100A4000652069732072657365742E205365742068
:100A50006974206166746572207265737461727462
:100A6000696E6729005072696E7465722068616CE6
:100A70007465642E206B696C6C28292063616C6C32
:100A8000656421005072696E7465722068616C74CF
:100A900065642E206B696C6C28292063616C6C6521
:100AA00064210020436F756E7420583A2000204363
:100AB0006F756E7420583A20004649524D57415286
:100AC000455F4E414D453A4D61726C696E2056311D
:100AD0002E302E323B20537072696E7465722F6710
:100AE00072626C206D617368757020666F7220672A
:100AF000656E36204649524D574152455F55524C1E
:100B00003A68747470733A2F2F6769746875622E2F
:100B1000636F6D2F707275736133642F50727573CC
:100B2000612D69332D506C75732F2050524F544FE7
:100B3000434F4C5F56455253494F4E3A312E302069
:100B40004D414348494E455F545950453A5072759E
:100B500073612069332045585452554445525F43D0
:100B60004F554E543A3120555549443A3030303083
:100B7000303030302D303030302D303030302D307E
:100B80003030302D30303030303030303030303068
:100B90000A004649524D574152455F4E414D453A34
:100BA0004D61726C696E2056312E302E323B2053CF
:100BB0007072696E7465722F6772626C206D6173FA
:100BC00068757020666F722067656E3620464952E0
:100BD0004D574152455F55524C3A68747470733AA0
:100BE0002F2F6769746875622E636F6D2F70727531
:100BF000736133642F50727573612D69332D506C9E
:100C000075732F2050524F544F434F4C5F564552EF
:100C100053494F4E3A312E30204D414348494E45BD
:100C20005F545950453A50727573612069332045BD
:100C3000585452554445525F434F554E543A312013
:100C4000555549443A30303030303030302D303026
:100C500030302D303030302D303030302D3030309D
:100C60003030303030303030300A00426564204F50
:100C70004B2E0042656420646F6E652E005A6168D9
:100C8000726976616E69206265642E2E2E0042655F
:100C9000642048656174696E672E005A61687269E4
:100CA00076616E69204F4B2E0048656174696E67EE
:100CB00020646F6E652E005A6168726976616E6994
:100CC0002E2E2E0048656174696E672E2E2E004D03
:100CD00031303920496E76616C69642065787472B0
:100CE0007564657220004D31303920496E76616C33
:100CF000696420657874727564657220004E6F2097
:100D0000746865726D6973746F7273202D206E6FD5
:100D10002074656D7065726174757265004E6F2028
:100D2000746865726D6973746F7273202D206E6FB5
:100D30002074656D7065726174757265004D323234
:100D40003120496E76616C696420657874727564CF
:100D5000657220004D32323120496E76616C6964D3
:100D600020657874727564657220004D32313820C8
:100D7000496E76616C696420657874727564657219
:100D800020004D32313820496E76616C69642065EF
:100D90007874727564657220004D32303020496E6F
:100DA00076616C6964206578747275646572200080
:100DB0004D32303020496E76616C696420657874FC
:100DC000727564657220004D31303520496E766150
:100DD0006C696420657874727564657220004D31A9
:100DE000303520496E76616C69642065787472755F
:100DF00064657220004D31303420496E76616C6933
:100E00006420657874727564657220004D313034E9
:100E100020496E76616C69642065787472756465CA
:100E2000722000456E642066696C65206C6973747D
:100E300000456E642066696C65206C6973740042BD
:100E40006567696E2066696C65206C697374004221
:100E50006567696E2066696C65206C69737400440F
:100E60006F6E65207072696E74696E672066696C5A
:100E70006500446F6E65207072696E74696E6720DC
:100E800066696C65004E6F204C696E65204E756D0D
:100E9000626572207769746820636865636B737537
:100EA0006D2C204C617374204C696E653A20004EA5
:100EB0006F204C696E65204E756D62657220776992
:100EC000746820636865636B73756D2C204C617367
:100ED00074204C696E653A20004E6F20436865634C
:100EE0006B73756D2077697468206C696E65206E10
:100EF000756D6265722C204C617374204C696E654F
:100F00003A20004E6F20436865636B73756D2077E0
:100F1000697468206C696E65206E756D6265722CEF
:100F2000204C617374204C696E653A2000636865DB
:100F3000636B73756D206D69736D617463682C20CC
:100F40004C617374204C696E653A20006368656378
:100F50006B73756D206D69736D617463682C204CC3
:100F6000617374204C696E653A20004C696E65208F
:100F70004E756D626572206973206E6F74204C61CE
:100F80007374204C696E65204E756D6265722B31ED
:100F90002C204C617374204C696E653A20004C69BA
:100FA0006E65204E756D626572206973206E6F7478
:100FB000204C617374204C696E65204E756D6265BE
:100FC000722B312C204C617374204C696E653A2071
:100FD00000446F6E6520736176696E672066696C88
:100FE000652E00446F6E6520736176696E672066BA
:100FF000696C652E006F6B006F6B002020506C6178
:101000006E6E657242756666657242797465733A92
:1010100020002020506C616E6E65724275666665B8
:101020007242797465733A20002046726565204DDE
:10103000656D6F72793A20002046726565204D65B6
:101040006D6F72793A2000204C6173742055706482
:10105000617465643A2000204C617374205570649B
:10106000617465643A2000207C20417574686F7259
:101070003A2000207C20417574686F723A2000206D
:10108000536F6674776172652052657365740020D2
:10109000536F6674776172652052657365740020C2
:1010A0005761746368646F672052657365740020CC
:1010B0005761746368646F672052657365740020BC
:1010C00042726F776E206F7574205265736574007D
:1010D0002042726F776E206F75742052657365744D
:1010E000002045787465726E616C2052657365747A
:1010F000002045787465726E616C2052657365746A
:1011000000506F776572557000506F77657255703B
:1011100000656E717565696E67202200656E717578
:1011200065696E672022002070726F2070726F6A8E
:101130006576656E69207A6D656E0020666F722037
:1011400074616B65206566666563740052657374CF
:10115000617274756A7465207469736B61726E75FF
:10116000005265626F6F7420746865207072696EDA
:10117000746572004D6F6420205B7679732E207643
:10118000796B6F6E5D004D6F6465205B68696768A1
:1011900020706F7765725D004D6F642020202020E5
:1011A00020205B74696368795D004D6F6465202061
:1011B0002020205B73696C656E745D0056796D65E7
:1011C0006E612066696C616D656E7475210043689F
:1011D000616E67696E672066696C616D656E74210A
:1011E00000566C6F7A74652066696C616D656E740B
:1011F00000496E736572742066696C616D656E740A
:10120000004120737469736B6E65746520746C6142
:101210006369746B6F00416E642070726573732034
:10122000746865206B6E6F62005A6D656E61207523
:10123000737065736E6121004368616E676520732A
:10124000756363657373210043697374656E692008
:101250006261727679004C6F6164696E6720636FBA
:101260006C6F720050726F73696D2063656B656A95
:10127000746500506C656173652077616974005A0C
:1012800061766164656E692066696C616D656E7416
:1012900075004C6F6164696E672066696C616D658D
:1012A0006E74004261727661206E656E69206369BA
:1012B00073746100436F6C6F72206E6F7420636C87
:1012C0006561720046696C616D656E74206E657A49
:1012D00061766564656E0046696C616D656E74204B
:1012E0006E6F74206C6F61646564004E65004E6FB4
:1012F00000416E6F005965730056796D656E61200F
:101300006F6B3F004368616E67656420636F727244
:101310006563746C793F00506F64706F7261005345
:101320007570706F72740050726564656872656A7A
:10133000746520747279736B7521005072656865ED
:10134000617420746865206E6F7A7A6C6521004341
:10135000485942413A004552524F523A0052656351
:101360007472616374005265637472616374005ACD
:1013700061766573742066696C616D656E74004C8E
:101380006F61642066696C616D656E740056796A80
:101390006D6F75742066696C616D656E7400556E55
:1013A0006C6F61642066696C616D656E740050726B
:1013B0006564656872657600507265686561740081
:1013C0004E6173746176656E690053657474696EFD
:1013D0006773004B616C6962726F766174205A00AA
:1013E00043616C696272617465205A004175746F63
:1013F00020646F6C61646974205A203F00417574E9
:101400006F2061646A757374205A203F00456E64D2
:1014100073746F702061626F727400456E647374D0
:101420006F702061626F727400446F6C6164656EEE
:1014300069206F7379205A004C6976652061646A6F
:10144000757374205A004261627973746570205913
:10145000004261627973746570205900426162795B
:1014600073746570205800426162797374657020EE
:1014700058005A204F6666736574005A204F66669E
:1014800073657400486F6D6520582F59206265663A
:101490006F7265205A00486F6D6520582F59206281
:1014A00065666F7265205A005A2070726F626520FF
:1014B0006F75742E20626564005A2070726F6265C9
:1014C000206F75742E206265640056796D656E69B3
:1014D00074205344004368616E6765205344206361
:1014E00061726400496E69632E20534400496E693D
:1014F000742E20534420636172640056796D656ECA
:1015000069742066696C616D656E74004368616E14
:1015100067652066696C616D656E74004175746FF6
:10152000526574722E004175746F526574722E008C
:10153000556E52657420205600556E5265742020F9
:1015400056005320556E5265742B6D6D0053205517
:101550006E5265742B6D6D00556E526574202B6D47
:101560006D00556E526574202B6D6D00486F7020B4
:101570006D6D00486F70206D6D005265747261630F
:1015800074202056005265747261637420205600E6
:10159000537761702052652E6D6D00537761702016
:1015A00052652E6D6D0052657472616374206D6DAD
:1015B0000052657472616374206D6D0053544F5016
:1015C0005045442E200053544F505045442E200087
:1015D0004B494C4C45442E20004B494C4C45442E25
:1015E00020004E6F206D6F76652E004E6F206D6F60
:1015F00076652E005469736B207072657275736521
:101600006E005072696E742061626F72746564005E
:101610004F626E6F76656E69207469736B750052E8
:101620006573756D696E67207072696E74005761BD
:10163000697420666F7220757365722E2E2E0057A6
:1016400061697420666F7220757365722E2E2E008C
:10165000536C6565702E2E2E00536C6565702E2EB2
:101660002E005A61646E61205344206B6172746174
:10167000004E6F2053442063617264005469736BA1
:10168000207A205344005072696E742066726F6D28
:10169000205344005A6173746176697420746973CD
:1016A0006B0053746F70207072696E7400506F6BB2
:1016B0007261636F76617400526573756D65207039
:1016C00072696E7400506F7A617374617669742008
:1016D0007469736B005061757365207072696E7404
:1016E000004C616469740054756E650050726970D5
:1016F00072617661005072657061726500496E6654
:101700006F726D61636500496E666F207363726509
:10171000656E004F626E6F76697400526566726521
:101720007368004F626E6F76697420767963686FB4
:101730007A6900526573746F7265206661696C73B3
:1017400061666500556C6F7A69742070616D6574AF
:10175000004C6F6164206D656D6F72790053746F1A
:101760007265206D656D6F72790053746F726520BC
:101770006D656D6F7279004C434420636F6E7472B7
:10178000617374004C434420636F6E7472617374B0
:101790000046696C2E204469612E20330046696C36
:1017A0002E204469612E20330046696C2E20446946
:1017B000612E20320046696C2E204469612E203251
:1017C0000046696C2E204469612E20310046696C08
:1017D0002E204469612E2031004520696E206D6DF8
:1017E00033004520696E206D6D330046696C616D74
:1017F000656E740046696C616D656E7400506F684B
:101800007962004D6F74696F6E005465706C6F740F
:10181000610054656D706572617475726500457321
:10182000746570732F6D6D004573746570732F6DE3
:101830006D005A73746570732F6D6D005A73746503
:1018400070732F6D6D005973746570732F6D6D001B
:101850005973746570732F6D6D0058737465707370
:101860002F6D6D005873746570732F6D6D00412D71
:101870007265747261637400412D72657472616384
:101880007400416D61782000416D617820005654EC
:10189000726176206D696E005654726176206D69B2
:1018A0006E00566D696E00566D696E0065006500CC
:1018B0007A007A007900790078007800566D6178B6
:1018C0002000566D6178200056652D6A65726B00A8
:1018D00056652D6A65726B00567A2D6A65726B00CB
:1018E000567A2D6A65726B005678792D6A65726B2F
:1018F000005678792D6A65726B00416363656C00F0
:10190000416363656C005049442D43005049442DA8
:1019100043005049442D44005049442D440050494F
:10192000442D49005049442D49005049442D500050
:101930005049442D50004F6666004F6666004F6E5A
:1019400020004F6E20004175746F74656D7000410A
:1019500075746F74656D70002002204661637400B9
:1019600020022046616374002002204D617800202F
:1019700002204D6178002002204D696E0020022077
:101980004D696E004B6F6E74726F6C6100436F6EC9
:1019900074726F6C00507275746F6B203200466CFD
:1019A0006F77203200507275746F6B203100466C77
:1019B0006F77203100507275746F6B203000466C69
:1019C0006F77203000507275746F6B00466C6F77C4
:1019D00000527963686C6F73742076656E742E00A4
:1019E00046616E20737065656400426564004265FF
:1019F0006400547279736B6133004E6F7A7A6C6550
:101A00003300547279736B6132004E6F7A7A6C6571
:101A10003200547279736B61004E6F7A7A6C650094
:101A2000527963686C6F737400537065656400501D
:101A30006F73756E6F7574206F2031306D6D004D52
:101A40006F76652031306D6D00506F73756E6F75F8
:101A500074206F20316D6D004D6F766520316D6D96
:101A600000506F73756E6F7574206F20302E316D5E
:101A70006D004D6F766520302E316D6D00457874A8
:101A8000727564657233004578747275646572337B
:101A900000457874727564657232004578747275A9
:101AA00064657232004578747275646572004578B9
:101AB00074727564657200506F73756E6F75742003
:101AC0005A004D6F7665205A00506F73756E6F75B2
:101AD000742059004D6F7665205900506F73756EF4
:101AE0006F75742058004D6F7665205800506F73E5
:101AF000756E6F7574206F7375004D6F766520611C
:101B0000786973005265747261637400526574720F
:101B1000616374004578747275646F766174004512
:101B2000787472756465005A61706E6F7574207A8E
:101B300064726F6A0053776974636820706F7765A9
:101B400072206F6666005679706E6F7574207A64C5
:101B5000726F6A0053776974636820706F7765727B
:101B6000206F6E005A63686C6164697400436F6F24
:101B70006C646F776E00507265646568726576207C
:101B800041425320636F6E660050726568656174F0
:101B90002041425320636F6E660050726564656831
:101BA0007265762041425320426564005072656838
:101BB000656174204142532042656400507265643F
:101BC00065687265762041425320416C6C0050720A
:101BD00065686561742041425320416C6C0050720D
:101BE0006564656872657620414253203300507207
:101BF000656865617420414253203300507265640A
:101C000065687265762041425320320050726568E3
:101C100065617420414253203200507265646568EA
:101C200072657620414253203100507265686561CB
:101C300074204142532031005072656465687265BA
:101C400076204142530050726568656174204142BC
:101C5000530050726564656872657620504C41206F
:101C6000636F6E66005072656865617420504C4108
:101C700020636F6E660050726564656872657620D9
:101C8000504C412042656400507265686561742063
:101C9000504C41204265640050726564656872650D
:101CA0007620504C4120416C6C0050726568656133
:101CB0007420504C4120416C6C0050726564656822
:101CC00072657620504C4120330050726568656122
:101CD0007420504C41203300507265646568726511
:101CE0007620504C41203200507265686561742046
:101CF000504C4120320050726564656872657620F0
:101D0000504C412031005072656865617420504C20
:101D10004120310050726564656872657620504CD0
:101D200041005072656865617420504C41004E61FD
:101D30007374617620706F636174656B00536574B2
:101D4000206F726967696E004E61737461762070EE
:101D50006F636174656B20686F6D650053657420F7
:101D6000686F6D65206F6666736574730041757486
:101D70006F20686F6D65004175746F20686F6D65C9
:101D8000005679706E6F7574206D6F746F72790084
:101D900044697361626C65207374657070657273F9
:101DA000004175746F7374617274004175746F7360
:101DB0007461727400486C61766E69206E6162694C
:101DC000646B61004D61696E004B617274612076D5
:101DD000796A6D75746100436172642072656D6F1C
:101DE000766564004B6172746120766C6F7A656E03
:101DF00061004361726420696E736572746564008A
:101E000050727573612069332070726970726176E7
:101E1000656E61005072757361206933207265616F
:101E200064792E004D383420582059205A2045001E
:101E30004D3234004D3233202573006175746F25A7
:101E4000692E67000A002F000A002E0044656C65A9
:101E500074696F6E206661696C65642C2046696CDC
:101E6000653A200046696C652064656C657465643C
:101E70003A002E002E002E002E004E6F7720667244
:101E80006573682066696C653A20004E6F77206440
:101E90006F696E672066696C653A20002220706F5A
:101EA00073002220706172656E743A2200535542AD
:101EB000524F5554494E452043414C4C2074617259
:101EC0006765743A2200747279696E6720746F20B6
:101ED00063616C6C207375622D67636F6465206647
:101EE000696C6573207769746820746F6F206D6109
:101EF0006E79206C6576656C732E204D4158206C90
:101F00006576656C2069733A0000002110422063F9
:101F1000308440A550C660E770088129914AA16BC2
:101F2000B18CC1ADD1CEE1EFF1311210027332525A
:101F300022B5529442F772D662399318837BB35A12
:101F4000A3BDD39CC3FFF3DEE3622443342004012A
:101F500014E664C774A44485546AA54BB528850962
:101F600095EEE5CFF5ACC58DD553367226111630FA
:101F700006D776F6669556B4465BB77AA7199738B2
:101F800087DFF7FEE79DD7BCC7C448E5588668A73A
:101F9000784008611802282338CCC9EDD98EE9AF02
:101FA000F9488969990AA92BB9F55AD44AB77A969A
:101FB0006A711A500A333A122AFDDBDCCBBFFB9E52
:101FC000EB799B588B3BBB1AABA66C877CE44CC56A
:101FD0005C222C033C600C411CAEED8FFDECCDCDA2
:101FE000DD2AAD0BBD688D499D977EB66ED55EF43A
:101FF0004E133E322E511E700E9FFFBEEFDDDFFCF2
:10200000CF1BBF3AAF599F788F8891A981CAB1EB96
:10201000A10CD12DC14EF16FE18010A100C230E3BF
:10202000200450254046706760B9839893FBA3DA7B
:10203000B33DC31CD37FE35EF3B1029012F322D20F
:10204000323542145277625672EAB5CBA5A895890B
:10205000856EF54FE52CD50DC5E234C324A014815F
:10206000046674476424540544DBA7FAB79987B81B
:10207000975FE77EF71DC73CD7D326F2369106B0AF
:102080001657667676154634564CD96DC90EF92F1B
:10209000E9C899E9898AB9ABA944586548067827FF
:1020A00068C018E1088238A3287DCB5CDB3FEB1EBB
:1020B000FBF98BD89BBBAB9ABB754A545A376A164F
:1020C0007AF10AD01AB32A923A2EFD0FED6CDD4D4B
:1020D000CDAABD8BADE89DC98D267C076C645C459F
:1020E0004CA23C832CE01CC10C1FEF3EFF5DCF7C5B
:1020F000DF9BAFBABFD98FF89F176E367E554E74EF
:102100005E932EB23ED10EF01E22004D32323020B0
:1021100053256900203A2000004C414E472053458A
:102120004C20464F52434544002200205A3A00209A
:10213000593A0020453A00205A3A0020593A0058AE
:102140003A0020002E0020423A0020453A00543A3E
:102150000020573A0020453A00543A002042403AC5
:102160000020403A00202F003A00205400202F0089
:1021700020423A00202F006F6B20543A002569203E
:102180006D696E2C202569207365630025692068C0
:102190006F757273202569206D696E7574657300A3
:1021A0004D313130004D32390046656220323120E8
:1021B0003230313600436F6D70696C65643A2000CF
:1021C000286E6F6E652C2064656661756C74206383
:1021D0006F6E6669672900466562203231203230B1
:1021E00031362031373A32313A323100737461720C
:1021F000740022002200FFFFFF0000A0400000A0AA
:10220000400000004000005643000046431FC54800
:102210004300000000000000001F856B3E000056D8
:102220004300004643000049430000000000000056
:10223000001F856B3E6563686F3A004572726F726E
:102240003A004731204534302046313030004731A4
:10225000204536352046343030004D383300473184
:1022600020452D38302046343030004D3833002D95
:102270002D3A2D2D002D2D2D00534400012000015D
:1022800020004D36303000464C4558202D2020325D
:1022900035302F35300050502020202D2020323571
:1022A000342F3130300048495053202D2020323215
:1022B000302F3130300050455420202D2020323432
:1022C000302F393000504C4120202D202032323028
:1022D0002F35300041425320202D20203238352F19
:1022E000313030004D3834004D38342058205920DA
:1022F0005A2045004D3234004D32332025730058AA
:102300000059005A0045787472756465720047324E
:1023100038004D383400473238205A0050727573F7
:10232000614E6D6B320052414D426F31336100336B
:102330006D6D002D2D2D2D2D2D2D2D2D2D2D2D00A7
:102340004669726D77617265202D20322E322E33F0
:102350000048617264636F646564204465666175FA
:102360006C742053657474696E6773204C6F61647C
:1023700065640046696C616D656E74207365747484
:10238000696E67733A2044697361626C656400200A
:1023900020204D32303020440046696C616D656EFE
:1023A000742073657474696E67733A002020204D41
:1023B0003230392053004175746F2D52657472614B
:1023C00063743A20533D3020746F206469736162F6
:1023D0006C652C203120746F20696E746572707288
:1023E000657420657874727564652D6F6E6C7920E4
:1023F0006D6F7665732061732072657472616374AA
:1024000073206F72207265636F7665726965730001
:102410002046002020204D32303820530052656382
:102420006F7665723A20533D4578747261206C6511
:102430006E67746820286D6D2920463A5370656573
:102440006420286D6D2F6D2900205A002046002041
:1024500020204D323037205300526574726163740E
:102460003A20533D4C656E67746820286D6D2920B5
:10247000463A537065656420286D6D2F6D29205A8A
:102480003A205A4C69667420286D6D29002044005A
:102490002049002020204D33303120500050494445
:1024A0002073657474696E67733A00205A0020596E
:1024B0000020204D323036205800486F6D65206F67
:1024C000666673657420286D6D293A0020450020EA
:1024D0005A0020580020420020540020204D323065
:1024E00035205300416476616E63656420766172C5
:1024F0006961626C65733A20533D4D696E20666573
:1025000065647261746520286D6D2F73292C2054C9
:102510003D4D696E2074726176656C2066656564F8
:102520007261746520286D6D2F73292C20423D6DDA
:10253000696E696D756D207365676D656E74207465
:10254000696D6520286D73292C20583D6D6178696F
:102550006D756D205859206A65726B20286D6D2F3E
:1025600073292C20205A3D6D6178696D756D205A54
:10257000206A65726B20286D6D2F73292C202045F1
:102580003D6D6178696D756D2045206A65726B20BF
:10259000286D6D2F73290020540020204D323034D7
:1025A000205300416363656C65726174696F6E3AB4
:1025B00020533D616363656C65726174696F6E2C55
:1025C00020543D7265747261637420616363656C4D
:1025D00065726174696F6E00204500205A002059B1
:1025E0000020204D3230312058004D6178696D75E2
:1025F0006D20416363656C65726174696F6E20283C
:102600006D6D2F7332293A00204500205A00205961
:102610000020204D3230332058004D6178696D75AF
:102620006D2066656564726174657320286D6D2F19
:1026300073293A00204500205A0020590020204DDF
:10264000393220580053746570732070657220759C
:102650006E69743A0045303A20005A3A2000593ADF
:102660002000583A20004D53312C4D5332205069F0
:102670006E730A005A00205A3A00590020593A0055
:10268000580020583A0024F4D43050C38E20C2A2FF
:102690004017828B7011127A910D816CD90AA86152
:1026A000E108C7586607615143061E4B5D05C145E9
:1026B000A7041A411104093D9803713931034036CA
:1026C000DB0265339102D4305402802E1D02632C4C
:1026D000EE01752AC501B028A001102781018F25C0
:1026E00064012B244B01E0223401AC211F018D2019
:1026F0000D01801FFC00841EED00971DDF00B81C3B
:10270000D200E61BC600201BBC00641AB200B2193E
:10271000A8000A19A0006A189900D1179100401763
:102720008B00B516840031167E00B31579003A157A
:102730007300C7146F0058146A00EE136600881304
:10274000630025135E00C7125B006C125700151260
:102750005400C111510070114F0021114B00D610CF
:1027600049008D1047004610440002104200C00F7F
:102770004000800F3E00420F3C00060F3B00CB0E96
:102780003800930E37005C0E3500270E3400F30D31
:102790003200C10D3100900D3000600D2E00320D61
:1027A0002D00050D2C00D90C2B00AE0C2900850C3A
:1027B00029005C0C2700350C27000E0C2600E80BC6
:1027C0002400C40B2400A00B23007D0B23005A0B14
:1027D0002100390B2100180B2000F80A1F00D90A2C
:1027E0001E00BB0A1E009D0A1D00800A1D00630A10
:1027F0001C00470A1B002C0A1B00110A1A00F709CB
:102800001A00DD091900C4091900AB091900920961
:1028100017007B091800630917004C0916003609D8
:102820001600200916000A091500F5081500E00831
:102830001400CC081400B8081400A4081400900870
:1028400013007D0812006B08130058081200460898
:1028500012003408110023081100120811000108A9
:102860001100F0071000E0071000D0071000C007AB
:102870001000B0070F00A107100091070E0083079A
:102880000F0074070F0065070E0057070E00490779
:102890000E003B070D002E070E0020070D0013074A
:1028A0000D0006070D00F9060C00ED060D00E00610
:1028B0000C00D4060C00C8060C00BC060C00B006C8
:1028C0000C00A4060B0099060C008D060B00820676
:1028D0000B0077060B006C060B0061060A0057061A
:1028E0000B004C060A0042060A0038060A002E06B3
:1028F0000A0024060A001A060A0010060900070644
:102900000A00FD050900F4050900EB050900E205D0
:102910000900D9050900D0050900C7050900BE0551
:102920000900B5050800AD050800A50509009C05CE
:102930000800940508008C050800840508007C0543
:102940000800740508006C050700650508005D05B2
:102950000700560508004E0507004705070040051B
:10296000080038050700310507002A050700230580
:1029700007001C050600160507000F0507000805DF
:10298000060002050700FB040600F5040700EE043C
:102990000600E8040600E2040700DB040600D50494
:1029A0000600CF040600C9040600C3040600BD04E7
:1029B0000600B7040600B1040500AC040600A60436
:1029C0000600A00405009B04060095040500900481
:1029D00006008A04050085040500800406007A04C8
:1029E000050075040500700405006B04050066040D
:1029F0000500610405005C0405005704050052044D
:102A000005004D04050048040500430405003E048C
:102A100004003A04050035040500300404002C04C9
:102A2000050027040400230405001E0404001A0402
:102A3000040016040500110404000D040400090438
:102A400005000404040000040400FC030400F8036F
:102A50000400F4030400F0030400EC030400E803A2
:102A60000400E4030400E0030400DC030400D803D2
:102A70000400D4030400D0030400CC030400C80302
:102A80000300C503030024F404D9201BC40C5C0E0E
:102A90009804C4095F0265077101F405F900FB049D
:102AA000B30048048700C1036900580355000303BD
:102AB0004500BE023A008402310053022A00290276
:102AC000250004022000E4011C00C8011900AF0128
:102AD00017009801140084011300710110006101B6
:102AE000100051010E0043010D0036010B002B01B7
:102AF0000B0020010B00150109000C010900030166
:102B00000800FB000800F3000800EB000700E400E9
:102B10000600DE000600D8000600D2000600CC0049
:102B20000500C7000500C2000500BD000400B90093
:102B30000400B5000400B1000400AD000400A900C9
:102B40000400A5000300A20003009F0004009B00F6
:102B5000030098000300950002009300030090001A
:102B600003008D0002008B00030088000200860035
:102B7000020084000300810002007F0002007D004B
:102B800002007B000200790002007700010076005D
:102B900002007400020072000100710002006F0068
:102BA00002006D0001006C0002006A000100690073
:102BB000020067000100660001006500010064007A
:102BC00002006200010061000100600001005F007E
:102BD00002005D0001005C0001005B0001005A0082
:102BE0000100590001005800010057000100560083
:102BF0000100550001005400010053000000530083
:102C000001005200010051000100500001004F007E
:102C100001004E0000004E0001004D0001004C007C
:102C200001004B0000004B0001004A000100490078
:102C30000100480000004800010047000100460074
:102C4000000046000100450000004500010044006E
:102C50000100430000004300010042000000420068
:102C600001004100000041000100400001003F0060
:102C700000003F0001003E0000003E0001003D005A
:102C800000003D0001003C0000003C0000003C0052
:102C900001003B0000003B0001003A0000003A0048
:102CA0000100390000003900010038000000380040
:102CB0000000380001003700000037000100360036
:102CC000000036000000360001003500000035002D
:102CD0000000350001003400000034000000340022
:102CE0000100330000003300000033000100320017
:102CF000000032000000320001003100000031000D
:102D00000000310001003000000030000000300001
:102D100001002F0000002F0000002F0000002F00F6
:102D200001002E0000002E0000002E0001002D00EA
:102D300000002D0000002D0000002D0001002C00DF
:102D400000002C0000002C0000002C0001002B00D3
:102D500000002B0000002B0000002B0001002A00C7
:102D600000002A0000002A0000002A0001002900BB
:102D700000002900000029000000290000002900AF
:102D800001002800000028000000280000002800A2
:102D90000000280001002700000027000000270095
:102DA0000000270000002700010026000000260088
:102DB000000026000000260000002600010025007B
:102DC000000025000000250000002500000025006F
:102DD0000000250001002400000024000000240061
:102DE0000000240000002400010023000000230054
:102DF0000000230000002300000023000000230047
:102E00000000230001002200000022000000220038
:102E1000000022000000220000002200010021002A
:102E2000000021000000210000002100000021001E
:102E3000000021000000210001002000000020000F
:102E40000000200000002000000020000000200002
:102E5000000020000000200001001F0000001F00F3
:102E600000001F0000001F0000001F0000001F00E6
:102E700000001F0001001E0000001E0000001E00D8
:102E800000001E0000000000090A02080B0C0D07DC
:102E90000603040100000000000000000000000024
:102EA0000000000000000000000000000000000022
:102EB000000011100F0000000000000000000000E2
:102EC0000000000000000000000000000000000002
:102ED00000000000000000000000000001021020BF
:102EE0002008081020401020408002010201080440
:102EF00002010102040810204080804020100804D4
:102F0000020180040201804020100804020108042C
:102F10000201010204081020408001020408102070
:102F20004080100804088010204004408010204099
:102F300004800505050507050808080802020202C5
:102F40000A0A080804040404010101010101010145
:102F50000303030303030303040707070C0C0C0C10
:102F60000C0C0C0C020202020606060606060606F9
:102F70000B0B0B0B0B0B0B0B07070A0A0A0A0A0AAF
:102F800005050504040408080000200023002600AD
:102F900029002C002F00320000010000030106016F
:102FA000090100002200250028002B002E0031001E
:102FB000340002010000050108010B01000021009E
:102FC000240027002A002D003000330001010000FA
:102FD000040107010A01024E414E494E4954594924
:102FE0004E46CDCCCC3D0AD7233C17B7D13877CC51
:102FF0002B329595E6241FB14F0A000020410000B6
:10300000C84200401C4620BCBE4CCA1B0E5AAEC56E
:103010009D746972FD8CD2BF6D7211241FBECFEFFB
:10302000D1E2DEBFCDBF00E00CBF17E0A0E0B2E010
:10303000EAE6F6EA01E00BBF02C007900D92A03F5E
:10304000B107D9F727E1A0EFB7E001C01D92A53085
:10305000B207E1F710E3C8E1D0E300E006C0229731
:103060000109FE010BBF0E94BDCCC231D10780E037
:103070000807A9F70E94D6C30C9424D30C9400002F
:10308000CF93DF93EC019C012C5F3F4F41E050E078
:1030900060E070E0898D9A8D0E94E222882399F089
:1030A0004D895E896F89788D452B462B472B59F4C6
:1030B0004C815D816E817F814D8B5E8B6F8B788FB4
:1030C000998190689983DF91CF910895CF92DF9293
:1030D000EF92FF920F931F93CF93DF93EC018989B7
:1030E0009A89AB89BC89803E9F4FAF41B10510F0F2
:1030F00080E06BC0CE01C4DF8823D1F30E94F620AC
:10310000182F8823A9F3E98DFA8DCC80DD80EE801D
:10311000FF8032E0C31AD108E108F108058404C039
:10312000CC0CDD1CEE1CFF1C0A94D2F7868597851B
:10313000A089B189C80ED91EEA1EFB1E81E08093CA
:10314000F607C092F909D092FA09E092FB09F092D1
:10315000FC0980E092E0E9EFF7E0DF019C011D92BD
:1031600021503040E1F701E0E98DFA8D84810817A4
:1031700090F429EF37E0B701A601400F511D611D02
:10318000711D8091F7079091F8070E94B14688233E
:10319000E1F00F5FE9CFC12C82E0D82EE12CF12CB9
:1031A000058404C0CC0CDD1CEE1CFF1C0A94D2F775
:1031B00049895A896B897C894C0D5D1D6E1D7F1D67
:1031C000498B5A8B6B8B7C8B812FDF91CF911F9119
:1031D0000F91FF90EF90DF90CF900895CF93DF9302
:1031E000EC0141E0611101C040E06C857D858E8578
:1031F0009F850E943621882341F0888920E2829FA2
:10320000C00111248750984F02C080E090E0DF9108
:10321000CF91089530E020E04EE2DC015C91503225
:1032200071F0383029F4FB01E20FF11D40832F5F6C
:10323000FB01E20FF11DDC015C9150832F5F3F5FCA
:1032400001963B3051F7FB01E20FF11D108208950A
:10325000CF93DF93EB01FC012381211102C080E0B9
:103260000EC02250223020F48FE28883198206C0DB
:1032700060E0B4DF009799F3BE01CCDF81E0DF911D
:10328000CF910895FB012BE030E231932150E9F713
:10329000DC0190E027E03A2FEB2F8D9181110AC0DD
:1032A000DA013C931196EC9381E0FB01908190321E
:1032B00039F525C08F32A1F38E3219F0EAE8F1E03A
:1032C00008C02A30E1F098E02AE0E5CF31963817BF
:1032D000B1F034913111FACF291788F03FED380F52
:1032E0003E3568F431E0390FFB01E90FF11D9FE92C
:1032F000980F9A3108F480528083932FCCCF80E0CE
:1033000008950F931F93CF93DF93EC018B018B8173
:10331000882311F080E042C0FB018789803139F1B8
:103320008032C1F783E08B83F801428D538D648D29
:10333000758D4D8B5E8B6F8B788F9E012F5E3F4F0F
:10334000C8010E94ED21882329F31A8F098F81E09B
:1033500089831C821D821E821F82188619861A8606
:103360001B861C861D861E861F86188A17C082E053
:103370008B831D8A1E8A1F8A188EFB01408D518DFA
:1033800060E070E095E0440F551F661F771F9A9527
:10339000D1F7498B5A8B6B8B7C8BD7CFDF91CF9139
:1033A0001F910F9108952F923F924F925F926F92CB
:1033B0007F928F929F92AF92BF92CF92DF92EF92C5
:1033C000FF920F931F93CF93DF93EC015B016A0190
:1033D0008B81811103C08FEF9FEFC7C0898180FF70
:1033E000FACF49895A896B897C8988859985AA850C
:1033F000BB852601612C712C8A019B01081B190BCE
:103400002A0B3B0B401651066206730618F06A0140
:10341000C81AD90A76013E0124E0620E711CE1143B
:10342000F10409F476C0488559856A857B854A018F
:1034300081E098222B811A012B01E9E056944794F0
:1034400037942794EA95D1F7898D9A8DFC01223023
:1034500049F4628D738D848D958D620D731D841D6D
:10346000951D3CC014811150122181149104C1F4A6
:10347000111116C0452B462B472B49F48D899E8987
:10348000AF89B88D8C839D83AE83BF8309C04C8187
:103490005D816E817F81930121D7882309F49BCFC1
:1034A000E98DFA8D6C817D818E819F8162507109D9
:1034B00081099109058404C0660F771F881F991F31
:1034C0000A94D2F72685378540895189620F731F88
:1034D000841F951F610F711D811D911D20E032E039
:1034E0002819390987012E153F0508F489010115AE
:1034F000F2E01F0769F52091F9093091FA0940912E
:10350000FB095091FC09621773078407950719F4AA
:103510001FC0C6012AC09501AB01BC018091F7070D
:103520009091F8070E943C46882309F454CFA00EDE
:10353000B11E88859985AA85BB85800F911FA11D25
:10354000B11D88879987AA87BB87E01AF10A67CFE0
:1035500040E08CD6882309F43ECFB4016750784F01
:10356000A801C5010E94E3CFE2CFDF91CF911F9167
:103570000F91FF90EF90DF90CF90BF90AF909F9012
:103580008F907F906F905F904F903F902F90089515
:10359000CF93DF931F92CDB7DEB741E050E0BE017D
:1035A0006F5F7F4F00DF019719F4898190E002C0BF
:1035B0008FEF9FEF0F90DF91CF910895CF92DF9221
:1035C000EF92FF920F931F93CF93DF936C01EB0168
:1035D0007A01FC018381823060F0008511852285AB
:1035E00033850F71112722273327012B022B032B41
:1035F00011F08FEF5CC04115510511F0F7011082F9
:103600001DE040E250E0BE01C601CDDE80329105F2
:1036100039F021E0892B09F420E0822F819547C001
:1036200028812223C1F0253E61F32E3251F33B85E0
:103630003F733F3061F4E114F10449F04A8D5B8D32
:10364000452B29F42F713FEF320F343030F02B85AA
:1036500023FDD7CF2CC080E02AC030E021503109B3
:10366000129FC001139F900D1124F701E80FF91F5D
:10367000298120832B8121832D8122832F81238304
:10368000298524832E852583288926832A892783D3
:103690002C8920872E892187288D22872C8D2387AE
:1036A0002E8D2487288126FFD2CF1586D0CFDF919B
:1036B000CF911F910F91FF90EF90DF90CF900895E1
:1036C0001F93CF93DF93EC018B81823018F480E05D
:1036D00090E023C0488559856A857B85A5E076956D
:1036E000679557954795AA95D1F7142F1F70CE016E
:1036F0004FDF97FDECCF488559856A857B85415E14
:103700005F4F6F4F7F4F488759876A877B8720E2DB
:10371000129FC00111248750984FDF91CF911F91C4
:1037200008954F925F926F927F92AF92BF92CF9225
:10373000DF92EF92FF920F931F93CF93DF93EC01F1
:103740006A017B012B81222349F089899A89AB89FF
:10375000BC8984179507A607B70710F480E06BC0F3
:10376000223009F463C0C114D104E104F10449F426
:103770001C821D821E821F82188619861A861B864D
:1037800059C088859985AA85BB85E98DFA8DE5851F
:10379000F0E03996AC01BD01415051096109710950
:1037A0000E2E04C076956795579547950A94D2F7E3
:1037B00097018601015011092109310904C036958C
:1037C000279517950795EA95D2F704171507260749
:1037D000370720F0892B8A2B8B2B49F48D899E8902
:1037E000AF89B88D8C839D83AE83BF8304C0041BD7
:1037F000150B260B370B280139015E0184E0A80E5A
:10380000B11C411451046104710481F04C815D814B
:103810006E817F819501898D9A8D60D591E0491ADD
:103820005108610871088111ECCF05C0C886D9869E
:10383000EA86FB8681E0DF91CF911F910F91FF9087
:10384000EF90DF90CF90BF90AF907F906F905F90A0
:103850004F9008950F931F93CF93DF93EC018B81CB
:103860008823D1F1898187FF32C061E0CE01B6DCC7
:103870008C01009789F1FC018081853E69F18B8183
:10388000823040F449895A896B897C89448F558FED
:10389000668F778F4D895E896F89788DF801538F98
:1038A000428F758B648BE091F007F091F1073097B0
:1038B00059F0B8016A5E7F4FC80148961995F80122
:1038C000808D918D938B828B89818F778983DF9116
:1038D000CF911F910F918AC481E0888380E0DF91AE
:1038E000CF911F910F910895CF93DF93EC01B2DF39
:1038F0001B82DF91CF910895FC0123812111F4CF28
:1039000008954F925F926F927F92AF92BF92CF9243
:10391000DF92EF92FF920F931F93CF93DF9300D02C
:103920001F92CDB7DEB75C016A017B01FC01838188
:103930008130E9F4818181FF1AC0F5018189928982
:10394000A389B48984179507A607B70780F0892B48
:103950008A2B8B2B09F472C0F50140845184628458
:103960007384B701A601C501DCDE811102C080E0CD
:1039700066C0F501818D928DC114D104E104F1047A
:1039800069F4458956896789708D25D7882379F32D
:10399000F501158A168A178A108E37C0F501448101
:1039A0005581668177819E012F5F3F4F97D4882391
:1039B000F1F249815A816B817C81F501818D928D73
:1039C000FC012789203139F4483FFFEF5F0761058B
:1039D0007105D8F407C0483F2FEF520762072FE068
:1039E000720798F4F8D6882309F4C1CFF501448111
:1039F0005581668177810FEF1FEF2FEF3FE0818DBB
:103A0000928D51D5882309F4B2CFF501C18AD28AAB
:103A1000E38AF48A818180688183C5011BDF882362
:103A200009F4A5CFB701A6014C145D046E047F0410
:103A300010F4B301A201C50174DE01C081E00F9052
:103A40000F900F900F90DF91CF911F910F91FF90EA
:103A5000EF90DF90CF90BF90AF907F906F905F908E
:103A60004F900895FF920F931F93CF93DF93EC0134
:103A7000F42E80E2689FF0011124E750F84F83850F
:103A8000817121F0842F827109F04EC08091F90973
:103A90009091FA09A091FB09B091FC098C879D8750
:103AA000AE87BF87688B4489558960E070E0BA01B2
:103AB00055274427028D138D20E030E0402B512BF9
:103AC000622B732B4D8B5E8B6F8B788F8385887108
:103AD00051F4048D158D268D378D098B1A8B2B8B08
:103AE0003C8B81E00BC08031F9F49E012F5E3F4F8B
:103AF000898D9A8D72D48823B9F084E08B838F2DC1
:103B00008F7089831C821D821E821F8218861986EF
:103B10001A861B86F4FE0BC040E050E0BA01CE01CD
:103B2000F0DE811104C011C01B8280E00EC0F5FEE2
:103B30000BC049895A896B897C89CE01DF91CF916D
:103B40001F910F91FF90EDCD81E0DF91CF911F91FB
:103B50000F91FF900895AF92BF92CF92DF92EF92B4
:103B6000FF920F931F93CF93DF937C01EB016A01C8
:103B7000B22E898D9A8DF701928F818F40E050E0AF
:103B8000BA01CE01CEDDA12C088519852A853B8599
:103B900089899A89AB89BC89081719072A073B07C5
:103BA000A0F585E036952795179507958A95D1F765
:103BB0000F70CE0185DD009709F481C0FC012081E2
:103BC000222311F0253EB9F4A1100EC04091F9094D
:103BD0005091FA096091FB097091FC09F701448743
:103BE000558766877787008BFC018081AA24A39480
:103BF0008111CACF0AC04BE050E0BC01C6010E944F
:103C0000D6CF892B09F0C0CF58C08B2D8274823457
:103C100009F055C0AA2049F0F701008961E0C70109
:103C2000DDDAEC01009769F44AC08B81823009F437
:103C300046C0CE014BDA882309F441C0C9EFD7E072
:103C400000E080E2FE0111928A95E9F78BE0F6012F
:103C5000DE0101900D928A95E1F7E091F007F09175
:103C6000F107309739F0BE01625F7F4FCE01409679
:103C7000199508C081E298E2998B888B80E098E0E2
:103C80009F878E87888999899B8B8A8B998F888F4C
:103C90008E859F859F8B8E8BA9D2882381F04B2D9B
:103CA000602FC701DF91CF911F910F91FF90EF908F
:103CB000DF90CF90BF90AF90D5CEB7FEF0CF80E031
:103CC000DF91CF911F910F91FF90EF90DF90CF90F8
:103CD000BF90AF9008953F924F925F926F927F9204
:103CE0008F929F92AF92BF92CF92DF92EF92FF920C
:103CF0000F931F93CF93DF93CDB7DEB7C354D10992
:103D00000FB6F894DEBF0FBECDBF5C016B012496E9
:103D10005FAF4EAF2497522E1C8E1F8E19821C82CD
:103D20006115710511F410E073C0FC0183818111EC
:103D3000FACF2496EEADFFAD249780818F3211F03B
:103D400076011DC02496EEADFFAD249780818F32A1
:103D500031F431962496FFAFEEAF2497F3CFF601FE
:103D600083818250823060F3F601618D728DCE01C5
:103D70000196C7DA8823B9F2CE0101967C018E0143
:103D8000045E1F4F3801FE0131964F01402E312E47
:103D900019C08823A9F121E0AE01495C5F4FB7014A
:103DA000C801D9DE882309F4BECFEC14FD0411F05C
:103DB000C7019ADD0615170501F1942D832D7801B1
:103DC000092F182FAE014E5B5F4FBE01695C7F4F1C
:103DD00024968EAD9FAD249755DA882309F4A3CF9E
:103DE0002496EEADFFAD249780818F3291F6319607
:103DF0002496FFAFEEAF2497F3CF982D892DDFCF18
:103E0000252DAE01495C5F4FB701C501A4DE182F17
:103E1000CE01019671DDCE014C966EDD812FCD5B1A
:103E2000DF4F0FB6F894DEBF0FBECDBFDF91CF914D
:103E30001F910F91FF90EF90DF90CF90BF90AF90C8
:103E40009F908F907F906F905F904F903F900895DC
:103E5000CF93DF93EC0140E050E0BA0152DD8823BC
:103E600061F061E0CE01BAD9009739F025EEFC018E
:103E700020831B82DF91CF91B9C180E0DF91CF9188
:103E800008951F93CF93DF93CDB7DEB76B970FB62F
:103E9000F894DEBF0FBECDBFAB0119821C8222E0B9
:103EA000BC01CE01019617DF182F882321F0CE0127
:103EB0000196CEDF182FCE0101961EDD812F6B9665
:103EC0000FB6F894DEBF0FBECDBFDF91CF911F912B
:103ED00008952F923F924F925F926F927F928F92AE
:103EE0009F92AF92BF92CF92DF92EF92FF920F9389
:103EF0001F93CF93DF9300D01F921F92CDB7DEB7F1
:103F00008C015B013A01DC0113968C91139781308F
:103F1000C1F411968C9181FF14C082FF18C0F80182
:103F2000418952896389748980859185A285B38589
:103F300084179507A607B70751F0C801F2DB811176
:103F400006C081E0F80180838FEF9FEF37C16301E6
:103F500083C0D80159968D919C915A97FC01F481A8
:103F6000F1501A012B0169E0569447943794279435
:103F70006A95D1F7F221FD834A0121E09222FF23C5
:103F800009F476C080E092E08819990976018C15D1
:103F90009D0508F47C01D8015996ED91FC915A9742
:103FA00014962D903D904D905C901797B2E02B1A8F
:103FB000310841085108058404C0220C331C441CFC
:103FC000551C0A94D2F786859785A089B189280E59
:103FD000391E4A1E5B1EED812E0E311C411C511CE8
:103FE000E114F2E0FF0609F089C08091F90990918F
:103FF000FA09A091FB09B091FC0982159305A4056B
:10400000B50569F41092F6078FEF9FEFDC018093FE
:10401000F9099093FA09A093FB09B093FC09950163
:10402000B201A1018091F7079091F8070E94B14673
:10403000882309F486CFF80180859185A285B38510
:104040008E0D9F1DA11DB11D80879187A287B3870B
:10405000AE0CBF1CCE18DF08D80118964D915D91AB
:104060006D917C911B97C114D10409F072CF7AC075
:104070008114910409F086CF14964D915D916D9154
:104080007C911797411551056105710559F45596B5
:104090008D919D910D90BC91A02D0097A105B1052A
:1040A00039F520C09E012F5F3F4F18D1882309F4B6
:1040B00048CF89819A81AB81BC81F801218D328DF5
:1040C000F9012789203139F4883FFFEF9F07A105C7
:1040D000B10540F40DC0883F2FEF9207A2072FE0F3
:1040E000B20730F0C8010E94401881114BCF29CF90
:1040F000F80184839583A683B78344CF8114910408
:1041000011F5D80118964D915D916D917C911B9799
:1041100051968D919D910D90BC91A02D48175907F6
:104120006A077B0780F062D0882309F40ACF81E018
:104130008093F6072092F9093092FA094092FB0920
:104140005092FC0907C041E0C201B1018FD0882321
:1041500009F4F7CEA701B501C4018750984F0E941A
:10416000E3CF69CF51968D919D910D90BC91A02D7B
:10417000F801218184179507A607B70738F4418B0A
:10418000528B638B748B206821830CC08091F00765
:104190009091F107892B31F06114710419F02068B6
:1041A000F8012183D80111968C9183FD02C0C301CF
:1041B00005C0C8014FDB8111FACFC3CE0F900F901D
:1041C0000F900F900F90DF91CF911F910F91FF9063
:1041D000EF90DF90CF90BF90AF909F908F907F90A7
:1041E0006F905F904F903F902F900895CF93809164
:1041F000F6078823B9F14091F9095091FA096091C5
:10420000FB097091FC0929EF37E08091F707909145
:10421000F8070E94B146C82F811102C0C0E023C038
:104220004091F2075091F3076091F4077091F50700
:10423000411551056105710591F029EF37E0809135
:10424000F7079091F8070E94B146882339F310923E
:10425000F2071092F3071092F4071092F5071092EC
:10426000F60701C0C1E08C2FCF910895CF92DF9265
:10427000EF92FF92CF936B017C01C42F8091F909DB
:104280009091FA09A091FB09B091FC098C159D054C
:10429000AE05BF05C9F0AADF811102C080E018C0D9
:1042A00029EF37E0B701A6018091F7079091F80751
:1042B0000E943C46882391F3C092F909D092FA09F2
:1042C000E092FB09F092FC0981E0C1118093F607AE
:1042D000CF91FF90EF90DF90CF9008958F929F92B3
:1042E000AF92BF92CF92DF92EF92FF920F931F9304
:1042F000CF93DF93EC016A017B01890189859A855F
:10430000AB85BC850196A11DB11D84179507A60735
:10431000B70710F480E054C08F89803129F49927C1
:10432000872F762F652F0BC08032A1F7CB01BA0102
:1043300027E096958795779567952A95D1F78B888D
:104340009C88AD88BE88680D791D8A1D9B1D809054
:10435000F9099090FA09A090FB09B090FC09681542
:1043600079058A059B0581F48F89803191F4DD24DC
:10437000EE24FF24F601EE0FFF1FE750F84F808177
:104380009181A0E0B0E016C040E070DF8111ECCF79
:10439000C1CFE894C7F8DD24EE24FF24F601EE0F28
:1043A000FF1FEE0FFF1FE750F84F80819181A28120
:1043B000B381BF70F80180839183A283B38381E0CE
:1043C000DF91CF911F910F91FF90EF90DF90CF90F1
:1043D000BF90AF909F908F9008954F925F926F9291
:1043E0007F92AF92BF92CF92DF92EF92FF920F93A4
:1043F0001F93CF93DF9300D01F92CDB7DEB78C0110
:1044000049835A836B837C835901C12CD12C76015B
:10441000412C42E0542E612C712C49815A816B81D0
:104420007C819E012F5F3F4FC80158DF882341F1F7
:10443000D301C201F801058404C0880F991FAA1F87
:10444000BB1F0A94D2F7C80ED91EEA1EFB1E498173
:104450005A816B817C818789803139F481E0483FC2
:104460005F4F6105710538F4D8CF81E0483F5F4F59
:104470006F4F7F4090F2F501C082D182E282F382D9
:104480000F900F900F900F90DF91CF911F910F9190
:10449000FF90EF90DF90CF90BF90AF907F906F90A4
:1044A0005F904F9008954F925F926F927F928F929C
:1044B0009F92AF92BF92CF92DF92EF92FF920F93B3
:1044C0001F93CF93DF93EC014A015B01280139016F
:1044D000423051056105710508F462C049855A856D
:1044E0006B857C854F5F5F4F6F4F7F4F4815590538
:1044F0006A057B0508F454C08F89803129F4FF24B4
:10450000EB2CDA2CC92C0CC0803209F049C07501A3
:10451000640177E0F694E794D794C7947A95D1F73D
:104520004B895C896D897E89C40ED51EE61EF71EF7
:1045300041E0C701B6019ADE882391F19F8990314D
:1045400059F49924AA24BB24F401EE0FFF1FE7506D
:10455000F84F5182408210C0E89487F89924AA2429
:10456000BB24F401EE0FFF1FEE0FFF1FE750F84FC3
:1045700040825182628273829A89923090F04D819A
:104580005E816F8178854C0D5D1D6E1D7F1D409392
:10459000F2075093F3076093F4077093F50701C097
:1045A00080E0DF91CF911F910F91FF90EF90DF900E
:1045B000CF90BF90AF909F908F907F906F905F90C3
:1045C0004F9008952F923F924F925F926F927F92F9
:1045D0008F929F92AF92BF92CF92DF92EF92FF9213
:1045E0000F931F93CF93DF93CDB7DEB72F970FB6FF
:1045F000F894DEBF0FBECDBF1C014C875D876E8770
:104600007F873B872A87DC0119960D911D912D919B
:104610003C911C970F5F1F4F2F4F3F4F0D831E8301
:104620002F833887EA85FB8580809180A280B380C4
:1046300081149104A104B10431F0FFEF8F1A9F0A95
:10464000AF0ABF0A10C0DC018D909D90AD90BC9068
:10465000B1E0B9870C851D852E853F850130110598
:104660002105310509F0198675016401412C512C91
:104670003201F10181859285A385B48548165906DA
:104680006A067B0608F04EC00D811E812F81388599
:104690000C151D052E053F0550F4F2E0CF2ED12C50
:1046A000E12CF12CA2E08A2E912CA12CB12C9E01A0
:1046B0002F5F3F4FB701A601C10110DE882391F1A2
:1046C00049815A816B817C81D701C6010196A11D68
:1046D000B11D452B462B472B19F04C015D010FC036
:1046E000AC01BD01481959096A097B090C851D8572
:1046F0002E853F85401751076207730741F01FEF72
:10470000411A510A610A710A6C017D01B2CF0FEFA3
:104710001FEF2FEF3FE0B701A601C101C4DE8D837B
:10472000811113C01D823DC02601370121E0421ACC
:1047300051086108710897018601B301A201C10106
:10474000B2DE882379F3730162018C149D04AE04F8
:10475000BF0450F3AA85BB854D915D916D917C910D
:104760004115510561057105A9F4EA85FB85808233
:104770009182A282B382F985FF2399F00FEF801A0C
:10478000900AA00AB00AD1018D929D92AD92BC927E
:10479000139707C095018401C10185DE8111E5CF22
:1047A000C1CF8D812F960FB6F894DEBF0FBECDBF5F
:1047B000DF91CF911F910F91FF90EF90DF90CF90FD
:1047C000BF90AF909F908F907F906F905F904F9031
:1047D0003F902F900895AF92BF92CF92DF92EF92C9
:1047E000FF920F931F93CF93DF9300D01F92CDB70B
:1047F000DEB75C016A017B0182E090E0A0E0B0E0FE
:10480000F50180839183A283B3839E012F5F3F4F85
:10481000B701A601C50162DD811102C080E023C09D
:1048200000E010E09801B701A601C5013CDE882335
:10483000A9F3C980DA80EB80FC80F501878980319B
:1048400049F481E0F8EFCF16FFEFDF06E104F10451
:1048500050F4DBCF81E098EFC9169FEFD906E90647
:104860009FE0F90690F20F900F900F900F90DF915C
:10487000CF911F910F91FF90EF90DF90CF90BF905D
:10488000AF9008957F928F929F92AF92BF92CF92F6
:10489000DF92EF92FF920F931F93CF93DF93EC0180
:1048A000142F7093F8076093F7071F8A82E090E057
:1048B000A0E0B0E088839983AA83BB831092F607B7
:1048C0001092F2071092F3071092F4071092F50776
:1048D0008FEF9FEFDC018093F9099093FA09A09381
:1048E000FB09B093FC09442349F1453008F0DEC0D0
:1048F00040E060E070E0CB01B9DC882309F4D6C069
:1049000020E1129FF0011124E955F64F80818F7745
:1049100009F0CCC084859585A685B7858436910538
:10492000A105B10508F4C2C0C084D184E284F38437
:10493000C114D104E104F10421F4B8C0C12CD12C7C
:10494000760140E0C701B60191DC782E882309F496
:10495000ADC080910408909105088115924009F03E
:10496000A5C030910908332309F4A0C0809107083D
:1049700090910808892B09F499C0209106082223F8
:1049800009F494C03A8B2C831D8630E041E050E05E
:104990006D85062FCA01062E02C0880F991F0A9442
:1049A000E2F72817390731F081E0860F8D876830EC
:1049B00078F37CC020910F08309110082115310543
:1049C00019F040E050E008C020911D0830911E0809
:1049D00040911F08509120082D833E834F835887B4
:1049E000809107089091080846015701880E991E8A
:1049F000A11CB11C8B8A9C8AAD8ABE8AE0910A08F0
:104A0000F0910B08F98FE88FA0910908B0E00E949F
:104A1000ADCC680D791D8A1D9B1D6A8F7B8F8C8F95
:104A20009D8FB5E0EE0FFF1FBA95E1F7E150FE4F05
:104A3000EF2FFF27E695DC01CB018E0F9F1FA11DF5
:104A4000B11D8E879F87A88BB98B80900C089090A2
:104A50000D088114910419F0A12CB12C08C080908C
:104A6000190890901A08A0901B08B0901C08A70184
:104A70009601281B390B4A0B5B0BDA01C901880D23
:104A8000991DAA1DBB1D04C0B695A795979587953E
:104A90000A95D2F789879A87AB87BC87853F3FE025
:104AA0009307A105B10520F48CE08F8B712C15C004
:104AB000853F9F4FA105B10510F480E10DC08091A5
:104AC000250890912608A0912708B09128088A8F80
:104AD0009B8FAC8FBD8F80E28F8B872DDF91CF9125
:104AE0001F910F91FF90EF90DF90CF90BF90AF900C
:104AF0009F908F907F9008954F925F926F927F92D8
:104B00008F929F92AF92BF92CF92DF92EF92FF92DD
:104B10000F931F93CF93DF932C0124E733E081E0C1
:104B200090E0F90145915491441655060CF062C08D
:104B3000AC0141505109DA01AA0FBB1FAA0FBB1FDC
:104B4000AE58BC4FFD0165917491440F551F440F41
:104B5000551F40595C4FFA0165907490FC01EE0FAF
:104B6000FF1FEE0FFF1FEE58FC4FA590B490FD0104
:104B700005911491F901C591D491FA018590949011
:104B8000882777FD8095982F0E9427C96B017C01AB
:104B9000B20166197709882777FD8095982F0E94C2
:104BA00027C92B013C01B501601B710B882777FDDC
:104BB0008095982F0E9427C99B01AC01C301B201C7
:104BC0000E945ACB2B013C01BE0168197909882744
:104BD00077FD8095982F0E9427C99B01AC01C301E6
:104BE000B2010E948CC89B01AC01C701B6010E94B2
:104BF000ACC711C001962C5F3F4F8D33910509F072
:104C000090CFE2E6F4E065917491882777FD809576
:104C1000982F0E9427C9DF91CF911F910F91FF908C
:104C2000EF90DF90CF90BF90AF909F908F907F904C
:104C30006F905F904F9008954F925F926F927F9226
:104C40008F929F92AF92BF92CF92DF92EF92FF929C
:104C50000F931F93CF93DF932C01662371F1EBE346
:104C6000F2E28491882341F09091C00095FFFCCF3F
:104C70008093C6003196F5CF70E04AE050E083EEB5
:104C80009FE00E945AA3E9E5F2E08491882341F075
:104C90009091C00095FFFCCF8093C6003196F5CF70
:104CA0008091C00085FFFCCF8AE08093C6000E94FF
:104CB000BB5060E070E0CB017EC024E733E081E0D0
:104CC00090E0F90145915491441655060CF062C0EC
:104CD000AC0141505109DA01AA0FBB1FAA0FBB1F3B
:104CE000AE58BC4FFD0165917491440F551F440FA0
:104CF000551F40595C4FFA0165907490FC01EE0F0E
:104D0000FF1FEE0FFF1FEE58FC4FA590B490FD0162
:104D100005911491F901C591D491FA01859094906F
:104D2000882777FD8095982F0E9427C96B017C0109
:104D3000B20166197709882777FD8095982F0E9420
:104D400027C92B013C01B501601B710B882777FD3A
:104D50008095982F0E9427C99B01AC01C301B20125
:104D60000E945ACB2B013C01BE01681979098827A2
:104D700077FD8095982F0E9427C99B01AC01C30144
:104D8000B2010E948CC89B01AC01C701B6010E9410
:104D9000ACC711C001962C5F3F4F8D33910509F0D0
:104DA00090CFE2E6F4E065917491882777FD8095D5
:104DB000982F0E9427C9DF91CF911F910F91FF90EB
:104DC000EF90DF90CF90BF90AF909F908F907F90AB
:104DD0006F905F904F90089560E08091520A90919B
:104DE000530A2ADF60934E0A70934F0A8093500A49
:104DF0009093510A80914C0A90914D0A7DDE609308
:104E0000480A7093490A80934A0A90934B0A8FB7D5
:104E1000F8941092400A8FBF0895209114023091A7
:104E20001502409116025091170260E070E08FE782
:104E300093E40E948CC86093200A7093210A8093A7
:104E4000220A9093230A089597FF03C08091470A8E
:104E500004C0FC01E65EF54F808190E00895CF9399
:104E6000DF93D82FC62FC19561E00E9436C26C2F08
:104E70008D2F0E946FC26C2F70E08D2FDF91CF912C
:104E80000C942CC1CF93C1E020E030E048E452E420
:104E900060914E0A70914F0A8091500A9091510A88
:104EA0000E9488CA18160CF0C0E06C2F86E090E0D3
:104EB000CF91D5CF2F923F924F925F926F927F9278
:104EC0008F929F92AF92BF92CF92DF92EF92FF921A
:104ED0000F931F93CF93DF93CDB7DEB728970FB60D
:104EE000F894DEBF0FBECDBF8091400A882309F43D
:104EF000F8C172DF80904E0A90904F0AA090500A3D
:104F0000B090510A0091560A1091570AB8018827AB
:104F100077FD8095982F0E9427C9A50194010E94D2
:104F2000ABC76B017C016093280A7093290A8093B8
:104F30002A0A90932B0A20E030E040E251E40E94DC
:104F400088CA181624F481E080931F0AF7C020E075
:104F500030E040E251ECC701B6010E9485C887FDF0
:104F600002C0012B21F481E080931F0A0CC18091C3
:104F70001F0A882351F010923C0A10923D0A1092A9
:104F80003E0A10923F0A10921F0A20911802309197
:104F9000190240911A0250911B02C701B6010E94EA
:104FA0005ACB69837A838B839C836093340A709392
:104FB000350A8093360A9093370A20913C0A309143
:104FC0003D0A40913E0A50913F0AC701B6010E9436
:104FD000ACC72B013C012090240A3090250A109187
:104FE000260A0091270A9101412F502F0E9485C85F
:104FF00087FD14C02090200A3090210A1091220AC7
:105000000091230A9101412F502FB201C3010E9448
:1050100088CA18161CF01201162D072DC101A12FE8
:10502000B02F80933C0A90933D0AA0933E0AB09320
:105030003F0A2091140230911502409116025091BE
:105040001702B101812F902F0E945ACB6D837E836E
:105050008F8398876093300A7093310A8093320A65
:105060009093330A2091380A3091390A40913A0AD4
:1050700050913B0AC501B4010E94ABC720911002B8
:105080003091110240911202509113020E945ACBAA
:1050900020ED3CEC4CE45DE30E945ACB2B013C013B
:1050A00023E333E343E75FE360912C0A70912D0A19
:1050B00080912E0A90912F0A0E945ACB9B01AC013D
:1050C000C301B2010E94ACC72B013C0160932C0AC2
:1050D00070932D0A80932E0A90932F0A2D813E8182
:1050E0004F81588569817A818B819C810E94ACC7F0
:1050F000A30192010E94ABC72B013C0120E030E0EC
:105100004FE753E40E9488CA20E030E0A901181656
:10511000E4F4C701B6010E9488CA18167CF4A701FE
:105120009601B101812F902F0E94ABC760933C0A7A
:1051300070933D0A80933E0A90933F0A412C512C74
:105140009FE7692E93E4792E21C0C301B2010E942A
:1051500085C887FF1BC020E030E0A901C701B60168
:105160000E9485C887FF0FC0A7019601B101812F5A
:10517000902F0E94ABC760933C0A70933D0A8093C6
:105180003E0A90933F0A412C512C32018092380AFA
:105190009092390AA0923A0AB0923B0A6091120AA0
:1051A0007091130A882777FD8095982F0E9427C950
:1051B0009B01AC01C501B4010E9488CA1816DCF439
:1051C0006091080270910902882777FD8095982FD9
:1051D0000E9427C99B01AC01C501B4010E9485C88A
:1051E00087FF09C0C301B2010E94F4C87595679595
:1051F00060931A0A02C010921A0A0E9416C3009104
:10520000160A1091170A2091180A3091190A601B8A
:10521000710B820B930B653C79408105910558F029
:1052200031DE0E9416C36093160A7093170A8093AA
:10523000180A9093190A0E9416C300911B0A109134
:105240001C0A20911D0A30911E0A601B710B820BF3
:10525000930B683873418105910508F442C00E94A0
:1052600016C360931B0A70931C0A80931D0A9093C7
:105270001E0AC090480AD090490AE0904A0AF0906D
:105280004B0A20E030E040E751E4C701B6010E943C
:1052900088CA18161CF520E030E046E153E4C70147
:1052A000B6010E9485C887FF19C06091540A7091A9
:1052B000550A882777FD8095982F0E9427C99B0162
:1052C000AC01C701B6010E9488CA87FD03C01092D5
:1052D000470A07C08FE78093470A03C01092470A26
:1052E000A59828960FB6F894DEBF0FBECDBFDF910C
:1052F000CF911F910F91FF90EF90DF90CF90BF90D3
:10530000AF909F908F907F906F905F904F903F9065
:105310002F900895CF93DF931092240A1092250ABC
:105320001092260A1092270A209114023091150239
:10533000409116025091170260E070E08FE793E40D
:105340000E948CC86093200A7093210A8093220ADD
:105350009093230A6D9A80910101806180930101ED
:105360009D9A8091010180628093010187ED809375
:105370007A0010927E0010927D0080917E00816004
:1053800080937E0080917E00826080937E00809179
:105390007E00846080937E0080E888BD80916E00EE
:1053A000846080936E006AEF70E080E090E00E947D
:1053B00045C38FE090E09093130A8093120A60E057
:1053C00080910A0290910B0237DC20E030E040E748
:1053D00051E40E9485C887FF0AC080910A0290911B
:1053E0000B02409790930B0280930A02E8CF8BE365
:1053F00091E0909309028093080260E08091140A82
:105400009091150A19DC20E030E84DE953E40E9440
:1054100088CA181654F48091140A9091150A40967F
:105420009093150A8093140AE8CFC091100AD09186
:10543000110ACE0161DB20E030E046E153E40E9436
:1054400088CA181634F46096D093110AC093100AD3
:10545000ECCFDF91CF91089508951092570A1092E2
:10546000560A1092550A1092540A10921A0A759808
:105470001092550A1092540A1092470AA59808955E
:105480002F923F924F925F926F927F928F929F9254
:10549000AF92BF92CF92DF92EF92FF920F931F9342
:1054A000CF93DF93CDB7DEB7AE970FB6F894DEBFDC
:1054B0000FBECDBF6B8F7C8F8D8F292E5A8749876A
:1054C0003CA72BA70E9416C36F8F78A389A39AA32A
:1054D0000E9416C36FA378A789A79AA729853A8542
:1054E000121613061CF0E4EAF6E017C0E7EBF6E04C
:1054F0008191882339F09091C00095FFFCCF809373
:10550000C600F6CF8091C00085FFFCCF1BC29091F2
:10551000C00095FFFCCF8093C60081918111F7CF29
:105520008091C00085FFFCCF8AE08093C60095DFA4
:1055300049855A858FE7452B99F18093470A8F8DCE
:1055400098A1A9A1BAA1898B9A8BAB8BBC8B8D87B3
:105550009E87AF87B88B1D8290E4988FACE1A98FAE
:10556000B6E4BA8F1DA61D8A1E8A1F8A2FE730E077
:1055700040E050E029833A834B835C83EFE74E2E73
:10558000512C612C712C1BA21CA21DA21EA231E069
:105590003E8F1C861B86312C00E010E01EA605C045
:1055A00080931A0ACCCF0E9497848091400A882366
:1055B00009F4F6C011DC49855A85452B51F030902D
:1055C000480A0091490A10914A0A50914B0A5EA775
:1055D00009C030904E0A00914F0A1091500A8091F4
:1055E000510A8EA7232D302F412F5EA56DA57D89F1
:1055F0008E899F890E9488CA18162CF03DA60D8BB3
:105600001E8B9EA59F8B232D302F412F5EA56D8174
:10561000788D898D9A8D0E9485C887FD05C03D8251
:10562000088F198FAEA5AA8F0E9416C32FA138A587
:1056300049A55AA5621B730B840B950B653C7940F9
:105640008105910538F01EDC0E9416C36FA378A770
:1056500089A79AA74E8D442309F44FC02B8D3C8D0A
:105660004D8D522D632D702F812F9EA50E9488CACB
:1056700018160CF095C00E9416C329893A894B89E7
:105680005C89621B730B840B950B69387341810530
:10569000910508F485C0D301C20129813A814B816B
:1056A0005C81821B930BA40BB50B49855A85B5957C
:1056B000A79597958795452B19F08093470A02C0C7
:1056C00080931A0A0E9416C36D877E878F87988BF6
:1056D000DC01CB0129893A894B895C89821B930BB8
:1056E000A40BB50B8BA39CA3ADA3BEA33B8D3DA781
:1056F0004C8D4D8B5D8D5E8B2F8A2B8D3C8D4D8D12
:10570000522D632D702F812F9EA50E9485C887FF83
:10571000EEC20E9416C32D853E854F855889621BB7
:10572000730B840B950B693873418105910508F45F
:10573000DEC20E9416C3698B7A8B8B8B9C8BDC013B
:10574000CB012D853E854F855889821B930BA40B79
:10575000B50B4B855C85452B09F010C189819A8179
:10576000AB81BC81840D951DA61DB71D29853A8589
:10577000B595A79597958795232B09F4B5C2809386
:10578000470A4B855C854F5F5F4F5C874B875B8D1E
:105790005D838C8D888F9D8D998F2A8EA1E0AE8F31
:1057A00020E030E040EA51E46B8D7C8D8D8D922DB0
:1057B0000E94ACC79B01AC01632D702F812F9EA569
:1057C0000E9488CA181694F4EFEFF2E084918823BF
:1057D00041F09091C00095FFFCCF8093C6003196B8
:1057E000F5CF8091C00085FFFCCFACC00E9416C3EE
:1057F0002F8D38A149A15AA1621B730B840B950B05
:10580000613D77408105910508F44FC049855A856F
:10581000452B81F0E090470AF12CE9EFF2E084910A
:105820008823C1F09091C00095FFFCCF8093C60003
:105830003196F5CFE0901A0AF12CE3EFF2E0849173
:10584000882341F09091C00095FFFCCF8093C60063
:105850003196F5CF22E030E0432D502F612F7EA509
:1058600083EE9FE00E9430A4EFEEF2E08491882363
:1058700041F09091C00095FFFCCF8093C600319617
:10588000F5CF4AE050E0B70183EE9FE00E945AA3B3
:105890008091C00085FFFCCF8AE08093C6000E9403
:1058A00016C36F8F78A389A39AA30E9416C36B01B6
:1058B0007C010E9416C389889A88AB88BC882D8594
:1058C0003E854F855889820E931EA41EB51EC818AA
:1058D000D908EA08FB08C60ED71EE81EF91E31E8F3
:1058E000C3163FE4D30632E1E306F10490F0E2EDA3
:1058F000F2E08491882341F09091C00095FFFCCFA5
:105900008093C6003196F5CF8091C00085FFFCCF13
:1059100019C04B855C858BA59CA5841795070CF059
:1059200042CEE6E7F2E08491882341F09091C000F6
:1059300095FFFCCF8093C6003196F5CF8091C000D3
:1059400085FFFCCF8AE08093C600AE960FB6F89430
:10595000DEBF0FBECDBFDF91CF911F910F91FF90A2
:10596000EF90DF90CF90BF90AF909F908F907F90FF
:105970006F905F904F903F902F9008958BA09CA0C8
:10598000ADA0BEA0880E991EAA1EBB1E2BA13CA1D5
:105990004DA15EA1281B390B4A0B5B0BCA01B90153
:1059A00029813A814B815C810E9420CCA501940120
:1059B0000E9485CC240D351D461D571D243131050F
:1059C0004105510504F129013A013CEE4316510409
:1059D000610471042CF06BEE462E512C612C712C5D
:1059E00040E84416510461047104DCF08EEF90E04D
:1059F000A0E0B0E084199509A609B70989839A83C4
:105A0000AB83BC8312C054E1452E512C612C712C08
:105A100024E130E040E050E029833A834B835C830B
:105A200004C049825A826B827C82E8E6F3E084916A
:105A3000882341F09091C00095FFFCCF8093C60071
:105A40003196F5CF2AE030E0B301A20183EE9FE06A
:105A50000E942FA3E3E6F3E08491882341F0909124
:105A6000C00095FFFCCF8093C6003196F5CF2AE0A9
:105A700030E049815A816B817C8183EE9FE00E94F6
:105A80002FA3ECE5F3E08491882341F09091C000CE
:105A900095FFFCCF8093C6003196F5CF22E030E031
:105AA0004D81588D698D7A8D83EE9FE00E9430A4E0
:105AB000E5E5F3E08491882341F09091C00095FFE3
:105AC000FCCF8093C6003196F5CF22E030E04DA5A3
:105AD0005D896E897F8983EE9FE00E9430A480916A
:105AE000C00085FFFCCF8AE08093C6002B853C85F3
:105AF000233031050CF432CE69817A818B819C810F
:105B00000E9427C920E030E040E850E40E945ACBD0
:105B10006B017C012D81388D498D5A8D6DA57D8954
:105B20008E899F890E94ABC720ED3FE049E450E495
:105B30000E945ACB20E030E040E05FE30E945ACB65
:105B40009B01AC01C701B6010E948CC86B017C01AE
:105B5000C501B4010E9427C920E030E04AE754E4BF
:105B60000E948CC84B015C01EFE4F3E08491882330
:105B700041F09091C00095FFFCCF8093C600319614
:105B8000F5CF22E030E0B701A60183EE9FE00E944E
:105B900030A4E9E4F3E08491882341F09091C000BF
:105BA00095FFFCCF8093C6003196F5CF22E030E020
:105BB000B501A40183EE9FE00E9430A48091C00053
:105BC00085FFFCCF8AE08093C6002AE939E949E1E4
:105BD0005FE3C701B6010E945ACB6B017C019B01B8
:105BE000AC010E94ACC7A50194010E948CC86D83D2
:105BF0007E838F839887A5019401C701B6010E9417
:105C00005ACB20E030E040E05EE30E945ACB4B01EB
:105C10005C01EBE3F3E08491882341F09091C000B4
:105C200095FFFCCF8093C6003196F5CF8091C000E0
:105C300085FFFCCF8AE08093C600E5E3F3E0849122
:105C4000882341F09091C00095FFFCCF8093C6005F
:105C50003196F5CF22E030E0B701A60183EE9FE058
:105C60000E9430A48091C00085FFFCCF8AE0809321
:105C7000C600EFE2F3E08491882341F09091C000E8
:105C800095FFFCCF8093C6003196F5CF22E030E03F
:105C90004D815E816F81788583EE9FE00E9430A404
:105CA0008091C00085FFFCCF8AE08093C600E9E2C6
:105CB000F3E08491882341F09091C00095FFFCCFE0
:105CC0008093C6003196F5CF22E030E0B501A40103
:105CD00083EE9FE00E9430A48091C00085FFFCCF3E
:105CE0008AE08093C6003ACD80931A0A4ACD1E8E70
:105CF00057CDCF93C82FB1DB0E940A56811134C013
:105D0000EBE3F2E29491992341F08091C00085FF8A
:105D1000FCCF9093C6003196F5CF6C2F70E04AE02F
:105D200050E083EE9FE00E945AA38091C00085FF5F
:105D3000FCCF8AE08093C600ECE2F2E084918823F5
:105D400041F09091C00095FFFCCF8093C600319642
:105D5000F5CF8091C00085FFFCCF8AE08093C6001C
:105D60008FE192E00E94F583CF910C94B255CF93CE
:105D7000C82F73DB0E940A56811134C0EBE3F2E2B4
:105D80009491992341F08091C00085FFFCCF9093BE
:105D9000C6003196F5CF6C2F70E04AE050E083EEFC
:105DA0009FE00E945AA38091C00085FFFCCF8AE04B
:105DB0008093C600E2EFF1E08491882341F0909156
:105DC000C00095FFFCCF8093C6003196F5CF80913F
:105DD000C00085FFFCCF8AE08093C60085EE91E08D
:105DE0000E94F583CF910C94B255A5980E940A5653
:105DF000811125C0EBE3F2E28491882341F0909178
:105E0000C00095FFFCCF8093C6003196F5CFEBEA3A
:105E1000F1E08491882341F09091C00095FFFCCF80
:105E20008093C6003196F5CF8091C00085FFFCCFEE
:105E30008AE08093C6008AE991E00E94F5830C9481
:105E4000B2551F920F920FB60F9211240BB60F92FC
:105E50000F931F932F933F934F935F936F937F9372
:105E60008F939F93AF93BF93CF93DF93EF93FF9362
:105E700080910702811112C080911A0A80930F0A43
:105E8000882311F0759A01C075988091470A809314
:105E90000E0A882311F0A59A01C0A59890910F0AC7
:105EA00080910702981708F4759890910E0A8091D6
:105EB0000702981708F4A598809107028F5F8F77E3
:105EC000809307028091060290E08B30910508F0E4
:105ED00093C0FC01EE58FF4F0C94A1CC10927B00B4
:105EE00080E480937C0080917A00806480937A00C3
:105EF0000E94FE8381E019C02091780030917900E2
:105F000080910A0A90910B0AA0910C0AB0910D0A97
:105F1000820F931FA11DB11D80930A0A90930B0A53
:105F2000A0930C0AB0930D0A82E08093060264C02D
:105F300010927B0082E480937C0080917A008064E0
:105F400080937A000E94FE8383E0EFCF2091780057
:105F5000309179008091060A9091070AA091080A71
:105F6000B091090A820F931FA11DB11D8093060AEB
:105F70009093070AA093080AB093090A84E0D5CF4A
:105F800010927B0081E480937C0080917A00806491
:105F900080937A000E94FE8385E0C7CF209178002D
:105FA000309179008091020A9091030AA091040A2D
:105FB000B091050A820F931FA11DB11D8093020AA3
:105FC0009093030AA093040AB093050A86E0ADCF2C
:105FD0000E94FE8387E0A9CF88E0A7CF0E94FE83BE
:105FE00089E0A3CF109206028091010A8F5F80930F
:105FF000010A02C0109206028091010A803108F461
:1060000063C08091400A811110C080910A0A90916A
:106010000B0A9093530A8093520A8091060A90913A
:10602000070A90934D0A80934C0A81E08093400ABE
:106030001092010A10920A0A10920B0A10920C0A8E
:1060400010920D0A1092020A1092030A1092040A8A
:106050001092050A1092FD091092FE091092FF0994
:106060001092000A1092060A1092070A1092080A6B
:106070001092090A2091520A3091530A8091140A11
:106080009091150A8217930714F080E032DE209178
:10609000520A3091530A80910A0290910B022817FC
:1060A000390714F080E063DE20914C0A30914D0AEC
:1060B0008091100A9091110A821793072CF0109288
:1060C000550A1092540A91DE00E010E0E801CC0F6E
:1060D000DD1FCF5BD54F888199811816190644F4CE
:1060E00061E0802F0E9446AD88819981019709C0A7
:1060F000892B49F060E0802F0E9446AD888199810C
:106100000196998388830F5F1F4F03301105F1F6C5
:10611000FF91EF91DF91CF91BF91AF919F918F91BF
:106120007F916F915F914F913F912F911F910F91AF
:106130000F900BBE0F900FBE0F901F9018952CEA7A
:1061400035EC47E25EE30C945ACB2CEA35EC47E29F
:106150005EE30C948CC82CEA35EC47E25EE30C94C9
:106160008CC82CEA35EC47E25EE30C945ACBCF9313
:10617000DF93EC0160E08E810E946FC281E090E0CD
:106180000E9469C361E08E810E946FC281E090E04D
:106190000E9469C360E08E810E946FC284E690E035
:1061A000DF91CF910C9469C3CF92DF92EF92FF926F
:1061B0000F931F93CF93DF937C01C0E0D0E0C62EF6
:1061C000D12C87010C0F1D1F61E0F80187810E940F
:1061D00036C2B6010C2E02C0759567950A94E2F797
:1061E0006170F80187810E946FC22196C430D10589
:1061F00041F7C701DF91CF911F910F91FF90EF9071
:10620000DF90CF90B4CFCF92DF92EF92FF920F93B7
:106210001F93CF93DF937C01C0E0D0E0C62ED12C3A
:1062200087010C0F1D1F61E0F80187810E9436C2B3
:10623000B6010C2E02C0759567950A94E2F761705D
:10624000F80187810E946FC22196C830D10541F7BD
:10625000C701DF91CF911F910F91FF90EF90DF90D9
:10626000CF9085CF1F93CF93DF93EC01162F642F30
:106270008C810E946FC28D818F3F19F060E00E9477
:106280006FC28F85612F84FF05C0CE01DF91CF9152
:106290001F91B9CF70E084E0759567958A95E1F715
:1062A000CE0182DF612FCE01DF91CF911F917CCF94
:1062B00040E0D8CF61E0FCDF80E496E00C9469C355
:1062C00062E0F6DF80E496E00C9469C3CF93DF933D
:1062D000CDB7DEB728970FB6F894DEBF0FBECDBF9F
:1062E00028E0EFE1F6E0DE01119601900D922A958B
:1062F000E1F7FC012389421710F04FEF420FFE0136
:106300003196E40FF11DE40FF11D2081260F206866
:10631000622F28960FB6F894DEBF0FBECDBFDF9177
:10632000CF91C6CFFC016089262F2460208B6C6042
:10633000BFCFCF93DF93EC01423018F08F85886098
:106340008F874B8B1C8A222329F0413019F48F85CB
:1063500084608F8780E593EC0E9469C360E08C8144
:106360000E946FC260E08E810E946FC28D818F3F5C
:1063700019F060E00E946FC26F8564FD19C063E090
:10638000CE0112DF84E991E10E9469C363E0CE018E
:106390000BDF84E991E10E9469C363E0CE0104DF71
:1063A00086E990E00E9469C362E0CE01FDDE13C081
:1063B0006062CE017DDF84E991E10E9469C36F854F
:1063C0006062CE0175DF86E990E00E9469C36F8547
:1063D0006062CE016DDF6F856062CE0169DF8CE3A4
:1063E00090E00E9469C384E0888BCE019BDF8CE340
:1063F00090E00E9469C3CE015DDF88EB9BE00E94C4
:1064000069C382E0898B66E0CE0152DF8CE390E0C5
:10641000DF91CF910C9469C36F927F928F92AF926C
:10642000CF92EF920F931F93CF93DF93CDB7DEB749
:106430003C01162F842F5E854F8538899989F30199
:10644000848325830683E782C086A186828653875C
:1064500044873587968761E00E9436C2F3018581C3
:106460008F3F19F061E00E9436C261E0F30186813E
:106470000E9436C2112319F0F301178603C080E190
:10648000F301878720E041E060E1C301DF91CF9114
:106490001F910F91EF90CF90AF908F907F906F9062
:1064A00048CF8F92AF92CF92EF920F93DC01139669
:1064B0001C921E921297E5EEF6E0ED93FC931F926C
:1064C0001F921F921F928C2CAE2CC02EE22E042FF6
:1064D0002FEF462F61E0A0DF0F900F900F900F90ED
:1064E0000F91EF90CF90AF908F900895CF93DF935F
:1064F000EC01423018F08F8588608F874B8B1C8AA7
:10650000222329F0413019F48F8584608F8780E53C
:1065100093EC0E9469C360E08C810E946FC260E0CE
:106520008E810E946FC28D818F3F19F060E00E94C2
:106530006FC26F8564FD19C063E0CE0135DE84E96A
:1065400091E10E9469C363E0CE012EDE84E991E10E
:106550000E9469C363E0CE0127DE86E990E00E94D5
:1065600069C362E0CE0120DE13C06062CE01A0DE0E
:1065700084E991E10E9469C36F856062CE0198DE73
:1065800086E990E00E9469C36F856062CE0190DE6B
:106590006F856062CE018CDE8CE390E00E9469C35F
:1065A00084E0888BCE01BEDE8CE390E00E9469C35C
:1065B000CE0186DE80E496E00E9469C382E0898B8A
:1065C00066E0CE0175DE8CE390E00E9469C340E096
:1065D00068E0CE017BDE6FEB77E0CE010E94A3C7BF
:1065E00041E068E0CE0172DE6FEB77E0CE010E9401
:1065F000A3C742E066E0CE0169DE6DEB77E0CE0135
:10660000DF91CF910C94A3C7CF92DF92EF92FF92CC
:106610000F931F93CF93DF931F921F92CDB7DEB7D7
:106620008C01677088E0689FB00111246064C80124
:1066300049835A833DDE4981C42E5A81D52EE12CEF
:10664000F12CD6016D916D01D801ED91FC91019075
:10665000F081E02DC8011995BFEFEB1AFB0AE8E0C5
:10666000EE16F10471F70F900F90DF91CF911F910B
:106670000F91FF90EF90DF90CF90089541E0F2DD11
:1066800081E090E008950F931F93CF93DF93EC0187
:106690008B0144E150E0BC0188E59AE00E94ADCF57
:1066A000CE010E948CCF992744E150E0481B590B42
:1066B000B801885A954F0E94ADCF88E59AE0DF91E6
:1066C000CF911F910F910895AF92BF92CF92DF9219
:1066D000EF92FF920F931F93CF93DF93EC015B0137
:1066E0007A01690144E150E0BC0188E59AE00E942A
:1066F000ADCFCE010E948CCFEC01DD2704E110E08C
:10670000A8014C1B5D0BB501CE01885A954F0E9424
:10671000ADCFC5010E948CCFC80FD91FDD27A801BE
:106720004C1B5D0BB701CE01885A954F0E94ADCF2F
:10673000C7010E948CCF8C0F9D1F9927A801481B71
:10674000590BB601885A954F0E94ADCF88E59AE063
:10675000DF91CF911F910F91FF90EF90DF90CF903D
:10676000BF90AF9008952F923F924F925F926F9299
:106770007F928F929F92AF92BF92CF92DF92EF92D1
:10678000FF920F931F93CF93DF93CDB7DEB7CF5414
:10679000D1090FB6F894DEBF0FBECDBF1C017E8FAE
:1067A0006D8F4A012FAB09AF2896EFAE28972C9634
:1067B000ACAEBDAECEAEDFAE2C9734E0239F500121
:1067C0001124FC01EA0DFB1D80819181A281B3811E
:1067D000898F9A8FAB8FBC8FDA01AA0DBB1DBCAF1E
:1067E000ABAF4D905D906D907C90A3019201698D4F
:1067F0007A8D8B8D9C8D0E94ACC721966CAF7DAF3E
:106800008EAF9FAF2197B4E00B9F80011124F1015F
:10681000E00FF11F20813181428153812F8F38A3F6
:1068200049A35AA3A401400F511F23965FAF4EAF57
:106830002397DA01CD90DD90ED90FC90A7019601B1
:106840006F8D78A189A19AA10E94ACC727966CAFE1
:106850007DAF8EAF9FAF27972896EFAD2897B4E016
:10686000EB9FC0011124F101E80FF91F2081318154
:10687000428153812BA33CA34DA35EA3ED8DFE8DDE
:10688000E80FF91F60817181828193810E94ABC7FB
:106890006FA378A789A79AA7AD8DBE8D1C968D9101
:1068A0009D910D90BC91A02D60968CAF9DAFAEAF29
:1068B000BFAF6097D1011C962D913D914D915C9198
:1068C0001F972BA73CA74DA75EA7A3019201505885
:1068D0002D8B3E8B4F8B588FD701C601B058898BBB
:1068E0009A8BAB8BBC8BED8DFE8DEA0DFB1D208151
:1068F0003181428153812FA738AB49AB5AAB2196E6
:106900002CAD3DAD4EAD5FAD21976FA578A989A99E
:106910009AA90E94ABC76B017C01ED8DFE8DE00F43
:10692000F11F80819181A281B3818BAB9CABADAB18
:10693000BEAB27962CAD3DAD4EAD5FAD2797BC01EC
:10694000CD010E94ABC74B015C01A70196016D8987
:106950007E898F89988D0E945ACB2B013C01A5011D
:10696000940169897A898B899C890E945ACB9B0101
:10697000AC01C301B2010E94ACC72B013C01A501CF
:1069800094016D897E898F89988D0E945ACB4B0125
:106990005C01A701960169897A898B899C890E948B
:1069A0005ACB9B01AC01C501B4010E94ABC7A30146
:1069B00092010E941FC86B017C0120E030E0A90118
:1069C0000E9485C887FF0AC02BED3FE049EC50E4E8
:1069D000C701B6010E94ACC76B017C01AA968FADBE
:1069E000AA97882351F02BED3FE049EC50E4C70112
:1069F000B6010E94ABC76B017C012FA538A949A93C
:106A00005AA9698D7A8D8B8D9C8D0E9485C88111C4
:106A10001FC02BA93CA94DA95EA96F8D78A189A1A2
:106A20009AA10E9485C8811113C020E030E0A9011D
:106A3000C701B6010E9485C881110AC02BED3FE055
:106A400049EC50E4C701B6010E94ACC76B017C0160
:106A5000A9962CAD3DAD4EAD5FADA997C701B6016E
:106A60000E945ACB2FA138A549A55AA55F770E944D
:106A700095CA4B015C012FE632E143E85AE30E94DC
:106A800085C887FDC8C1C501B4010E9462C90E94C2
:106A9000F9C87A8F698FDB01AB2B21F4E1E0F0E0DC
:106AA000FA8FE98F298D3A8DB90180E090E00E943C
:106AB00025C94B015C019B01AC01C701B6010E94D5
:106AC0008CC82B013C01A50194016FA178A589A573
:106AD0009AA50E948CC86FA778AB89AB9AAB2BA5FF
:106AE0003CA54DA55EA560966CAD7DAD8EAD9FAD10
:106AF00060970E94ABC7A50194010E948CC86BAB44
:106B00007CAB8DAB9EAB20E030E040E05FE3C301A7
:106B1000B2010E945ACBA30192010E945ACB9B0161
:106B2000AC0160E070E080E89FE30E94ABC76FA318
:106B300078A789A79AA7CE010196FC0128964FADA8
:106B4000289734E0439FE00DF11D11242BA13CA1B7
:106B50004DA15EA120833183428353832BA53CA5A5
:106B60004DA55EA52D873E874F87588BB12C41E000
:106B700050E058A34F8F1C01BFA9A4E0BA9F800D1D
:106B8000911D112498AF8FAB910159AD44E0549FF2
:106B9000200D311D11243AAF29AFFCA7EBA74F8D73
:106BA00058A1898D9A8D4817590708F01AC188E1B4
:106BB0008B150CF444C02FA138A549A55AA56989A5
:106BC0007A898B899C890E945ACB6B017C01A30135
:106BD00092016D897E898F89988D0E945ACBA70179
:106BE00096010E94ACC7A62E172F982E892E2FA192
:106BF00038A549A55AA56D897E898F89988D0E94EF
:106C00005ACB6B017C01A301920169897A898B8936
:106C10009C890E945ACB9B01AC01C701B6010E941E
:106C2000ABC76D8B7E8B8F8B988FB3948A2D912FF2
:106C3000A92DB82D898B9A8BAB8BBC8B6CC0AF8D7B
:106C4000B8A1BD0180E090E00E9425C9A301920196
:106C50000E945ACB6B017C010E9489C8698B7A8B98
:106C60008B8B9C8BC701B6010E94BDCB4B015C0195
:106C7000EBADFCADC080D180E280F380F7FAF094F8
:106C8000F7F8F0942396AEADBFAD23972D913D91CB
:106C90004D915C912BA33CA34DA35EA329893A8916
:106CA0004B895C89C701B6010E945ACB6D8B7E8BE4
:106CB0008F8B988FA50194016BA17CA18DA19EA1C2
:106CC0000E945ACB9B01AC016D897E898F89988D7A
:106CD0000E94ACC76D8B7E8B8F8B988FA501940122
:106CE000C701B6010E945ACB6B017C0129893A8900
:106CF0004B895C896BA17CA18DA19EA10E945ACB7E
:106D00009B01AC01C701B6010E94ABC7698B7A8BAE
:106D10008B8B9C8BB12C2D893E894F89588D219668
:106D20006CAD7DAD8EAD9FAD21970E94ACC7EFA934
:106D3000F8AD608371838283938329893A894B8973
:106D40005C8927966CAD7DAD8EAD9FAD27970E9477
:106D5000ACC7A9ADBAAD6D937D938D939C931397FA
:106D60002FA538A949A95AA9EBA5FCA56081718175
:106D7000828193810E94ACC7ABA5BCA56D937D9326
:106D80008D939C9313972BA93CA94DA95EA96D8562
:106D90007E858F8598890E94ACC76D877E878F8797
:106DA000988BC1010E94034DFE01E659FF4F6F0110
:106DB0002C96ECACFDAC0EAD1FAD2C979E01235F65
:106DC0003F4FAE01475F5F4FBE016B5F7F4FC10119
:106DD0000E9441B42F8D38A12F5F3F4F38A32F8FD2
:106DE000DECE2D8D3E8D245F3F4F4D8D5E8D485FF5
:106DF0005F4F6D8D7E8D6C5F7F4FDE01A659BF4F5B
:106E00006D012C96ECACFDAC0EAD1FAD2C978D8DAD
:106E10009E8D0E9441B4C15BDF4F0FB6F894DEBF78
:106E20000FBECDBFDF91CF911F910F91FF90EF90DB
:106E3000DF90CF90BF90AF909F908F907F906F909A
:106E40005F904F903F902F900895FC01148217821D
:106E5000138212828CED97E09183808308952CED4C
:106E600037E0FC01318320832781222319F0049627
:106E70000C94741C0895CF92DF92EF92FF920F93BF
:106E80001F93CF93DF93EC01875B9F4FDEDFCE0133
:106E900086599F4FDADF7E0129E8E20EF11C870157
:106EA0006E0131E4C31A3EEFD30AC801CEDF015EA2
:106EB0001F4F0C151D05C9F7FE01EF53FE4F89E169
:106EC000818314823596178ACE018C519E4FBDDF87
:106ED000FE01EB56FD4F108211821282138238960A
:106EE00010821182128213821A821B8218821982E6
:106EF0006E0187E6C81A8DEFD80AF601108211825A
:106F000012821382F80111821082FE01ED5FFD4FA3
:106F1000108286E391E0F7019C01119221503040EC
:106F2000E1F7FE01EF55FD4F81E08083C95BDF4F44
:106F3000198218820E9416C368577C4E8F4F9F4F4C
:106F4000F6016083718382839383DF91CF911F91D8
:106F50000F91FF90EF90DF90CF900895FC0120E01B
:106F60003EE2DB014C91403241F0283011F4308395
:106F70003196DB014C91408331962F5F6F5F7F4FDD
:106F80002B3079F7108208952F923F924F925F92A3
:106F90006F927F928F929F92AF92BF92CF92DF9229
:106FA000EF92FF920F931F93CF93DF93CDB7DEB78E
:106FB000CA58D1090FB6F894DEBF0FBECDBF8C0101
:106FC0006B017A014901CA57DF4F1882C658D04079
:106FD00084E0E80EF11C180191E1290E311CF80142
:106FE000EA5BFF4FC957DF4FF983E883C758D040AA
:106FF0003801FEE56F1AFDEF7F0A58018CE5A81AEB
:107000008DEFB80A90E4492E512C4C0E5D1E94E091
:10701000490E511CA101BE016F5F7F4FC7010E9445
:10702000DE1A18160CF04AC12C85322F3871303117
:1070300009F0ACC0F301808191810197029708F4B7
:10704000A5C0BE016F5F7F4FCE0187589F4F86DF7F
:10705000A0961FAEA097F6018081811107C069EE4E
:1070600076E0CE01815A9F4F0E9406D0B601CE0134
:10707000815A9F4F0E9406D0BE0167587F4FCE01B4
:10708000815A9F4F0E9406D069EE76E0CE01815A68
:107090009F4F0E9406D0CE01805C9F4FD6DE21E03C
:1070A000AE0147585F4FB701C2010E946B1E8111AC
:1070B00047C0F30180819181892B09F041C0E5E34C
:1070C000F2E28491882341F09091C00095FFFCCFBB
:1070D0008093C6003196F5CFE091780CF0E0EE0F8A
:1070E000FF1FE45EFD4F0190F081E02DEA57FE4F57
:1070F0000190F081E02D8191882339F09091C000BA
:1071000095FFFCCF8093C600F6CF8091C00085FF2D
:10711000FCCF8AE08093C600FE01E758FF4F8191C3
:10712000882339F09091C00095FFFCCF8093C60072
:10713000F6CF8091C00085FFFCCF8AE08093C60027
:107140008BE1FE01EC5BFF4FDE01959601900D9205
:107150008A95E1F724968EAD9FAD24979CA38BA3CF
:107160008CED97E09AA389A320E030E0AE014F5D5B
:107170005F4FBE01615A7F4FC80106DFCE01819685
:107180006EDECE01805C9F4F6ADE44CF898188230A
:1071900009F494C08E3209F43DCF8F3509F43ACF0B
:1071A000F80181898E3209F435CF8F3509F432CF59
:1071B00023FD30CF81E0303109F080E0C957DF4F47
:1071C000E881F981C758D0408083811108C0898542
:1071D000873409F01FCF8A858E3709F41BCF9801B9
:1071E0002C5F3F4FBE016F5F7F4FC901C757DF4F15
:1071F0002883C958D040C657DF4F3883CA58D0407B
:10720000ADDEF30180819181C757DF4F2881C958D6
:10721000D040C657DF4F3881CA58D0400097F1F4AC
:10722000F6018191882339F09091C00095FFFCCF41
:107230008093C600F6CFF9018191882339F09091AF
:10724000C00095FFFCCF8093C600F6CF8091C000B0
:1072500085FFFCCF8AE08093C600DCCE81309105AB
:1072600039F4F50180819181019691838083D2CE9A
:10727000029709F0CFCE8114910439F0B901C4010D
:107280000E94F3CF892B71F419C0CA57DF4FF881E0
:10729000C658D0402F2F30E0F5018081918128170A
:1072A000390761F0CA57DF4FF881C658D040FF5FF9
:1072B000CA57DF4FF883C658D040ACCEC657DF4F11
:1072C0000FB6F894DEBF0FBECDBFDF91CF911F91F7
:1072D0000F91FF90EF90DF90CF90BF90AF909F9075
:1072E0008F907F906F905F904F903F902F90089578
:1072F0000F931F93CF93DF93CDB7DEB76F970FB682
:10730000F894DEBF0FBECDBF8C01FC01EE55FD4FE2
:107310001182108240E050E0BA01835B9F4F0E94CF
:10732000911BC801875B9F4F2BE1FC013496DE0166
:10733000159601900D922A95E1F7FC0182819381C7
:107340009C838B838CED97E09A83898320E030E0E7
:10735000AE014F5F5F4F63EC77E0C80115DECE01F1
:1073600001967DDD6F960FB6F894DEBF0FBECDBFE0
:10737000DF91CF911F910F9108952BE1FB0134967E
:10738000DC01149601900D922A95E1F7FB01228110
:107390003381FC01338322830895EF92FF920F9390
:1073A0001F93CF93DF93EC011B82FC01E05BFF4F47
:1073B0008081882329F0CE01835B9F4F0E94741C3B
:1073C0007E018FE3E81A8EEFF80A45E360E0C7011B
:1073D0000E94894581112CC0E5E3F2E28491882363
:1073E00041F09091C00095FFFCCF8093C60031968C
:1073F000F5CFE091780CF0E0EE0FFF1FE45EFD4F5B
:107400000190F081E02DE857FE4F0190F081E02DD2
:107410008491882341F09091C00095FFFCCF809328
:10742000C6003196F5CF8091C00085FFFCCF9EC08D
:107430008E010A531E4F41E0B701C8010E94422449
:10744000811133C040E0B701C8010E94422481117C
:107450002CC0EBE3F2E28491882341F09091C000CC
:1074600095FFFCCF8093C6003196F5CFE091780C64
:10747000F0E0EE0FFF1FE45EFD4F0190F081E02D84
:10748000E657FE4F0190F081E02D8491882341F072
:107490009091C00095FFFCCF8093C6003196F5CF48
:1074A0008091C00085FFFCCF61C0B801CE01835B35
:1074B0009F4F0E94811981112CC0EBE3F2E284916D
:1074C000882341F09091C00095FFFCCF8093C600C7
:1074D0003196F5CFE091780CF0E0EE0FFF1FE45EFF
:1074E000FD4F0190F081E02DE457FE4F0190F081B7
:1074F000E02D8491882341F09091C00095FFFCCF4E
:107500008093C6003196F5CF8091C00085FFFCCFF7
:107510002DC081E08B83E5E3F2E28491882341F082
:107520009091C00095FFFCCF8093C6003196F5CFB7
:10753000E091780CF0E0EE0FFF1FE45EFD4F01904C
:10754000F081E02DE257FE4F0190F081E02D849113
:10755000882341F09091C00095FFFCCF8093C60036
:107560003196F5CF8091C00085FFFCCF8AE08093F3
:10757000C6008E01075B1F4FB801CE0186599F4F91
:10758000FCDEC859DF4F19830883DF91CF911F912B
:107590000F91FF90EF900895FC01128213820895DD
:1075A000FC012381222311F021E022830895FC01B4
:1075B0002281211112820895AF92BF92CF92DF9261
:1075C000EF92FF920F931F93CF93DF931F92CDB74C
:1075D000DEB78C018FE2FB0181935F01D12C41E08A
:1075E0007801F1E4EF1AFEEFFF0A6FE1C62E2D2DB0
:1075F00030E0F7018081918128173907D8F4C29EC5
:10760000C001C39E900D112483579F4FB501800F79
:10761000911F49830E942819C50149815C01019687
:10762000F5012081222321F04D3810F44F5FF6CF71
:10763000D394DDCF47FD11C0B501C80188519E4FDD
:107640000F90DF91CF911F910F91FF90EF90DF90FE
:10765000CF90BF90AF900C942819F50110820F9035
:10766000DF91CF911F910F91FF90EF90DF90CF901E
:10767000BF90AF9008953F924F925F926F927F922A
:107680008F929F92AF92BF92CF92DF92EF92FF9232
:107690000F931F93CF93DF93CDB7DEB7AC970FB6A1
:1076A000F894DEBF0FBECDBF7C015B01FC0183817E
:1076B000882309F408C1C70188519E4F0E94741C99
:1076C000F7011282CE0101966C01BFDB270198E61B
:1076D000490E511CC701875B9F4FF2019183808344
:1076E000F50180818F3209F084C06FE270E0C5013E
:1076F0000E9411D08C010F5F1F4F7AE0372E0115C9
:10770000110509F47CC06FE270E0C8010E9411D03D
:107710004C01009709F474C00817190708F070C0ED
:107720003C01601A710AA301B801CE0180960E9443
:107730003AD0E0E2F0E0EC0FFD1FE60DF71D1082FD
:10774000FE01B0968191882339F09091C00095FF99
:10775000FCCF8093C600F6CF8091C00085FFFCCFA0
:107760003092C600F201608171816115710519F0D6
:107770006C5F7F4F02C060E070E021E0AE01405ED0
:107780005F4FCE0105960E946B1E81112BC0EBEE60
:10779000F6E08491882341F09091C00095FFFCCFE2
:1077A0008093C6003196F5CFFE01B0968191882373
:1077B00039F09091C00095FFFCCF8093C600F6CFC2
:1077C000E2E7FEE18491882341F09091C00095FFAB
:1077D000FCCF8093C6003196F5CF8091C00085FF25
:1077E000FCCF6CC0F201D182C08284010F5F1F4FB9
:1077F00086CFC70186599F4FF2019183808385010F
:10780000F20180819181009711F0049602C080E01E
:1078100090E0B8010E94411F882339F1E4E6FEE1BF
:107820008491882341F09091C00095FFFCCF809314
:10783000C6003196F5CFF8018191882339F09091F7
:10784000C00095FFFCCF8093C600F6CF8091C000AA
:1078500085FFFCCF8AE08093C600F701E356FD4F19
:1078600010821182128213822CC0ECE4FEE184911A
:10787000882341F09091C00095FFFCCF8093C60013
:107880003196F5CFF8018191882339F09091C000AD
:1078900095FFFCCF8093C600F6CFEAE4FEE1849129
:1078A000882341F09091C00095FFFCCF8093C600E3
:1078B0003196F5CF8091C00085FFFCCF8AE08093A0
:1078C000C600C601CCDAAC960FB6F894DEBF0FBE88
:1078D000CDBFDF91CF911F910F91FF90EF90DF907F
:1078E000CF90BF90AF909F908F907F906F905F9060
:1078F0004F903F9008958F929F92AF92BF92CF92F8
:10790000DF92EF92FF92CF93DF931F92CDB7DEB756
:107910007C01FC018281882309F4BCC071968191AD
:10792000882339F09091C00095FFFCCF8093C6006A
:10793000F6CFE8E4FEE18491882341F09091C00005
:1079400095FFFCCF8093C6003196F5CFE091780C7F
:10795000F0E0EE0FFF1FE45EFD4F0190F081E02D9F
:10796000E456FE4F0190F081E02D8491882341F090
:107970009091C00095FFFCCF8093C6003196F5CF63
:10798000F701E356FD4F40815181628173812AE006
:1079900030E083EE9FE00E9486A3E6E4FEE184915E
:1079A000882341F09091C00095FFFCCF8093C600E2
:1079B0003196F5CFF701EB56FD4F40815181628141
:1079C00073812AE030E083EE9FE00E9486A38091DD
:1079D000C00085FFFCCF8AE08093C6000E9416C3DA
:1079E000E0E6CE2EEAEEDE2EE12CF12CA701960188
:1079F0000E9463CC49015A016091750A7091760A20
:107A00008091770A9091780AA70196010E9463CC31
:107A1000821A930AC4016CE370E00E943CCC698333
:107A2000CE0101960E948185FC012191CF01222384
:107A300039F03091C00035FFFCCF2093C600F4CF61
:107A400040E050E06AE383EE9FE00E943EA3C40161
:107A50006CE370E00E943CCC8983CE0101960E94C9
:107A60008185FC012191CF01222339F03091C000A2
:107A700035FFFCCF2093C600F4CFE4E4FEE184910F
:107A80008823E1F09091C00095FFFCCF8093C60061
:107A90003196F5CFEFEFF6E08491882341F0909195
:107AA000C00095FFFCCF8093C6003196F5CF809142
:107AB000C00085FFFCCF8AE08093C6000F90DF9165
:107AC000CF91FF90EF90DF90CF90BF90AF909F90BD
:107AD0008F900895AF92BF92CF92DF92EF92FF9274
:107AE0000F931F93CF93DF935C01EB01FB01019098
:107AF0000020E9F78F0101501109061B170B6C01DB
:107B0000F8E1CF1AFEEFDF0AF60110826EE470E0B2
:107B1000CE010E9411D07C01009729F4F801319721
:107B2000EC0FFD1F0DC060E270E00E9411D0EC016F
:107B300021966AE270E0C7010E9411D0FC013197E2
:107B40008DE081838AE082831382BE01C5018C515E
:107B50009E4F0E9443A4F6018081882371F1EBE3DC
:107B6000F2E28491882341F09091C00095FFFCCF10
:107B70008093C6003196F5CFE091780CF0E0EE0FDF
:107B8000FF1FE45EFD4F0190F081E02DE056FE4FB7
:107B90000190F081E02D8491882341F09091C00004
:107BA00095FFFCCF8093C6003196F5CF8091C00041
:107BB00085FFFCCF8AE08093C600DF91CF911F91B3
:107BC0000F91FF90EF90DF90CF90BF90AF9008950E
:107BD0002F923F924F925F926F927F928F929F92DD
:107BE000AF92BF92CF92DF92EF92FF920F931F93CB
:107BF000CF93DF93CDB7DEB7CC55D1090FB6F8944C
:107C0000DEBF0FBECDBF4C018C010F551D4F66234B
:107C100039F0F8011082F401838181111DC015C073
:107C2000F8018081882309F4AFC0F401E756FD4FC5
:107C3000C080D180E280F3800E9416C3C616D706AA
:107C4000E806F90608F4A0C0E4CFC401A6DBF401FD
:107C50008381882309F498C07401F7E4EF0EF11CC6
:107C6000F70181818F9380818F938BE39EE19F93B6
:107C70008F938E01015C1F4F1F930F930E9449D079
:107C80000F900F900F900F900F900F90B12CF80164
:107C900001900020E9F73197E01BF10BBE1684F448
:107CA0006801CB0CD11CB7FCDA94F60180819927CE
:107CB00087FD90950E947DCFF6018083B394E7CF36
:107CC000FDE48F0E911C40E050E0BA01C4010E9417
:107CD000911B512CCE0101966C0184E3682E8EE13C
:107CE000782E5E0191E2A90EB11C40E050E0B60191
:107CF000C4010E94DE1A1816DCF5412CF601019031
:107D00000020E9F73197EC19FD094E1674F41601BD
:107D1000240C311C47FC3A94F101808190E00E94D0
:107D20007DCFF10180834394E9CF8A858E37E9F2D4
:107D300045E050E0B801C6010E942CD0892BA9F67D
:107D40001F930F937F926F92BF92AF920E9449D080
:107D5000C5010E948A4880E39EE10E940A490F9073
:107D60000F900F900F900F900F9055245394BDCF0C
:107D7000511004C08FEF9FEFF70104C0F70180811D
:107D80009181019691838083C45ADF4F0FB6F89496
:107D9000DEBF0FBECDBFDF91CF911F910F91FF903E
:107DA000EF90DF90CF90BF90AF909F908F907F909B
:107DB0006F905F904F903F902F9008950F931F9377
:107DC000CF93DF93EC018C0108511E4FC8010E9434
:107DD0002A1CC8010E94741C18821982DF91CF915D
:107DE0001F910F910895CF92DF92EF92FF920F9320
:107DF0001F93CF93DF93CDB7DEB76F970FB6F8948D
:107E0000DEBF0FBECDBF8C016A017C0188E6E80EA3
:107E1000F11CC80186599F4FF70191838083E65C6E
:107E2000FD4F22E030E031832083329671836083FE
:107E300040E050E0BA0104960E94911BF701808156
:107E400091812BE1FC013496DE01159601900D9293
:107E50002A95E1F7FC01828193819C838B838CEDD1
:107E600097E09A8389839601AE014F5F5F4F63EC81
:107E700077E0C80189D8CE0101960E942F376F960E
:107E80000FB6F894DEBF0FBECDBFDF91CF911F912B
:107E90000F91FF90EF90DF90CF9008952F923F9237
:107EA0004F925F926F927F928F929F92AF92BF920A
:107EB000CF92DF92EF92FF920F931F93CF93DF93B6
:107EC000CDB7DEB7AC970FB6F894DEBF0FBECDBF0F
:107ED0008C016B01342EDC0113968C91882309F4FC
:107EE00049C3F801E551FE4F8081882309F4F5C0AC
:107EF0002111C1C07801BDEFEB1AFB0AF7018081A7
:107F0000882361F1EBE3F2E28491882341F09091C0
:107F1000C00095FFFCCF8093C6003196F5CFE6EC0C
:107F2000FEE18491882341F09091C00095FFFCCF41
:107F30008093C6003196F5CF4AE050E061E070E0F2
:107F400083EE9FE00E945AA38091C00085FFFCCF82
:107F50008AE08093C6000E94BB500CC3E5E3F2E2C6
:107F60008491882341F09091C00095FFFCCF8093CD
:107F7000C6003196F5CFEDEAFEE18491882341F009
:107F80009091C00095FFFCCF8093C6003196F5CF4D
:107F9000F6018191882339F09091C00095FFFCCFC4
:107FA0008093C600F6CFE2EAFEE18491882341F097
:107FB0009091C00095FFFCCF8093C6003196F5CF1D
:107FC000D7018C91FDE8BF2EB801B89E600D711DE0
:107FD0001124685F7D4FC801EFDAF7018081F80155
:107FE000B89EE00DF11D1124E85FFD4F81918823BB
:107FF00039F09091C00095FFFCCF8093C600F6CF7A
:10800000ECE9FEE18491882341F09091C00095FF56
:10801000FCCF8093C6003196F5CF5801F3E6AF1A36
:10802000FDEFBF0AD5014D915D916D917C912AE0E4
:1080300030E083EE9FE00E9486A38091C00085FF20
:10804000FCCF8AE08093C600F7012081F80184E02C
:10805000289FE00DF11D1124EC5FFD4FD5014D91DE
:108060005D916D917C9140835183628373832F5F17
:10807000F70120832CC0E5E3F2E28491882341F0EC
:108080009091C00095FFFCCF8093C6003196F5CF4C
:10809000EBE8FEE18491882341F09091C00095FFC8
:1080A000FCCF8093C6003196F5CFF60181918823ED
:1080B00039F09091C00095FFFCCF8093C600F6CFB9
:1080C0008091C00085FFFCCF8AE08093C600C80184
:1080D00088519E4F0E94741C30C0F801ED5FFD4F27
:1080E0001082E5E3F2E28491882341F09091C00090
:1080F00095FFFCCF8093C6003196F5CFEAE7FEE10D
:108100008491882341F09091C00095FFFCCF80932B
:10811000C6003196F5CFF6018191882339F0909110
:10812000C00095FFFCCF8093C600F6CF8091C000C1
:1081300085FFFCCF8AE08093C600D80112961C927E
:10814000FE0131965F01CF010E9425372801F8E634
:108150004F0E511CC801875B9F4FD2018D939C939A
:10816000F60180818F3209F091C06FE270E0C601A4
:108170000E9411D001967C01EAE02E2EE114F10458
:1081800009F48AC06FE270E0C7010E9411D04C016F
:10819000009709F482C0E816F90608F07EC03C0199
:1081A0006E187F08A301B701CE0180960E943AD0D5
:1081B000E0E2F0E0EC0FFD1FE60DF71D1082FE017E
:1081C000B0968191882339F09091C00095FFFCCF43
:1081D0008093C600F6CF8091C00085FFFCCF20922F
:1081E000C600D2016D917C916115710519F06C5F2B
:1081F0007F4F02C060E070E021E0AE01405E5F4F63
:10820000CE0105960E946B1E811138C0E091780C5A
:10821000F0E0EE0FFF1FE45EFD4F0190F081E02DD6
:10822000EE56FE4F0190F081E02D8491882341F0BD
:108230009091C00095FFFCCF8093C6003196F5CF9A
:10824000FE01B0968191882339F09091C00095FF8E
:10825000FCCF8093C600F6CFE8E7FEE18491882347
:1082600041F09091C00095FFFCCF8093C6003196FD
:10827000F5CF8091C00085FFFCCF43C1F201B182F0
:10828000A0827401FFEFEF1AFF0A78CFC801865968
:108290009F4FD2018D939C937601F801E851FE4FD8
:1082A0004F01332009F4E5C0D2016D917C91611535
:1082B000710519F06C5F7F4F02C060E070E021E053
:1082C000A701C4010E946B1E2091780C882309F439
:1082D0009AC0F40181899289A389B489F801EB5687
:1082E000FD4F80839183A283B383E22FF0E0EE0FF2
:1082F000FF1FE45EFD4F0190F081E02DEC56FE4F34
:108300000190F081E02D8491D801AB56BD4F8823B8
:1083100049F09091C00095FFFCCF8093C600319644
:108320008491F5CFF7018191882339F09091C000B5
:1083300095FFFCCF8093C600F6CFE091780CF0E07B
:10834000EE0FFF1FE45EFD4F0190F081E02DEA5635
:10835000FE4F0190F081E02D8491882341F09091AF
:10836000C00095FFFCCF8093C6003196F5CF4D91AC
:108370005D916D917C912AE030E083EE9FE00E9458
:1083800086A38091C00085FFFCCF8AE08093C60061
:10839000F801E356FD4F1082118212821382E091A0
:1083A000780CF0E0EE0FFF1FE45EFD4F0190F081CE
:1083B000E02DE856FE4F0190F081E02D8491882356
:1083C00041F09091C00095FFFCCF8093C60031969C
:1083D000F5CF8091C00085FFFCCF8AE08093C60076
:1083E000A70160E070E0C801FEDCD80151968C91D5
:1083F000882319F0C801419601C0C7010E94B883C3
:108400008CE097E0B2C0E22FF0E0EE0FFF1FE45ED9
:10841000FD4F0190F081E02DEE56FE4F0190F0816E
:10842000E02D8491882341F09091C00095FFFCCF0E
:108430008093C6003196F5CFF7018191882339F0FA
:108440009091C00095FFFCCF8093C600F6CFE6E781
:10845000FEE18491882341F09091C00095FFFCCF0C
:108460008093C6003196F5CF8091C00085FFFCCF88
:1084700048C0F201608171816115710519F06C5F6E
:108480007F4F02C060E070E026E5A701C4010E94B2
:108490006B1E81113AC0E091780CF0E0EE0FFF1FE7
:1084A000E45EFD4F0190F081E02DEE56FE4F01900D
:1084B000F081E02D8491882341F09091C00095FFD8
:1084C000FCCF8093C6003196F5CFF70181918823C8
:1084D00039F09091C00095FFFCCF8093C600F6CF95
:1084E000E4E7FEE18491882341F09091C00095FF7C
:1084F000FCCF8093C6003196F5CF8091C00085FFF8
:10850000FCCF8AE08093C60032C081E0D8018C9312
:10851000E091780CF0E0EE0FFF1FE45EFD4F01905C
:10852000F081E02DE656FE4F0190F081E02D849120
:10853000882341F09091C00095FFFCCF8093C60046
:108540003196F5CFF6018191882339F09091C000E2
:1085500095FFFCCF8093C600F6CF8091C00085FFC9
:10856000FCCF8AE08093C600C7010E94B883C50192
:108570000E942F37AC960FB6F894DEBF0FBECDBF6A
:10858000DF91CF911F910F91FF90EF90DF90CF90EF
:10859000BF90AF909F908F907F906F905F904F9023
:1085A0003F902F90089521E0FC01218340E076CC9C
:1085B000CF92DF92EF92FF920F931F93CF93DF93AF
:1085C000CDB7DEB76F970FB6F894DEBF0FBECDBF45
:1085D0008C016C0128E6C20ED11C86599F4FF60112
:1085E00091838083E65CFD4F21E030E0318320837E
:1085F0007801FCE5EF1AFDEFFF0AF7011182108206
:1086000040E050E0BA0104960E94911BF60180817F
:1086100091812BE1FC013496DE01159601900D92BB
:108620002A95E1F7FC01828193819C838B838CEDF9
:1086300097E09A83898320E030E0AE014F5F5F4F7F
:1086400063EC77E0C8010E94C437CE0101960E9416
:108650002F37F701808191816F960FB6F894DEBFB6
:108660000FBECDBFDF91CF911F910F91FF90EF9083
:10867000DF90CF900895AF92BF92CF92DF92EF92AA
:10868000FF920F931F93CF93DF93CDB7DEB76F9712
:108690000FB6F894DEBF0FBECDBF8C017B01CE01BB
:1086A00001960E942537F801EF58FF4F808168013D
:1086B000811104C029E4C20ED11C03C08AE6C80E91
:1086C000D11C21E0A701B6016C5F7F4FCE0105965A
:1086D0000E946B1E81113AC0E5E3F2E28491882387
:1086E00041F09091C00095FFFCCF8093C600319679
:1086F000F5CFE091780CF0E0EE0FFF1FE45EFD4F48
:108700000190F081E02DEE55FE4F0190F081E02DBB
:108710008491882341F09091C00095FFFCCF809315
:10872000C6003196F5CFF7018191882339F09091F9
:10873000C00095FFFCCF8093C600F6CF8091C000AB
:1087400085FFFCCF8AE08093C60036C0F801E15473
:10875000FE4F808191818A30910530F59C012F5F19
:108760003F4F318320832FE1289F7001299FF00C18
:10877000112429E8E20EF11CE00EF11E5C01B701A4
:10878000C7014F960E94BD3981E0A81AB1082FE1B8
:10879000E21AF1088FEFA816B80689F7B601C801EA
:1087A00087579F4F0E94BD39BE016F5F7F4FC80141
:1087B00086599F4F0E94BD39CE0101960E942F37E6
:1087C0006F960FB6F894DEBF0FBECDBFDF91CF918D
:1087D0001F910F91FF90EF90DF90CF90BF90AF90DF
:1087E0000895EF92FF920F931F93CF93DF93EC01C5
:1087F000C154DE4F2881398121153105F9F021500E
:108800003109398328838C0107571F4FB8018659D6
:108810009F4F0E94BD39C80100E010E07C012FE1AC
:10882000E20EF11C288139810217130738F40F5F1B
:108830001F4FB7010E94BD39C701F0CFDF91CF9123
:108840001F910F91FF90EF900895EF92FF920F9379
:108850001F93CF93DF93EC010E94AEAC8E010D5FAE
:108860001D4FF80180819E0128513E4F79018823D8
:10887000A1F1C9010E94741CF8018081815080839C
:10888000BE01FDE88F9F600D711D1124685F7D4F53
:1088900021E041E0CE0102DBF8018081FE0124E00D
:1088A000829FE00DF11D1124EC5FFD4F408151814D
:1088B00062817381FE01E356FD4F408351836283E1
:1088C0007383C7010E94911BCE01DF91CF911F914D
:1088D0000F91FF90EF900C94D03A0E9424ADC70105
:1088E0000E94741C1A8284E29EE1DF91CF911F9155
:1088F0000F91FF90EF908EC48FEF8EBD0DB407FEE9
:10890000FDCF8EB508958EBD0DB407FEFDCF089541
:1089100061E0FC0180810C946FC2FC012281322F46
:10892000306A36953CBD20FD06C031E0263009F4A2
:1089300030E0232F01C020E02DBD60E0FC018081EC
:108940000C946FC2CF92DF92EF92FF920F931F931E
:10895000CF93DF93EC018B017A010E9416C36B0168
:10896000CBDF8B838F3F49F40E9416C36C197D09BE
:108970006D327140A8F381E144C08E3F11F08FE069
:1089800040C0E114F104D9F0C70101972FEF2EBDCB
:10899000F8014FEF9F01201B310B2817390738F4DE
:1089A0000DB407FEFDCF2EB521934EBDF3CF0DB410
:1089B00007FEFDCF2EB5F801E80FF91F2083D8017F
:1089C000E00EF11EC12CD12CAE15BF0579F08D91B2
:1089D000ED2DFF27E827EE0FFF1FE75FF04E859193
:1089E0009491DC2CCC24C826D926EECF85DF082F25
:1089F00010E0102F002780DF082BC016D10631F0C1
:108A000080E28983CE0184DF80E003C0CE0180DF75
:108A100081E0DF91CF911F910F91FF90EF90DF9058
:108A2000CF9008950F931F93CF93DF93EB010E9494
:108A300016C38B0161DF8F3F49F00E9416C3601B94
:108A4000710B6C177D07B0F380E001C081E0DF910E
:108A5000CF911F910F910895CF92DF92FF920F93C4
:108A60001F93CF93DF9300D01F92CDB7DEB76C0179
:108A7000F62E29833A834B835C834FDF6CE271E0EF
:108A8000C601D0DF8F2D80643EDF08E110E05C81FD
:108A90004B813A812981DA01C901002E04C0B695C3
:108AA000A795979587950A94D2F729833A834B83A4
:108AB0005C8329DF0850110929813A814B815C814F
:108AC000083F8FEF180739F7FF2029F0E8E0FE167E
:108AD00021F08FEF03C085E901C087E814DFFCE0D7
:108AE000FF1201C009DF10E007DFF601838387FF73
:108AF00004C01F3F11F01F5FF7CF0F900F900F9032
:108B00000F90DF91CF911F910F91FF90DF90CF9049
:108B10000895BF92CF92DF92EF92FF920F931F932F
:108B2000CF93DF93EC01B62E1C82198248830E94FA
:108B300016C38B0161E088810E9436C2CE01E8DE57
:108B400060E082E30E9436C261E083E30E9436C2A5
:108B500061E084E30E9436C261E085E30E9436C290
:108B600061E085E30E946FC285E08A8382E58CBD67
:108B70001DBC6AE0F62E8FEFC6DEFA94E1F720E026
:108B800030E0A90160E0CE0167DFF82E8B8381E041
:108B9000F81649F00E9416C3601B710B613D7740C7
:108BA00070F381E046C02AEA31E040E050E068E03E
:108BB000CE0152DF82FF02C0FC820CC054E0F52ED1
:108BC0009BDE8B83FA94E1F78A3A11F082E031C0A0
:108BD00082E08C838C81823031F4C12CD12CE12C49
:108BE00040E4F42E03C0C12CD12C760120E030E00B
:108BF000A90167E3CE0130DFA701960169E2CE014A
:108C00002BDF8B83882349F00E9416C3601B710BF6
:108C1000613D774058F38AE00CC08C818230B1F41A
:108C200020E030E0A9016AE3CE0116DF882329F0B5
:108C300088E08983CE016CDE14C05EDE807C803CDF
:108C400011F483E08C8358DE57DE56DECE0160DE01
:108C500086E08B1518F488E1898303C0BA8281E02D
:108C600001C080E0DF91CF911F910F91FF90EF90B5
:108C7000DF90CF90BF900895AF92BF92CF92DF92D6
:108C8000EF92FF920F931F93CF93DF93EC016A0152
:108C90007B0189018C81833039F0F9E0CC0CDD1C3B
:108CA000EE1CFF1CFA95D1F773E0B72EE4E0AE2E70
:108CB000BA94A701960161E1CE01CEDE882311F0BE
:108CC000A98207C040E052E0B801CE013BDE81112D
:108CD0000EC0CE01BB2049F01BDE20E030E0A90130
:108CE0006CE0CE01B9DE1982E3CF12DE80E0DF91C5
:108CF000CF911F910F91FF90EF90DF90CF90BF9099
:108D0000AF900895CF93DF93EC016EBD20E030E08B
:108D10000DB407FEFDCFFA01E20FF31F80818EBD77
:108D20000DB407FEFDCF81818EBD2E5F3F4F211513
:108D300082E0380769F70DB407FEFDCF8FEFE3DD62
:108D40008FEFE1DDD9DD8B838F71853031F083E1E9
:108D50008983CE01DDDD80E001C081E0DF91CF912C
:108D600008950F931F93CF93DF93EC0189018C81BA
:108D7000833039F0B9E0440F551F661F771FBA954D
:108D8000D1F79A01AB0168E1CE0166DE882311F0CC
:108D900086E01EC0A8016EEFCE01B4DF8823C9F0C3
:108DA00068E572E0CE013EDE182F811102C087E136
:108DB0000FC020E030E0A9016DE0CE014DDE811151
:108DC00006C09ADD811103C0CE01A2DD05C086E197
:108DD0008983CE019DDD10E0812FDF91CF911F911E
:108DE0000F910895FC016591759185919491089575
:108DF0002F923F924F925F926F927F928F929F92AB
:108E0000AF92BF92CF92DF92EF92FF920F931F9398
:108E1000CF93DF9300D000D0CDB7DEB71C01FC01AB
:108E2000EA50FE4D14919C01220F331F220F331F75
:108E30003E832D832959334F4901F9011082118254
:108E40001282138223E73CE04FE65CE06BE67CE0B5
:108E500087E69CE00E9423BE8D819E818B5F9D4DA5
:108E6000C1DF6B017C01612F772767FD7095872F2C
:108E7000972F0E9427C92B013C012D813E812E5C3A
:108E8000334F590120E030E040EC5FE3C701B60109
:108E90000E945ACBA30192010E945ACBF501608334
:108EA0007183828393832D813E8121523A4F3C838B
:108EB0002B83F90160817181828193816093A10587
:108EC0007093A2058093A3059093A40520E030E061
:108ED00040E752E40E948CC823E5C22E2CE0D22E3B
:108EE0007B018C012EE33CE04AE35CE066E37CE03E
:108EF00082E39CE00E9441B40E94AEACF401108277
:108F000011821282138223E73CE04FE65CE06BE6BD
:108F10007CE087E69CE00E9423BE2D813E812750A5
:108F20003E4D3A832983C9015DDF9058A301920128
:108F30000E945ACBF501608371838283938320E082
:108F400030E040E752E46091A1057091A205809164
:108F5000A3059091A4050E948CC87B018C012EE38F
:108F60003CE04AE35CE066E37CE082E39CE00E9454
:108F700041B40E94AEAC89819A8134DF9B01AC017F
:108F80000E94ACC7A30192010E945ACBF5016083F5
:108F900071838283938320E030E040E05FE3EB81E4
:108FA000FC8160817181828193810E945ACB6093A0
:108FB000A1057093A2058093A3059093A40520E0DA
:108FC00030E040E752E40E948CC87B018C012EE324
:108FD0003CE04AE35CE066E37CE082E39CE00E94E4
:108FE00041B40E94AEAC8D819E818F5E9D4DFADEB4
:108FF0000D811E81055A134FF80120813181428174
:1090000053810E94ACC7F401608371838283938390
:109010008D819E81875D9D4DE5DE2D813E812D53A5
:109020003A4F7901F80120813181428153810E94B8
:10903000ACC7F70160837183828393838D819E81A6
:10904000835E9D4DCFDE2D813E8129543A4F7901BB
:10905000F80120813181428153810E94ACC7F70120
:109060006083718382839383F40180819181A281E3
:10907000B381F50180839183A283B3831092A1050C
:109080001092A2051092A3051092A4050E9427A594
:10909000F101E85AF34F81E0808326960FB6F894E9
:1090A000DEBF0FBECDBFDF91CF911F910F91FF901B
:1090B000EF90DF90CF90BF90AF909F908F907F9078
:1090C0006F905F904F903F902F900895FC012491F6
:1090D000222341F03091C00035FFFCCF2093C60021
:1090E0000196F4CF22E030E083EE9FE00C9430A4B0
:1090F000FC012491222341F03091C00035FFFCCFC8
:109100002093C6000196F4CF2AE030E083EE9FE082
:109110000C9486A32091870A3091880A2430310567
:109120000CF077C04091890A50918A0A60E6649FEA
:109130009001659F300D1124BC01C9018F56954FD8
:109140000E9425D0E5E3F2E28491882341F09091DA
:10915000C00095FFFCCF8093C6003196F5CFE0911B
:10916000780CF0E0EE0FFF1FE45EFD4F0190F08100
:10917000E02DEA5DFE4F0190F081E02D849188237F
:1091800041F09091C00095FFFCCF8093C6003196CE
:10919000F5CF8091890A90918A0A20E6289FF001F4
:1091A000299FF00D1124EF56F54F8191882339F056
:1091B0009091C00095FFFCCF8093C600F6CFE4EFFE
:1091C000F1E28491882341F09091C00095FFFCCF9B
:1091D0008093C6003196F5CF8091C00085FFFCCF0B
:1091E0008AE08093C6008091890A90918A0A01964C
:1091F00064E070E00E9450CC90938A0A8093890AC0
:109200008091870A9091880A01969093880A8093AA
:10921000870A08952091870A3091880A2430310501
:109220000CF077C04091890A50918A0A60E6649FE9
:109230009001659F300D1124BC01C9018F56954FD7
:109240000E9485CFE5E3F2E28491882341F090917A
:10925000C00095FFFCCF8093C6003196F5CFE0911A
:10926000780CF0E0EE0FFF1FE45EFD4F0190F081FF
:10927000E02DEA5DFE4F0190F081E02D849188237E
:1092800041F09091C00095FFFCCF8093C6003196CD
:10929000F5CF8091890A90918A0A20E6289FF001F3
:1092A000299FF00D1124EF56F54F8191882339F055
:1092B0009091C00095FFFCCF8093C600F6CFE2EFFF
:1092C000F1E28491882341F09091C00095FFFCCF9A
:1092D0008093C6003196F5CF8091C00085FFFCCF0A
:1092E0008AE08093C6008091890A90918A0A01964B
:1092F00064E070E00E9450CC90938A0A8093890ABF
:109300008091870A9091880A01969093880A8093A9
:10931000870A08959B9AA3980895FCDF40E052ECD9
:1093200061E070E083EE9FE00E943EA2ECEEF1E28D
:109330008491882341F09091C00095FFFCCF8093E9
:10934000C6003196F5CF8091C00085FFFCCF8AE042
:109350008093C60025E332E2F9018491882341F02D
:109360009091C00095FFFCCF8093C6003196F5CF59
:1093700084B780FF20C0A091780CB0E0AA0FBB1F7B
:10938000A45EBD4FED91FC91E85DFE4F0190F08130
:10939000E02D9491992341F04091C00045FFFCCF0E
:1093A0009093C6003196F5CF9091C00095FFFCCF09
:1093B0009AE09093C60081FF20C0A091780CB0E0A5
:1093C000AA0FBB1FA45EBD4FED91FC91E65DFE4F61
:1093D0000190F081E02D9491992341F04091C000DB
:1093E00045FFFCCF9093C6003196F5CF9091C00019
:1093F00095FFFCCF9AE09093C60082FF20C0A09119
:10940000780CB0E0AA0FBB1FA45EBD4FED91FC919C
:10941000E45DFE4F0190F081E02D9491992341F09D
:109420004091C00045FFFCCF9093C6003196F5CF28
:109430009091C00095FFFCCF9AE09093C60083FF07
:1094400020C0A091780CB0E0AA0FBB1FA45EBD4F56
:10945000ED91FC91E25DFE4F0190F081E02D949141
:10946000992341F04091C00045FFFCCF9093C60086
:109470003196F5CF9091C00095FFFCCF9AE0909384
:10948000C60085FF20C0A091780CB0E0AA0FBB1FDA
:10949000A45EBD4FED91FC91E05DFE4F0190F08127
:1094A000E02D8491882341F09091C00095FFFCCF7E
:1094B0008093C6003196F5CF8091C00085FFFCCF28
:1094C0008AE08093C60014BEE1E2F7E0849188232D
:1094D00041F09091C00095FFFCCF8093C60031967B
:1094E000F5CFE8E2F7E08491882341F09091C00045
:1094F00095FFFCCF8093C6003196F5CF8091C000D8
:1095000085FFFCCF8AE08093C600F9018491E5E3F2
:10951000F2E2882349F09091C00095FFFCCF809340
:10952000C60031968491F5CFA091780CB0E0AA0FD7
:10953000BB1FA45EBD4FED91FC91EC5CFE4F019012
:10954000F081E02D8491882341F09091C00095FF37
:10955000FCCF8093C6003196F5CFE7EDF1E2849120
:10956000882341F09091C00095FFFCCF8093C60006
:109570003196F5CFA091780CB0E0AA0FBB1FA45E86
:10958000BD4FED91FC91EE5CFE4F0190F081E02D1E
:109590004491442341F05091C00055FFFCCF4093CB
:1095A000C6003196F5CFE0ECF1E28491882341F0DA
:1095B0009091C00095FFFCCF8093C6003196F5CF07
:1095C0008091C00085FFFCCF8AE08093C600E5EB68
:1095D000F1E28491882341F09091C00095FFFCCF87
:1095E0008093C6003196F5CFE9EAF1E284918823B1
:1095F00041F09091C00095FFFCCF8093C60031965A
:10960000F5CF8091C00085FFFCCF8AE08093C60033
:10961000F9012491E5E3F2E2222349F08091C000B0
:1096200085FFFCCF2093C60031962491F5CFE091C1
:10963000780CF0E0EE0FFF1FE45EFD4F0190F0812B
:10964000E02DEA5CFE4F0190F081E02D84918823AB
:1096500041F09091C00095FFFCCF8093C6003196F9
:10966000F5CF0E9422B04AE050E0BC0183EE9FE0BB
:109670000E945AA3E091780CF0E0EE0FFF1FE45E29
:10968000FD4F0190F081E02DE85CFE4F0190F081EC
:10969000E02D8491882341F09091C00095FFFCCF8C
:1096A0008093C6003196F5CF4AE050E060ED74E05B
:1096B00083EE9FE00E945AA38091C00085FFFCCFFB
:1096C0008AE08093C60010928D0A10928E0A109242
:1096D0008F0A1092900A0E945FA00E94319C0E9403
:1096E0008A290E94F1B30E9410AF0E945C8480918D
:1096F000000186FD29C0FFEF23ED80E3F1502040FB
:109700008040E1F700C000008091000186FD25C087
:10971000809101018460809301019FB7F89480914A
:1097200002018460809302019FBF0E949383809115
:10973000000186FFFCCF9FB7F894809102018B7FD8
:10974000809302019FBF08959FEFE3EDF0E39150F6
:10975000E040F040E1F700C0000008958091810AE8
:109760009091820A60E070E001960C94DCCC8091CC
:10977000810A9091820A4AE050E060E070E0019630
:109780000C9444CE682F772767FD709520918B0A43
:1097900030918C0A40E6429FC001439F900D1124F6
:1097A0008F56954F0E9411D09093820A8093810A20
:1097B00021E0892B09F420E0822F08950E9416C32E
:1097C00060937D0A70937E0A80937F0A9093800A4B
:1097D00008950E9416C360937D0A70937E0A809359
:1097E0007F0A9093800AE0918B0AF0918C0AE357EC
:1097F000F54F8081811121C0E091780CF0E0EE0FEF
:10980000FF1FE45EFD4F0190F081E02DE65CFE4F0E
:109810000190F081E02D8491882341F09091C00067
:1098200095FFFCCF8093C6003196F5CF8091C000A4
:1098300085FFFCCF8AE08093C600089583EE9FE009
:109840000E9490A2E091780CF0E0EE0FFF1FE45E22
:10985000FD4F0190F081E02DE659FE4F0190F0811F
:10986000E02D8491882341F09091C00095FFFCCFBA
:109870008093C6003196F5CF4091160C5091170C8D
:109880006091180C7091190C4F5F5F4F6F4F7F4FB5
:109890002AE030E083EE9FE00E942FA38091C00079
:1098A00085FFFCCF8AE08093C60093CF8F929F9272
:1098B000AF92BF92CF92DF92EF92FF920F931F93DE
:1098C000CF93DF93B5EAEB2EB7E0FB2E07E61CE063
:1098D000C2E3DCE08DE7C82E8CE0D82EF701819141
:1098E0007F0150DF882311F139DF4B015C01F60164
:1098F0008081811103C06091110C01C061E070E0B2
:1099000080E090E00E9427C9F801208131814281E6
:1099100053810E945ACB9B01AC01C501B4010E9446
:10992000ACC7688379838A839B8309C0F8018081EF
:109930009181A281B38188839983AA83BB830C5FC1
:109940001F4F2496FFEFCF1ADF0A89EAE81687E057
:10995000F80621F686E416DF8823D1F0FFDE6B01DE
:109960007C016093220C7093230C8093240C9093C1
:10997000250C20E030E0A9010E9488CA181644F4A2
:10998000C092A105D092A205E092A305F092A40591
:10999000DF91CF911F910F91FF90EF90DF90CF90CB
:1099A000BF90AF909F908F90089580DF89E4EADEAA
:1099B000882351F0D3DE6093260C7093270C80939C
:1099C000280C9093290C08C01092260C1092270C9A
:1099D0001092280C1092290C8AE4D4DE882351F0CE
:1099E000BDDE60932A0C70932B0C80932C0C90930B
:1099F0002D0C089510922A0C10922B0C10922C0C06
:109A000010922D0C0895CF92DF92EF92FF92CF9398
:109A1000DF93EC01C090C305D090C405E090C5056C
:109A2000F090C605A7019601688179818A819B81A2
:109A30000E9485C887FF04C0C882D982EA82FB825F
:109A4000C090C705D090C805E090C905F090CA0540
:109A5000A70196016C817D818E819F810E9485C8BE
:109A600087FF04C0CC82DD82EE82FF8220E030E0FE
:109A7000A9016091CB057091CC058091CD059091A5
:109A8000CE050E94ACC76B017C019B01AC016885CF
:109A900079858A859B850E9485C887FF04C0C88612
:109AA000D986EA86FB86C090B705D090B805E090CD
:109AB000B905F090BA05A7019601688179818A817C
:109AC0009B810E9488CA181624F4C882D982EA822F
:109AD000FB82C090BB05D090BC05E090BD05F09026
:109AE000BE05A70196016C817D818E819F810E94B8
:109AF00088CA181624F4CC82DD82EE82FF82C090E0
:109B0000BF05D090C005E090C105F090C205A70147
:109B10009601688579858A859B850E9488CA181672
:109B200024F4C886D986EA86FB86DF91CF91FF9020
:109B3000EF90DF90CF900895CF92DF92EF92FF9257
:109B40000F931F9382E39CE05EDF0E9416C3609335
:109B50007D0A70937E0A80937F0A9093800A2091F9
:109B6000320C3091330C4091340C5091350C609193
:109B7000670C7091680C8091690C90916A0C0E943E
:109B800085C8811179C02091360C3091370C4091F5
:109B9000380C5091390C60916B0C70916C0C809169
:109BA0006D0C90916E0C0E9485C8811165C020E0FB
:109BB00030E040E752E46091A1057091A2058091E8
:109BC000A3059091A4050E948CC823E5C22E2CE029
:109BD000D22E7B018C012EE33CE04AE35CE066E39D
:109BE0007CE082E39CE00E9441B48091320C909131
:109BF000330CA091340CB091350C8093670C90938A
:109C0000680CA093690CB0936A0C8091360C90910B
:109C1000370CA091380CB091390C80936B0C909359
:109C20006C0CA0936D0CB0936E0C80913A0C9091DB
:109C30003B0CA0913C0CB0913D0C80936F0C909329
:109C4000700CA093710CB093720C80913E0C9091AB
:109C50003F0CA091400CB091410C8093730C9093F9
:109C6000740CA093750CB093760C1F910F91FF901C
:109C7000EF90DF90CF9008956091DD057091DE0543
:109C8000882777FD8095982F0E9427C92091A105EC
:109C90003091A2054091A3055091A4050E945ACB92
:109CA00020E030E040E752E40E948CC820E030E041
:109CB00048EC52E488CFCF92DF92EF92FF92CF939D
:109CC000C62FE091530CF0E0882309F4C2C0DF01F5
:109CD000A15BB34F8C91811196C18091670C9091DB
:109CE000680CA091690CB0916A0C8093320C90932F
:109CF000330CA093340CB093350C80916B0C909185
:109D00006C0CA0916D0CB0916E0C8093360C9093FE
:109D1000370CA093380CB093390C80916F0C909154
:109D2000700CA091710CB091720C80933A0C9093CE
:109D30003B0CA0933C0CB0933D0CC090730CD090A6
:109D4000740CE090750CF090760CC0923E0CD092A2
:109D50003F0CE092400CF092410CEE0FFF1FEE0F13
:109D6000FF1FE153FA4F20813181428153816623E5
:109D700049F06091AF057091B0058091B105909167
:109D8000B20508C06091B3057091B4058091B50526
:109D90009091B6050E948CC89B01AC01C701B60129
:109DA0000E94ACC76093730C7093740C8093750C15
:109DB0009093760C83E79CE00E94C8BEC090A105FA
:109DC000D090A205E090A305F090A40520E030E03B
:109DD00040E752E46091AB057091AC058091AD0510
:109DE0009091AE050E945ACB6093A1057093A20595
:109DF0008093A3059093A405E091530CF0E0E15B00
:109E0000F34F81E0808398DE20914B0C30914C0C15
:109E100040914D0C50914E0C60916F0C7091700CF4
:109E20008091710C9091720C0E94ABC760936F0C83
:109E30007093700C8093710C9093720C23E73CE04C
:109E40004FE65CE06BE67CE087E69CE00E9423BE88
:109E5000D1C0E15BF34F8081882309F4D4C08091A5
:109E6000670C9091680CA091690CB0916A0C80937A
:109E7000320C9093330CA093340CB093350C80913A
:109E80006B0C90916C0CA0916D0CB0916E0C80934A
:109E9000360C9093370CA093380CB093390C60912A
:109EA0006F0C7091700C8091710C9091720C60939A
:109EB0003A0C70933B0C80933C0C90933D0CC090FB
:109EC000730CD090740CE090750CF090760CC092EE
:109ED0003E0CD0923F0CE092400CF092410C20914D
:109EE0004B0C30914C0C40914D0C50914E0C0E94FB
:109EF000ACC760936F0C7093700C8093710C90934F
:109F0000720C23E73CE04FE65CE06BE67CE087E622
:109F10009CE00E9423BEF090530CCC2389F020914A
:109F2000430C3091440C4091450C5091460C60918B
:109F3000AF057091B0058091B1059091B20510C048
:109F40002091470C3091480C4091490C50914A0C9B
:109F50006091B3057091B4058091B5059091B605F7
:109F60000E94ACC724E0F29EF0011124E153FA4FA5
:109F700020813181428153810E948CC89B01AC01B8
:109F80006091730C7091740C8091750C9091760CAB
:109F90000E94ABC76093730C7093740C8093750C24
:109FA0009093760C83E79CE00E94C8BEC090A10508
:109FB000D090A205E090A305F090A40520E030E049
:109FC00040E752E46091A7057091A8058091A9052A
:109FD0009091AA050E945ACB6093A1057093A205A7
:109FE0008093A3059093A405E091530CF0E0E15B0E
:109FF000F34F1082A1DDC092A105D092A205E0929C
:10A00000A305F092A405CF91FF90EF90DF90CF9041
:10A010000895AF92BF92CF92DF92EF92FF920F938B
:10A020001F93CF93DF93D82F20912A0C30912B0CC4
:10A0300040912C0C50912D0C6091260C7091270CA6
:10A040008091280C9091290C0E9495CAC62F172F39
:10A05000082FF92E6091DD057091DE05882777FDC8
:10A060008095982F0E9427C92091A1053091A205C3
:10A070004091A3055091A4050E945ACB20E030E006
:10A0800040E752E40E948CC820E030E048EC52E403
:10A090000E948CC82091530C2F93DF93FF920F9353
:10A0A0001F93CF935B016C0142E0E42E01E020E0BE
:10A0B00046E25CE062E37CE087E69CE00E94B3332A
:10A0C0008091320C9091330CA091340CB091350CEE
:10A0D0008093670C9093680CA093690CB0936A0C02
:10A0E0008091360C9091370CA091380CB091390CBE
:10A0F00080936B0C90936C0CA0936D0CB0936E0CD2
:10A1000080913A0C90913B0CA0913C0CB0913D0C8D
:10A1100080936F0C9093700CA093710CB093720CA1
:10A1200080913E0C90913F0CA091400CB091410C5D
:10A130008093730C9093740CA093750CB093760C71
:10A140000E9416C360937D0A70937E0A80937F0AF3
:10A150009093800A0F900F900F900F900F900F9098
:10A16000DF91CF911F910F91FF90EF90DF90CF90F3
:10A17000BF90AF900895F8940E942D2A179A1092DC
:10A18000580C169A1092590C159A10925A0C149A4F
:10A1900060E087E40E9436C2EBE3F2E28491882318
:10A1A00041F09091C00095FFFCCF8093C60031969E
:10A1B000F5CFE091780CF0E0EE0FFF1FE45EFD4F6D
:10A1C0000190F081E02DEA59FE4F0190F081E02DE1
:10A1D0008491882341F09091C00095FFFCCF80933B
:10A1E000C6003196F5CF8091C00085FFFCCF8AE094
:10A1F0008093C600E091780CF0E0EE0FFF1FE45E64
:10A20000FD4F0190F081E02DE653FF4F8081918159
:10A210000E94F5837894C6E0D0E02197209749F01A
:10A2200068EC70E080E090E00E9445C30E94978453
:10A23000F4CFF894FFCF2F923F924F925F926F929C
:10A240007F928F929F92AF92BF92CF92DF92EF92C6
:10A25000FF920F931F93CF93DF93CDB7DEB76E9727
:10A260000FB6F894DEBF0FBECDBF30E6D32E44E06C
:10A27000E42EF12C5AE0C52EBB24B39480916410D7
:10A28000909165102091661030916710821B930B9E
:10A290008F779927892B09F467C28091870A90915B
:10A2A000880A04970CF060C283EE9FE00E9474A2BB
:10A2B0008093860A2091840A3091850A8A3061F061
:10A2C0008D3051F08A3321F49091830A992321F043
:10A2D0002F3531050CF442C12115310509F45CC15B
:10A2E0008091890A90918A0AD89E4001D99E900C4B
:10A2F0001124F401E20FF31FEF56F54F1082209165
:10A30000830A211126C11092830AFC01E357F54FFD
:10A31000108284010F56154F6EE470E0C8010E9450
:10A3200011D00097F1F19093820A8093810A801BEB
:10A33000910B880D991D4AE050E060E070E08E5668
:10A34000954F0E9444CE60931A0C70931B0C80931F
:10A350001C0C90931D0C4090160C5090170C6090A4
:10A36000180C7090190C2FEF421A520A620A720AE6
:10A370000091890A10918A0A64157505860597056A
:10A3800009F40DC1D09EC001D19E900D112460EA48
:10A3900071E28F56954F0E94BCCF892B09F0FFC008
:10A3A000A9C16AE270E0C8010E9411D0892B09F4AA
:10A3B00051C0EBE3F2E28491882341F09091C00018
:10A3C00095FFFCCF8093C6003196F5CFE091780CD5
:10A3D000F0E0EE0FFF1FE45EFD4F0190F081E02DF5
:10A3E000EC5BFE4F0190F081E02D8491882341F0D9
:10A3F0009091C00095FFFCCF8093C6003196F5CFB9
:10A400004091160C5091170C6091180C7091190C1A
:10A410002AE030E083EE9FE00E942FA38091C000ED
:10A4200085FFFCCF8AE08093C6001092850A1092C7
:10A43000840A0DC380911A0C90911B0CA0911C0CE6
:10A44000B0911D0C8093160C9093170CA093180CD0
:10A45000B093190C8091890A90918A0AD89E800144
:10A46000D99E100D1124C8018F56954F4C0167E4F9
:10A4700070E00E9411D0009709F447C09093820ABF
:10A480008093810A88199909800F911F60E070E01C
:10A490008E56954F0E94DCCC0E94F4C86430710542
:10A4A000A0F580916F0A882381F1E091780CF0E0AB
:10A4B000EE0FFF1FE45EFD4F0190F081E02DE859A3
:10A4C000FE4F0190F081E02D8491882341F090911E
:10A4D000C00095FFFCCF8093C6003196F5CF8091E8
:10A4E000C00085FFFCCFC092C600E091780CF0E080
:10A4F000EE0FFF1FE45EFD4F0190F081E02DE4536D
:10A50000FF4F808191810E94E8830091890A109118
:10A510008A0AD09EC001D19E900D11246EE277E090
:10A520008F56954F0E941CD0892B09F424DEC80158
:10A530000196B7010E9450CC90938A0A8093890AB1
:10A540008091870A9091880A01969093880A809357
:10A55000870A1092850A1092840A90CE8B3311F4E8
:10A56000B092830A9091830A911188CE4091890A12
:10A5700050918A0AB9016F5F7F4F7093850A60938B
:10A58000840AD49EF001D59EF00D1124E20FF31F32
:10A59000EF56F54F808372CE1092830A58C2D09E38
:10A5A0004001D19E900C1124C4018F56954F3C015F
:10A5B0006AE270E00E9411D0009709F03EC0EBE320
:10A5C000F2E28491882341F09091C00095FFFCCF86
:10A5D0008093C6003196F5CFE091780CF0E0EE0F55
:10A5E000FF1FE45EFD4F0190F081E02DEE5BFE4F1A
:10A5F0000190F081E02D8491882341F09091C0007A
:10A6000095FFFCCF8093C6003196F5CF4091160C94
:10A610005091170C6091180C7091190C2AE030E0E1
:10A6200083EE9FE00E942FA38091C00085FFFCCFA6
:10A630008AE08093C60002D9F8CE20E010E0F40151
:10A64000E20FF11DEF56F54F30813A3219F02F5FCE
:10A650001327F5CF9093820A8093810A8619970970
:10A66000880D991D60E070E08E56954F0E94DCCCFD
:10A670000E94F4C8212F30E02617370709F4DACEFC
:10A68000EBE3F2E28491882341F09091C00095FFC2
:10A69000FCCF8093C6003196F5CFE091780CF0E0C6
:10A6A000EE0FFF1FE45EFD4F0190F081E02DE05CB6
:10A6B000FE4F0190F081E02D8491882341F090912C
:10A6C000C00095FFFCCF8093C6003196F5CF409136
:10A6D000160C5091170C6091180C7091190C2AE00F
:10A6E00030E083EE9FE00E942FA38091C00085FFA1
:10A6F000FCCF9ECFEBE3F2E28491882341F090916E
:10A70000C00095FFFCCF8093C6003196F5CFE09155
:10A71000780CF0E0EE0FFF1FE45EFD4F0190F0813A
:10A72000E02DE25CFE4F0190F081E02D84918823C2
:10A7300041F09091C00095FFFCCF8093C600319608
:10A74000F5CF4091160C5091170C6091180C709138
:10A75000190C2AE030E083EE9FE00E942FA3809145
:10A76000C00085FFFCCF64CF8091890C882309F459
:10A770006EC18091840A9091850A892B09F067C186
:10A780008091870A9091880A892B11F410926D0AA2
:10A79000F8EE2F2EF3E03F2E412C512CACE3CA2EC5
:10A7A000D12CE12CF12C8E010F5F1F4FE0E66E2EB5
:10A7B000772473944091240F5091250F6091260FB8
:10A7C0007091270F80911C0F90911D0FA0911E0F6B
:10A7D000B0911F0F481759076A077B0708F037C168
:10A7E0008091870A9091880A04970CF030C180917B
:10A7F0006D0A81112CC18091770E9091780EA091F5
:10A80000790EB0917A0E8093240F9093250FA09328
:10A81000260FB093270F8FE69EE00E94C81A482F9C
:10A820008093860A8A30B9F04D30A9F0433229F47A
:10A830002091830A222379F002C04A33C9F3209180
:10A84000840A3091850A2F3531052CF48F3FAFEF04
:10A850009A0709F0DEC04091240F5091250F6091B6
:10A86000260F7091270F80911C0F90911D0FA091C2
:10A870001E0FB0911F0F481759076A077B0708F48E
:10A880008EC0E091780CF0E0EE0FFF1FE45EFD4F0C
:10A890000190F081E02DEA5BFE4F0190F081E02D08
:10A8A0008491882341F09091C00095FFFCCF809364
:10A8B000C6003196F5CF8091C00085FFFCCFBAE08D
:10A8C000B093C6000E9416C36093710A7093720A17
:10A8D0008093730A9093740A8090750A9090760A18
:10A8E000A090770AB090780A681979098A099B09BB
:10A8F000A20191010E9463CC49015A01CA01B90128
:10A90000A70196010E9463CCCA01B901A701960173
:10A910000E9463CC7F936F93C501B40120E13EE0B8
:10A9200040E050E00E9463CC3F932F93ACE8B1E24B
:10A93000BF93AF931F930F930E9449D0E5E3F2E2D8
:10A9400084910FB6F894DEBF0FBECDBF882349F0C7
:10A950009091C00095FFFCCF8093C6003196849102
:10A96000F5CFF8018191882339F09091C00095FFCF
:10A97000FCCF8093C600F6CF8091C00085FFFCCF4E
:10A980003AE03093C600C8010E94B88387E89CE093
:10A990000E94254461E087E89CE00E94E83D8091A8
:10A9A000860A833211F470926D0A2091840A3091E4
:10A9B000850A2115310509F4EFCD8091890A90911E
:10A9C0008A0A689EF001699EF00D1124E20FF31FC0
:10A9D000EF56F54F1082FC01E357F54F708220913E
:10A9E000870A3091880A2F5F3F4F3093880A20935F
:10A9F000870A019664E070E00E9450CC90938A0A26
:10AA00008093890A1092830A1092850A1092840A10
:10AA1000D1CE4B3311F47092830A4091830A4111D5
:10AA2000C5CE4091890A50918A0AB9016F5F7F4F64
:10AA30007093850A6093840A649EF001659EF00D10
:10AA40001124E20FF31FEF56F54F8083B3CE6E96BD
:10AA50000FB6F894DEBF0FBECDBFDF91CF911F912F
:10AA60000F91FF90EF90DF90CF90BF90AF909F90AD
:10AA70008F907F906F905F904F903F902F900895B0
:10AA8000CF92DF92EF92FF920F931F93CF93C82F35
:10AA90008091870A9091880A03970CF4CCDB0E947E
:10AAA00016C30091790A10917A0A20917B0A30919D
:10AAB0007C0AC0907D0AD0907E0AE0907F0AF090D8
:10AAC000800A6C197D098E099F0906171707280748
:10AAD000390728F4012B022B032B09F04CDB4091A2
:10AAE0009D0550919E0560919F057091A005452B95
:10AAF000462B472B19F10E9416C300917D0A109135
:10AB00007E0A20917F0A3091800A601B710B820BB4
:10AB1000930B00919D0510919E0520919F0530910A
:10AB2000A005061717072807390740F49091B510BC
:10AB30008091B410981302C0CC2349F0CF911F919B
:10AB40000F91FF90EF90DF90CF900C9425B4179A5F
:10AB50001092580C169A1092590C159A10925A0C81
:10AB6000149AECCF0E942D2A80916F0A811151C056
:10AB700081E080936F0A8091160C9091170CA09140
:10AB8000180CB091190C8093120C9093130CA09395
:10AB9000140CB093150CEBE3F2E28491882341F09E
:10ABA0009091C00095FFFCCF8093C6003196F5CF01
:10ABB000E091780CF0E0EE0FFF1FE45EFD4F019096
:10ABC000F081E02DE859FE4F0190F081E02D849155
:10ABD000882341F09091C00095FFFCCF8093C60080
:10ABE0003196F5CF8091C00085FFFCCF8AE080933D
:10ABF000C600E091780CF0E0EE0FFF1FE45EFD4F21
:10AC00000190F081E02DE453FF4F808191810C94FD
:10AC1000E883089580916F0A0895CF93DF93EC0144
:10AC20008091530C8093700A84E50E94C24B81117D
:10AC300002C080E0B8C00E94AE4B0E94F9C8609389
:10AC4000700A6623B1F3E5E3F2E28491882341F0D0
:10AC50009091C00095FFFCCF8093C6003196F5CF50
:10AC6000CD36D10509F454C0BCF4C836D10561F124
:10AC7000C936D10509F087C0E091780CF0E0EE0FFD
:10AC8000FF1FE45EFD4F0190F081E02DE25BFE4F7F
:10AC90000190F081E02D38C0CA3DD10509F451C0C2
:10ACA000CD3DD10509F06FC0E091780CF0E0EE0FDA
:10ACB000FF1FE45EFD4F0190F081E02DEC5AFE4F46
:10ACC0000190F081E02D5CC0E091780CF0E0EE0F97
:10ACD000FF1FE45EFD4F0190F081E02DE45BFE4F2D
:10ACE0000190F081E02D8191882309F44CC090916E
:10ACF000C00095FFFCCF8093C600F5CF9091C000B7
:10AD000095FFFCCF8093C60081918111F7CF3BC0A6
:10AD1000E091780CF0E0EE0FFF1FE45EFD4F019034
:10AD2000F081E02DE85AFE4F0190F081E02D8191F5
:10AD3000882349F19091C00095FFFCCF8093C60015
:10AD4000F6CFE091780CF0E0EE0FFF1FE45EFD4FD0
:10AD50000190F081E02DEE5AFE4F0190F081E02D40
:10AD60008191882381F09091C00095FFFCCF809362
:10AD7000C600F6CF9091C00095FFFCCF8093C6002F
:10AD800081918111F7CF40E050E06091700A83EE2D
:10AD90009FE00E9491A38091C00085FFFCCF8AE0D4
:10ADA0008093C60081E0DF91CF910895CF92DF922A
:10ADB000EF92FF922091770C2223F1F020E030E017
:10ADC00040E05FE30E945ACB6B017C0120E030E061
:10ADD000A9010E9485C8882379F0A7019601C701BF
:10ADE000B6010E945ACB2BED3FE049E450E40E94AB
:10ADF0005ACB9B01AC0104C020E030E040E85FE3A7
:10AE000060E070E080E89FE30E948CC8FF90EF90C4
:10AE1000DF90CF9008956091D3057091D405809113
:10AE2000D5059091D605C2DF6093CF057093D0050C
:10AE30008093D1059093D20508953F924F925F92EF
:10AE40006F927F928F929F92AF92BF92CF92DF923A
:10AE5000EF92FF920F931F93CF93DF93CDB7DEB79F
:10AE6000E9970FB6F894DEBF0FBECDBF81E40E9414
:10AE7000C24B882309F43FC082E70E94C24B88235B
:10AE8000A9F0E3E3F7E08191882339F09091C000C5
:10AE900095FFFCCF8093C600F6CF8091C00085FF60
:10AEA000FCCF8AE08093C6000C94A36F86E70E94D3
:10AEB000C24B8823A9F0E9E3F7E08191882339F0B8
:10AEC0009091C00095FFFCCF8093C600F6CF809193
:10AED000C00085FFFCCF8AE08093C6000C94A36F6E
:10AEE00087E60E94C24B882311F40C94A36F0E9442
:10AEF00093830C94A36F87E40E94C24B882309F4C8
:10AF00006EC20E94AE4B0E94F4C86A30710509F40B
:10AF1000BBC09CF46230710509F44CC024F477FF87
:10AF200025C00C94A36F6330710509F44EC06430E2
:10AF3000710509F455C00C94A36F6A35710509F4C5
:10AF4000FAC154F46B30710509F4A4C06C31710579
:10AF500009F4A6C00C94A36F6B35710509F4EFC119
:10AF60006C35710509F4F0C10C94A36F80916F0AE0
:10AF700081110C94A36F0E94564C8091500C882331
:10AF8000A9F088E50E94C24B811110C089E50E949A
:10AF9000C24B81110BC08AE50E94C24B811106C0D1
:10AFA00085E40E94C24B81110C94A66F0E949C4DB7
:10AFB0000C94A36F80916F0A81110C94A36F0E946F
:10AFC000D54C81E026D80C94A36F80916F0A811133
:10AFD0000C94A36F0E94D54C80E01BD80C94A36FF7
:10AFE000E091780CF0E0EE0FFF1FE45EFD4F019062
:10AFF000F081E02DE054FF4F808191810E94E88331
:10B0000080E50E94C24B882339F00E94AE4B0E941B
:10B01000F9C84B015C0103C0812C912C540183E5DC
:10B020000E94C24B882361F00E94AE4B20E030E0CA
:10B030004AE754E40E945ACB0E94F9C84B015C01D4
:10B040000E94AEAC0E9416C36B017C01C80CD91CD7
:10B05000EA1CFB1C0E9416C360937D0A70937E0A53
:10B0600080937F0A9093800A0E9416C36C157D0519
:10B070008E059F0510F00C94A36F0E945A2780E064
:10B08000FFDC0E949784F0CF60E081E00E945B4E7D
:10B090000C94A36F60E080E00E945B4E0C94A36F61
:10B0A0008091A1059091A205A091A305B091A4055E
:10B0B00080931E0C90931F0CA093200CB093210C36
:10B0C0008091DD059091DE0590937C0C80937B0C44
:10B0D00084E690E09093DE058093DD050E9416C320
:10B0E00060937D0A70937E0A80937F0A9093800A12
:10B0F00081E00E942EA58091670C9091680CA09130
:10B10000690CB0916A0C8093320C9093330CA0932D
:10B11000340CB093350C80916B0C90916C0CA09119
:10B120006D0CB0916E0C8093360C9093370CA093FD
:10B13000380CB093390C80916F0C9091700CA091E9
:10B14000710CB091720C80933A0C90933B0CA093CD
:10B150003C0CB0933D0C8091730C9091740CA091B9
:10B16000750CB091760C80933E0C90933F0CA0939D
:10B17000400CB093410C1092A1051092A2051092C0
:10B18000A3051092A40588E50E94C24B882311F004
:10B1900090E00AC089E50E94C24B8111F9CF8AE58F
:10B1A0000E94C24B91E098279093A50591110C94B1
:10B1B000D56F88E50E94C24B81110C94D56F8091A8
:10B1C000A50581110C94DB6F89E50E94C24B8111AA
:10B1D0000C94DB6F88E50E94C24B8823D1F00E945B
:10B1E000B74B672B682B692BA1F00E94AE4B2091C7
:10B1F0005B0C30915C0C40915D0C50915E0C0E9498
:10B20000ACC76093670C7093680C8093690C909343
:10B210006A0C89E50E94C24B8823D1F00E94B74B8B
:10B22000672B682B692BA1F00E94AE4B20915F0C1D
:10B230003091600C4091610C5091620C0E94ACC73F
:10B2400060936B0C70936C0C80936D0C90936E0CF0
:10B250008091A50581110C94E16F8AE50E94C24B93
:10B2600081110C94E16F8AE50E94C24B8823D1F0D2
:10B270000E94B74B672B682B692BA1F00E94AE4B45
:10B280002091630C3091640C4091650C5091660CD8
:10B290000E94ACC760936F0C7093700C8093710C1C
:10B2A0009093720C23E73CE04FE65CE06BE67CE0B9
:10B2B00087E69CE00E9423BE80E00E942EA580913C
:10B2C0001E0C90911F0CA091200CB091210C80932A
:10B2D000A1059093A205A093A305B093A405809126
:10B2E0007B0C90917C0C9093DE058093DD050E9491
:10B2F00016C360937D0A70937E0A80937F0A9093B1
:10B30000800A0E9427A58091890C882311F40C944F
:10B31000A36F65E87CE089EF9FE00E945C808091EC
:10B32000850C9091860C892B11F40C94A36F0E94CC
:10B3300007970C94A36F1092110C0C94A36F81E0EB
:10B340008093110C0C94A36F85E40E94C24B811171
:10B3500002C00E94AEAC95EAC92E97E0D92E2BE52B
:10B36000E22E2CE0F22E07E61CE0B12CF6018191D2
:10B370006F010E94C24B882339F1F3E0BF120CC069
:10B380000E94AE4BF801608371838283938383E7CD
:10B390009CE00E94C8BE18C00E94AE4BF7012081FD
:10B3A0003181428153810E94ACC7F801608371836F
:10B3B0008283938323E73CE04FE65CE06BE67CE02E
:10B3C00087E69CE00E9423BEB394F4E0EF0EF11CEC
:10B3D0000C5F1F4F24E0B212C9CF0C94A36F8DE411
:10B3E0000E94C24B882311F40C94AA6E0E94AE4BAB
:10B3F0000E94F4C86537710511F40C9400630CF0D9
:10B40000D0C06032710509F453C30CF071C06731CC
:10B41000710509F4A8C20CF044C06231710511F441
:10B420000C941F621CF577FF02C00C94A36F62306E
:10B4300071050CF498C16131710511F00C94A36F82
:10B44000E091780CF0E0EE0FFF1FE45EFD4F0190FD
:10B45000F081E02DE853FF4F808191810E94E883C5
:10B4600017981698159814980C94A36F6531710568
:10B4700009F46DC20CF071C26431710511F00C94C5
:10B48000A36FE091780CF0E0EE0FFF1FE45EFD4F3C
:10B490000190F081E02DE85BFE4F0190F081E02DFE
:10B4A00025C26B31710509F48AC2B4F469317105A2
:10B4B00009F471C20CF075C287E89CE00E94D03A92
:10B4C0000E9416C36093750A7093760A8093770A78
:10B4D0009093780A0C94A36F6E31710509F4AAC297
:10B4E0000CF082C36C31710509F46FC20C94A36F28
:10B4F0006C35710509F4F6C7ECF46235710509F491
:10B5000095C764F46035710509F448C70CF05DC750
:10B510006A32710509F4C6C30C94A36F64357105D2
:10B5200009F48DC70CF486C76535710509F4BFC7EA
:10B530000C94A36F6B36710509F42AC764F469365D
:10B54000710509F427C40CF0F3C66836710509F4D7
:10B55000F0C30C94A36F6037710509F408C434F488
:10B560006D36710509F423C50C94A36F623771051C
:10B5700011F40C9414636337710511F00C94A36FEC
:10B58000E091780CF0E0EE0FFF1FE45EFD4F0190BC
:10B59000F081E02DEE59FE4F0190F081E02D0C94EA
:10B5A000FB62623E710511F40C9413680CF05FC0ED
:10B5B0006B3C710511F40C945266ACF56C38710556
:10B5C00009F4D7C304F56837710511F40C940164CC
:10B5D0006937710511F40C9406646737710511F031
:10B5E0000C94A36FE091780CF0E0EE0FFF1FE45E87
:10B5F000FD4F0190F081E02DE258FE4F0190F08167
:10B60000E02D0C941164683C710511F40C94AF6545
:10B61000693C710511F40C9431666E3B710511F0B3
:10B620000C94A36F5AC56F3C710511F40C940F670D
:10B6300054F46D3C710511F40C94916614F40C945F
:10B640006F660C94F166613D710511F40C946E67A0
:10B6500014F40C9446676C3D710511F40C94DE678C
:10B660006D3D710511F40C94ED670C94A36F653F6B
:10B6700031E0730711F40C94C06954F56F3291E016
:10B68000790711F40C94856984F46D32F1E07F0739
:10B6900011F40C94A46814F00C9477696C32714026
:10B6A00011F40C946E680C94A36F6F3581E07807E9
:10B6B00011F40C944E6E603991E0790711F40C94FA
:10B6C000BD696E35714011F00C94A36F0C94176E28
:10B6D0006835F2E07F0711F40C94086BA4F4673F1F
:10B6E00031E0730711F40C94C86914F40C94C56923
:10B6F0006D3F714011F00C94A36F0E949383E5E3BA
:10B70000F2E20C94D2696B38E3E07E0711F40C94FA
:10B71000F16D3CF46335734011F40C94E3690C94BF
:10B72000A36F603A33E0730709F42BC2673E73409E
:10B7300011F00C94A36F10926F0A0E94FB8380910A
:10B74000120C9091130CA091140CB091150C8093D5
:10B75000160C9093170CA093180CB093190C0E9420
:10B760001E4C0C94A36F0091810A1091820A0E5F07
:10B770001F4F80E50E94C24B882379F00E94AE4B98
:10B780000E94F9C86B017C01BB24B394611571055B
:10B790008105910531F4B12C04C0B12CC12CD12C00
:10B7A000760183E50E94C24B882399F00E94AE4B3C
:10B7B00020E030E04AE754E40E945ACB0E94F9C8E6
:10B7C0006B017C01AA24A394611571058105910583
:10B7D00009F4A12C6AE270E0C8010E9411D0009720
:10B7E00011F0FC011082F801CF0121912032E1F328
:10B7F000B11007C0A11005C0222319F00E94B88320
:10B8000010C0E091780CF0E0EE0FFF1FE45EFD4FFA
:10B810000190F081E02DEE53FF4F808191810E94D5
:10B82000E88381E00E9498830E94AEAC0E9416C318
:10B8300060937D0A70937E0A80937F0A9093800ABA
:10B84000C114D104E104F104D1F00E9416C34B01EC
:10B850005C018C0C9D1CAE1CBF1C0E9416C368159D
:10B8600079058A059B05E0F40E947B85811118C04B
:10B870000E945A2780E004D90E949784EECF0E944C
:10B880007985882311F40C94A36F0E947B85811124
:10B890000AC00E945A2780E0F3D80E949784F5CF0F
:10B8A00080E00E9498838091890CE091780CF0E010
:10B8B000EE0FFF1FE45EFD4F0190F081E02D882325
:10B8C00041F0EC53FF4F808191810E94E8830C94FA
:10B8D000A36F808191810E94E8830C94A36F909163
:10B8E000C00095FFFCCF8093C600319684918111F2
:10B8F000F6CF8091C00085FFFCCF8AE08093C60020
:10B9000087E89CE00E947839E091780CF0E0EE0F37
:10B91000FF1FE45EFD4F0190F081E02DE65BFE4FDE
:10B920000190F081E02D8491882341F09091C00036
:10B9300095FFFCCF8093C6003196F5CF8091C00073
:10B9400085FFFCCF8AE08093C6000C94A36F87E844
:10B950009CE00E94CD390C94A36F87E89CE00E9484
:10B96000CC3A0C94A36F0091810A1091820A0C5F6B
:10B970001F4F6AE270E0C8010E9411D0009711F0D9
:10B98000FC01108221E041E0B80187E89CE00E94C0
:10B990004E3F0C94A36F87E89CE00E94D73A0C942A
:10B9A000A36F80918A0C882311F40C94A36F83E514
:10B9B0000E94C24B81110C94E76F0C94A36F87E82F
:10B9C0009CE00E947B3C0C94A36F8091810A909133
:10B9D000820A6AE270E004960E9411D08C010097FE
:10B9E000D9F020918B0A30918C0A40E6429FC00129
:10B9F000439F900D11246EE470E08F56954F0E9486
:10BA000011D060E270E00E9411D001969093820AFA
:10BA10008093810AF80110826091810A7091820AF4
:10BA20006C5F7F4F21E040E087E89CE00E944E3F42
:10BA30000C94A36F80918A0C882311F40C94A36F4B
:10BA400060E087E89CE00E94DE3E8091810A909150
:10BA5000820A6AE270E004960E9411D08C0100977D
:10BA6000D9F020918B0A30918C0A40E6429FC001A8
:10BA7000439F900D11246EE470E08F56954F0E9405
:10BA800011D060E270E00E9411D001969093820A7A
:10BA90008093810AF80110826091810A7091820A74
:10BAA0006C5F7F4F87E89CE00E943B3B0C94A36F48
:10BAB0008091890C81110E94AEAC0091810A109195
:10BAC000820A0C5F1F4F6AE270E0C8010E9411D029
:10BAD0007C0161E270E0C8010E9411D0009719F06A
:10BAE0008C010F5F1F4FE114F10411F0F701108278
:10BAF00080E50E94C24BF82E2091810A3091820A83
:10BB00000217130708F4F12C80918A0C882311F492
:10BB10000C94A36F21E02F2541E0B80187E89CE059
:10BB20000E944E3F83E50E94C24B8823B9F02091CA
:10BB3000810A3091820A2017310780F40E94B74BA6
:10BB4000AB01BC014093240F5093250F6093260F47
:10BB50007093270F8FE69EE00E94911B87E89CE080
:10BB60000E94D03AF1100C94A36F0E9416C3609308
:10BB7000750A7093760A8093770A9093780A0C94EA
:10BB8000A36F8091810A9091820A6AE270E0059623
:10BB90000E9411D08C010097D9F020918B0A30912E
:10BBA0008C0A40E6429FC001439F900D11246EE431
:10BBB00070E08F56954F0E9411D060E270E00E94B5
:10BBC00011D001969093820A8093810AF801108225
:10BBD0006091810A7091820A6B5F7F4F87E89CE0D9
:10BBE0000E94D3420C94A36F0E9416C36093710A03
:10BBF0007093720A8093730A9093740A0091750A85
:10BC00001091760A2091770A3091780A601B710BA7
:10BC1000820B930B28EE33E040E050E00E9463CCAF
:10BC2000CA01B9012CE330E040E050E00E9463CC4F
:10BC30007F936F933F932F938DE791E29F938F9321
:10BC4000CE0101969F938F930E9449D0E5E3F2E2E3
:10BC500084910FB6F894DEBF0FBECDBF882349F0A4
:10BC60009091C00095FFFCCF8093C60031968491DF
:10BC7000F5CFFE0131968191882339F09091C00073
:10BC800095FFFCCF8093C600F6CF8091C00085FF62
:10BC9000FCCF8AE08093C600CE0101960E94B88353
:10BCA0000C94A36F83E50E94C24B882311F40C947B
:10BCB000A36F0E94AE4B0E94F4C8F62EE72E862F8B
:10BCC0009E2D8C0180E50E94C24B882331F00F3FEE
:10BCD000110509F010F40C94F86F0DE010E0EDE69A
:10BCE000F7E0819191918017910711F40C94A36F63
:10BCF00037E0E53AF307A9F70830110539F48F2D3D
:10BD00009E2D9093520C8093510C04C017FF02C0DB
:10BD10000C94A36F61E0802F0E9436C26F2D802F9C
:10BD20000E946FC26F2D7E2D802F0E942CC10C941B
:10BD3000A36F88E690E00E940D5681110C94A36FCA
:10BD400083E50E94C24B882371F00091700A0E9423
:10BD5000AE4B10E0000F111F0A5A154F0E94F4C895
:10BD6000F801718360830E942C2A0C94A36F0E94B7
:10BD7000BB5083E50E94C24B882311F40C94A36F3F
:10BD80000E94AE4B0E94F4C87093550A6093540A07
:10BD90000C94A36F89E690E00E940D5681110C94DB
:10BDA000A36FE7E7F1E28491882341F09091C0000E
:10BDB00095FFFCCF8093C6003196F5CFE091700AD5
:10BDC00024E0E29FF0011124E25BF54F40815181B4
:10BDD0006281738121E030E083EE9FE00E9430A415
:10BDE000E4E7F1E28491882341F09091C00095FF4F
:10BDF000FCCF8093C6003196F5CFE091700AF0E059
:10BE0000EE0FFF1FEA5AF54F60817181882777FD99
:10BE10008095982F0E9427C9AB01BC0121E030E03A
:10BE200083EE9FE00E9430A4E0E7F1E28491882352
:10BE300041F09091C00095FFFCCF8093C6003196F1
:10BE4000F5CF4091480A5091490A60914A0A709191
:10BE50004B0A21E030E083EE9FE00E9430A4EDE643
:10BE6000F1E28491882341F09091C00095FFFCCFCE
:10BE70008093C6003196F5CF6091540A7091550AAF
:10BE8000882777FD8095982F0E9427C9AB01BC01B8
:10BE900021E030E083EE9FE00E9430A4EAE6F1E288
:10BEA0008491882341F09091C00095FFFCCF80934E
:10BEB000C6003196F5CF4AE050E060E070E083EED6
:10BEC0009FE00E945AA3E8E6F1E28491882341F0C2
:10BED0009091C00095FFFCCF8093C6003196F5CFBE
:10BEE00040914E0A50914F0A6091500A7091510A48
:10BEF00021E030E083EE9FE00E9430A4E5E6F1E22D
:10BF00008491882341F09091C00095FFFCCF8093ED
:10BF1000C6003196F5CF6091560A7091570A88276E
:10BF200077FD8095982F0E9427C9AB01BC0121E0C5
:10BF300030E083EE9FE00E9430A4E1E6F1E28491DC
:10BF4000882341F09091C00095FFFCCF8093C600FC
:10BF50003196F5CF8091700A90E00E9424274AE044
:10BF600050E0BC0183EE9FE00E945AA3ECE5F1E2B1
:10BF70008491882341F09091C00095FFFCCF80937D
:10BF8000C6003196F5CF8FEF9FEF0E9424274AE03D
:10BF900050E0BC0183EE9FE00E945AA38091C00054
:10BFA00085FFFCCF8AE08093C6000C9462718DE619
:10BFB00090E00E940D5681110C94A36FE091780CD3
:10BFC000F0E0EE0FFF1FE45EFD4F0190F081E02DE9
:10BFD000E65AFE4F808191810E94E88383E50E94AA
:10BFE000C24B882391F00091700A0E94AE4B10E082
:10BFF000000F111F0A5A154F0E94F4C8F8017183EF
:10C00000608381E080939C0515C082E50E94C24B4D
:10C01000882381F00091700A0E94AE4B10E0000F5F
:10C02000111F0A5A154F0E94F4C8F80171836083EA
:10C0300010929C050E942C2A0E9416C34B015C01A1
:10C040000091700A10E0F801EE0FFF1FEA5AF54F59
:10C0500060817181882777FD8095982F0E9427C97C
:10C06000F801EE0FFF1FEE0FFF1FE25BF54F11E02F
:10C0700020813181428153810E9488CA18160CF0B8
:10C0800010E010936E0A1092420CCC24CA94DC2C5F
:10C090007601F8EE4F2EF3E05F2E612C712CAAE0B2
:10C0A0003A2E8091420C81110C94FF6FFFEFCF1656
:10C0B000DF06EF06FF0611F40C942C70F7FE02C0A9
:10C0C0000C94FF6F0E9416C36C197D09683B7B407E
:10C0D00010F40C942C700C94FF6FE091780CF0E04D
:10C0E000EE0FFF1FE45EFD4F0190F081E02DE25A5C
:10C0F000FE4F808191810E94E88383E50E94C24BBC
:10C10000882361F00E94AE4B0E94F4C87093550AD8
:10C110006093540A81E080939C050FC082E50E94E1
:10C12000C24B882351F00E94AE4B0E94F4C870931A
:10C13000550A6093540A10929C050E9416C34B0145
:10C140005C011092420C6091540A7091550A882744
:10C1500077FD8095982F0E9427C911E02091480A09
:10C160003091490A40914A0A50914B0A0E9488CA6C
:10C1700018160CF010E010936E0A0EE411E28AE437
:10C18000E82E81E2F82E96E4C92E91E2D92E2AE01B
:10C19000722E80916E0A6091540A7091550A88231C
:10C1A00009F48BC08091420C811187C0882777FDEC
:10C1B0008095982F0E9427C92091480A3091490AFA
:10C1C00040914A0A50914B0A0E9488CA18160CF0F6
:10C1D0008BC00E9416C3681979098A099B09693EB8
:10C1E00073408105910508F460C0E091530C84E030
:10C1F000E89FF0011124E25BF54F4081518162819B
:10C200007381F8018491EEE4F1E2882349F0909182
:10C21000C00095FFFCCF8093C60031968491F5CF86
:10C2200022E030E083EE9FE00E9430A4F701849189
:10C23000EAE4F1E2882349F09091C00095FFFCCF39
:10C240008093C60031968491F5CF6091530C70E0D5
:10C250004AE050E083EE9FE00E945AA3F6018491E9
:10C26000E6E4F1E2882349F09091C00095FFFCCF0D
:10C270008093C60031968491F5CF4091480A509141
:10C28000490A60914A0A70914B0A21E030E083EE3E
:10C290009FE00E9430A48091C00085FFFCCF709287
:10C2A000C6000E9416C34B015C010E945A2780E021
:10C2B0000E9440550E9497846CCF882777FD809517
:10C2C000982F0E9427C92091480A3091490A40912D
:10C2D0004A0A50914B0A0E9485C887FF05C0809189
:10C2E0009C05882309F475CFE091780CF0E0EE0FFF
:10C2F000FF1FE45EFD4F0190F081E02DE05AFE4FFC
:10C30000808191810E94E8838091890C882321F0AB
:10C310008CE097E00E94B8830E9416C360937D0A68
:10C3200070937E0A80937F0A9093800A0C94A36F87
:10C3300083E50E94C24B882319F10E94AE4B20E096
:10C3400030E0A9010E9485C887FD0FC00E94AE4B56
:10C3500020E030E04FE753E40E9488CA181644F00A
:10C360000E94AE4B0E94F4C805C060E070E002C0BD
:10C370006FEF70E07093520C6093510C0C94A36FAC
:10C380008FEF90E09093520C8093510C0C94A36F1C
:10C390001092520C1092510C0C94A36F9B9AA3987C
:10C3A00081E08093A605E091780CF0E0EE0FFF1F8E
:10C3B000E45EFD4F0190F081E02D808191810E942B
:10C3C000E8830E9497840C94A36F0E942D2A0E94F8
:10C3D000AEAC149A0E9418AD1092520C1092510CEF
:10C3E00068EE73E080E090E00E9445C39B9AA39AB8
:10C3F0001092A605E091780CF0E0EE0FFF1FE45ECE
:10C40000FD4F0190F081E02DE459FF4F40815181B3
:10C4100024E431E262E471E282E597E00E94643351
:10C420000E94E8830E9497840C94A36F1092800C62
:10C430000C94A36F81E08093800C0C94A36F83E530
:10C440000E94C24B8823A1F00E94AE4B20E030E056
:10C450004AE754E40E945ACB0E94F9C860939D05B4
:10C4600070939E0580939F059093A0050C94A36FF5
:10C4700088E50E94C24B81110C94407189E50E94AD
:10C48000C24B81110C9440718AE50E94C24B81110C
:10C490000C94407185E40E94C24B81110C94407150
:10C4A0000E94AEAC149A0E9418AD0C94A36F83E561
:10C4B0000E94C24B882311F40C94A36F0E94AE4BD0
:10C4C00020E030E04AE754E40E945ACB0E94F9C8C9
:10C4D0006093790A70937A0A80937B0A90937C0A1E
:10C4E0000C94A36F25EA37E039AF28AF09EE15E1C8
:10C4F000E9EF8E2EE5E19E2EFDEAAF2EF5E1BF2E8F
:10C50000312CE8ADF9AD8191F9AFE8AF0E94C24B93
:10C51000882309F45BC0F3E03F1251C00E94AE4B88
:10C520006B017C0120E030E040EA51E40E9485C8C4
:10C5300087FF3FC0A7019601F80160817181828168
:10C5400093810E948CC82B013C019B01AC0160913E
:10C55000C1157091C2158091C3159091C4150E94A8
:10C560005ACB6093C1157093C2158093C3159093F5
:10C57000C415A3019201F4016081718182819381CC
:10C580000E945ACBF4016083718382839383F50107
:10C5900060817181828193810E9425C9A3019201EA
:10C5A0000E945ACB0E94F9C8F5016083718382838F
:10C5B0009383F801C082D182E282F38207C00E9495
:10C5C000AE4BF801608371838283938333940C5F55
:10C5D0001F4FF4E08F0E911C24E0A20EB11C34E03A
:10C5E00033128FCF0C94A36F9091C00095FFFCCFB6
:10C5F0008093C600319684918111F6CF0C94A36F7D
:10C600000091810A1091820A0B5F1F4F6AE270E06D
:10C61000C8010E9411D0009711F0FC011082C801DE
:10C620000E94B8830C94A36FEFE3F1E28491882316
:10C6300041F09091C00095FFFCCF8093C6003196E9
:10C64000F5CF4091670C5091680C6091690C709126
:10C650006A0C22E030E083EE9FE00E9430A4EBE31E
:10C66000F1E28491882341F09091C00095FFFCCFC6
:10C670008093C6003196F5CF40916B0C50916C0CB5
:10C6800060916D0C70916E0C22E030E083EE9FE0C3
:10C690000E9430A4E7E3F1E28491882341F0909175
:10C6A000C00095FFFCCF8093C6003196F5CF409136
:10C6B0006F0C5091700C6091710C7091720C22E0B3
:10C6C00030E083EE9FE00E9430A4E3E3F1E2849146
:10C6D000882341F09091C00095FFFCCF8093C60065
:10C6E0003196F5CF4091730C5091740C6091750C9C
:10C6F0007091760C22E030E083EE9FE00E9430A43F
:10C70000E091780CF0E0EE0FFF1FE45EFD4F01902A
:10C71000F081E02DEC59FE4F0190F081E02D8491E5
:10C72000882341F09091C00095FFFCCF8093C60014
:10C730003196F5CF0E940AAD0E9427C92091E915D4
:10C740003091EA154091EB155091EC150E948CC880
:10C75000AB01BC0122E030E083EE9FE00E9430A4F8
:10C76000EFE2F1E28491882341F09091C00095FFBF
:10C77000FCCF8093C6003196F5CF81E00E940AADD0
:10C780000E9427C92091ED153091EE154091EF15CB
:10C790005091F0150E948CC8AB01BC0122E030E042
:10C7A00083EE9FE00E9430A4EBE2F1E284918823C3
:10C7B00041F09091C00095FFFCCF8093C600319668
:10C7C000F5CF82E00E940AAD0E9427C92091F115A1
:10C7D0003091F2154091F3155091F4150E948CC8D8
:10C7E000AB01BC0122E030E083EE9FE00E9430A468
:10C7F0008091C00085FFFCCF8AE08093C6000C9436
:10C80000A36F80E00E942EA50C94A36F81E00E948C
:10C810002EA50C94A36F9091C00095FFFCCF809340
:10C82000C60081918111F7CF8091C00085FFFCCFB8
:10C830008AE08093C600E091780CF0E0EE0FFF1FD5
:10C84000E45EFD4F0190F081E02DEE58FE4F019027
:10C85000F081E02D8491882341F09091C00095FFF4
:10C86000FCCF8093C6003196F5CFE091780CF0E0D4
:10C87000EE0FFF1FE45EFD4F1E9B06C00190F0818E
:10C88000E02DE058FE4F05C00190F081E02DEE57FD
:10C89000FE4F90818181E92FF82F8191882339F013
:10C8A0009091C00095FFFCCF8093C600F6CF809199
:10C8B000C00085FFFCCF8AE08093C600E091780C31
:10C8C000F0E0EE0FFF1FE45EFD4F0190F081E02DE0
:10C8D000EC58FE4F0190F081E02D8491882341F0C7
:10C8E0009091C00095FFFCCF8093C6003196F5CFA4
:10C8F000E091780CF0E0EE0FFF1FE45EFD4F02992F
:10C9000006C00190F081E02DE058FE4F05C0019077
:10C91000F081E02DEE57FE4F90818181E92FF82FB5
:10C920008191882339F09091C00095FFFCCF8093CE
:10C93000C600F6CF8091C00085FFFCCF8AE08093CF
:10C94000C600E091780CF0E0EE0FFF1FE45EFD4FB3
:10C950000190F081E02DEA58FE4F0190F081E02D2A
:10C960008491882341F09091C00095FFFCCF809383
:10C97000C6003196F5CFE091780CF0E0EE0FFF1F86
:10C98000E45EFD4F1D9B06C00190F081E02DE05854
:10C99000FE4F05C00190F081E02DEE57FE4F9081D3
:10C9A0008181E92FF82F8191882339F09091C0007F
:10C9B00095FFFCCF8093C600F6CF8091C00085FF25
:10C9C000FCCF8AE08093C600E091780CF0E0EE0F97
:10C9D000FF1FE45EFD4F0190F081E02DE858FE4F0F
:10C9E0000190F081E02D8491882341F09091C00066
:10C9F00095FFFCCF8093C6003196F5CFE091780C7F
:10CA0000F0E0EE0FFF1FE45EFD4F019906C00190BC
:10CA1000F081E02DE058FE4F05C00190F081E02D3F
:10CA2000EE57FE4F90818181E92FF82F8191882365
:10CA300039F09091C00095FFFCCF8093C600F6CFEF
:10CA40008091C00085FFFCCF8AE08093C600E09112
:10CA5000780CF0E0EE0FFF1FE45EFD4F0190F081D7
:10CA6000E02DE658FE4F0190F081E02D849188235F
:10CA700041F09091C00095FFFCCF8093C6003196A5
:10CA8000F5CFE091780CF0E0EE0FFF1FE45EFD4F74
:10CA90001C9B06C00190F081E02DE058FE4F05C0C0
:10CAA0000190F081E02DEE57FE4F90818181E92FBA
:10CAB000F82F8191882339F09091C00095FFFCCF29
:10CAC0008093C600F6CF8091C00085FFFCCF8AE03E
:10CAD0008093C600E091780CF0E0EE0FFF1FE45E5B
:10CAE000FD4F0190F081E02DE458FE4F0190F08160
:10CAF000E02D8491882341F09091C00095FFFCCFF8
:10CB00008093C6003196F5CFE091780CF0E0EE0FFF
:10CB1000FF1FE45EFD4F379906C00190F081E02DC4
:10CB2000E058FE4F05C00190F081E02DEE57FE4F1A
:10CB300090818181E92FF82F8191882339F090919C
:10CB4000C00095FFFCCF8093C600F6CF8091C00057
:10CB500085FFFCCF8AE08093C6000C94A36F809180
:10CB6000530C8093700A84E50E94C24B882381F1A4
:10CB70000E94AE4B0E94F9C86093700A662341F18F
:10CB8000E5E3F2E28491882341F09091C00095FFA3
:10CB9000FCCF8093C6003196F5CFE091780CF0E0A1
:10CBA000EE0FFF1FE45EFD4F0190F081E02DE05B92
:10CBB000FE4F0190F081E02D8191882311F40C94B7
:10CBC000A36F9091C00095FFFCCF8093C600F4CF77
:10CBD00084E40E94C24B882311F40C94A36F0E943A
:10CBE000AE4B20E030E0A9010E9485C8811103C04E
:10CBF0001092770C32C00091700A10E00E94AE4B88
:10CC0000F801EE0FFF1FEE0FFF1FED52FA4F60838A
:10CC1000718382839383E090D305F090D4050091D3
:10CC2000D5051091D60520E030E0A901B701C80173
:10CC30000E9485C8811104C0E12CF12C00E410E4AD
:10CC4000C701D8018093D3059093D405A093D5054F
:10CC5000B093D60581E08093770C0E940B570C941B
:10CC6000A36F05EA17E029EDE22E25E1F22EF80187
:10CC700081918F010E94C24B882349F00E94AE4BE4
:10CC80000E94F9C8F7016083718382839383F4E083
:10CC9000EF0EF11C27E0093A120749F70E94F5BE92
:10CCA0000C94A36F05EA17E099EFE92E95E1F92EB0
:10CCB000F80181918F010E94C24B882339F00E94B4
:10CCC000AE4BF7016083718382839383F4E0EF0EB0
:10CCD000F11C27E0093A120759F70C94A36F83E57A
:10CCE0000E94C24B882351F00E94AE4B6093D11535
:10CCF0007093D2158093D3159093D41584E50E9438
:10CD0000C24B882311F40C94A36F0E94AE4B609326
:10CD1000CD157093CE158093CF159093D0150C94AC
:10CD2000A36F83E50E94C24B882351F00E94AE4B53
:10CD30006093D5157093D6158093D7159093D81519
:10CD400084E50E94C24B882351F00E94AE4B609351
:10CD5000BD157093BE158093BF159093C01582E4E6
:10CD60000E94C24B882361F00E94AE4B0E94F9C81A
:10CD70006093091670930A1680930B1690930C1605
:10CD800088E50E94C24B882351F00E94AE4B60930D
:10CD9000C9157093CA158093CB159093CC158AE56D
:10CDA0000E94C24B882351F00E94AE4B6093C51580
:10CDB0007093C6158093C7159093C81585E40E949B
:10CDC000C24B882311F40C94A36F0E94AE4B609366
:10CDD000C1157093C2158093C3159093C4150C941C
:10CDE000A36F05EA17E08BE5E82E8CE0F82EF8013A
:10CDF00081918F010E94C24B882339F00E94AE4B73
:10CE0000F7016083718382839383F4E0EF0EF11C5A
:10CE100027E0083A120711F40C94A36FE8CF83E5DA
:10CE20000E94C24B882351F00E94AE4B6093B30521
:10CE30007093B4058093B5059093B60586E40E947F
:10CE4000C24B882381F00E94AE4B20E030E040E7E7
:10CE500052E40E948CC86093AB057093AC0580933C
:10CE6000AD059093AE058AE50E94C24B882311F46C
:10CE70000C94A36F0E94AE4B60934B0C70934C0CC0
:10CE800080934D0C90934E0C0C94A36F83E50E94FD
:10CE9000C24B882351F00E94AE4B6093470C7093B5
:10CEA000480C8093490C90934A0C86E40E94C24B34
:10CEB000882311F40C94A36F0E94AE4B20E030E065
:10CEC00040E752E40E948CC86093A7057093A805C0
:10CED0008093A9059093AA050C94A36F83E50E9403
:10CEE000C24B882311F40C94A36F0E94AE4B0E9496
:10CEF000F4C86115710551F06130710569F481E084
:10CF00008093500C10924F0C0C94A36F1092500C05
:10CF100010924F0C0C94A36FE5E3F2E28491882306
:10CF200041F09091C00095FFFCCF8093C6003196F0
:10CF3000F5CFE091780CF0E0EE0FFF1FE45EFD4FBF
:10CF40000190F081E02DE459FE4F0190F081E02D39
:10CF50008491882341F09091C00095FFFCCF80938D
:10CF6000C6003196F5CF80918B0A90918C0A20E60D
:10CF7000289FF001299FF00D1124EF56F54F819164
:10CF8000882339F09091C00095FFFCCF8093C600B4
:10CF9000F6CFE9E2F1E28491882341F09091C0005C
:10CFA00095FFFCCF8093C6003196F5CF8091C000ED
:10CFB00085FFFCCF8AE08093C600C5C783E50E9449
:10CFC000C24B882309F4BFC70E94AE4B0E94F4C82D
:10CFD0007093DE056093DD05B6C783E50E94C24B02
:10CFE000882309F4B0C70E94AE4B0E94F4C86B01BD
:10CFF0007C0184E50E94C24B882381F08DED90E096
:10D000000E940D5681119FC7E091700AF0E0EE0F6B
:10D01000FF1FE752FA4FD182C08295C7D092DC053C
:10D02000C092DB0590C780E50E94C24B882309F4BB
:10D030008AC70E94AE4B0E94F4C8D62E062F172F27
:10D0400083E50E94C24B882331F00E94AE4B0E94C0
:10D05000F4C87B0103C0EE24EA94FE2CC7010196BC
:10D06000039708F070C7EDE6F7E081919191801782
:10D07000910709F468C737E0E53AF307B1F717FD00
:10D0800062C70E94AEACCD2C60E08D2D0E9436C2EE
:10D090008FEFE816F80631F0EA94EF2871F000E01F
:10D0A00010E00DC08D2D0E94A4C231E020E0892B3C
:10D0B00009F030E0032F122F02C001E010E08C2DA8
:10D0C0000E94A4C28017910709F43DC70E945A2705
:10D0D00080E00E9440550E949784F1CF83E50E9432
:10D0E000C24B882331F00E94AE4B0E94F4C88B01E2
:10D0F00002C00EE610E080E50E94C24B882331F0AA
:10D100000E94AE4B0E94F4C8CB0102C088EE93E0AF
:10D110006C01EE24D7FCE094FE2C101611067CF472
:10D1200020E030E0A901B80184E50E94E2C3C70114
:10D13000B6010E9445C384E50E94F3C604C7C70137
:10D14000B6010E9445C3FFC680E50E94C24B8823FA
:10D1500051F00E94AE4B60931802709319028093B5
:10D160001A0290931B0289E40E94C24B882361F04B
:10D170000E94AE4B0E949F30609314027093150280
:10D18000809316029093170284E40E94C24B882376
:10D1900061F00E94AE4B0E94AB306093100270931E
:10D1A0001102809312029093130283E40E94C24BF7
:10D1B000882351F00E94AE4B60930C0270930D02D5
:10D1C00080930E0290930F020E940D27E091780C3D
:10D1D000F0E0EE0FFF1FE45EFD4F0190F081E02DC7
:10D1E000E65CFE4F0190F081E02D8191882339F0BB
:10D1F0009091C00095FFFCCF8093C600F6CFEBE581
:10D20000F7E08191882339F09091C00095FFFCCF21
:10D210008093C600F6CF4091180250911902609198
:10D220001A0270911B0222E030E083EE9FE00E9420
:10D2300030A4EFE5F7E08191882339F09091C000A8
:10D2400095FFFCCF8093C600F6CF609114027091D9
:10D25000150280911602909117020E94A530AB0131
:10D26000BC0122E030E083EE9FE00E9430A4E3E6C0
:10D27000F7E08191882339F09091C00095FFFCCFB1
:10D280008093C600F6CF60911002709111028091D8
:10D290001202909113020E94B130AB01BC0122E056
:10D2A00030E083EE9FE00E9430A4E7E6F7E0819152
:10D2B000882339F09091C00095FFFCCF8093C60081
:10D2C000F6CF40910C0250910D0260910E027091C8
:10D2D0000F0222E030E083EE9FE00E9430A48091B4
:10D2E000C00085FFFCCF8AE08093C6002CC683E592
:10D2F0000E94C24B882319F00E94AE4B03C060E02D
:10D3000070E0CB010E94ECBE1EC685E40E94C24BB9
:10D31000882341F00E94AE4B0E94F4C88B0177FF36
:10D3200003C009C000E010E0C12CD12CF6E1EF2EC3
:10D33000F3E4FF2E06C0C12CD12CECE8EE2EE2E483
:10D34000FE2E83E50E94C24B882321F00E94AE4B43
:10D350006B017C0183E40E94C24B882331F00E9460
:10D36000AE4B0E94F4C89B0102C025E030E0A8014A
:10D37000C701B6010E94402AE6C50E94AEACE3C5D3
:10D380000E945FA00E94319CDEC50E945FA0DBC5A9
:10D390000E94319CD8C59091C00095FFFCCF80932E
:10D3A000C600319684918111F6CFE9E1F1E28491D2
:10D3B000882309F4C8C59091C00095FFFCCF8093E5
:10D3C000C6003196F4CF8AE50E94C24B882309F447
:10D3D000D6C00E94AE4B6B017C0120E030E040E7FC
:10D3E00051EC0E9488CA87FD57C020E030E040EA37
:10D3F00050ECC701B6010E9485C818160CF44CC049
:10D40000F7FAF094F7F8F094C092540CD092550CBF
:10D41000E092560CF092570CE5E3F2E284918823F7
:10D4200041F09091C00095FFFCCF8093C6003196EB
:10D43000F5CFE091780CF0E0EE0FFF1FE45EFD4FBA
:10D4400080819181FC01E65CFE4F40815181E25573
:10D45000F10928E131E262EC77E0808191810E945C
:10D460006433FC012491222341F03091C00035FF48
:10D47000FCCF2093C6000196F4CF8091C00085FFB9
:10D48000FCCF8AE08093C6008091C00085FFFCCF6E
:10D490008AE08093C60057C5E5E3F2E284918823D1
:10D4A00041F09091C00095FFFCCF8093C60031966B
:10D4B000F5CFE091780CF0E0EE0FFF1FE45EFD4F3A
:10D4C0000190F081E02DE851FF4F0190F081E02DB7
:10D4D0008491882341F09091C00095FFFCCF809308
:10D4E000C6003196F5CFE091780CF0E0EE0FFF1F0B
:10D4F000E45EFD4F0190F081E02DE658FE4F019073
:10D50000F081E02D8491882341F09091C00095FF37
:10D51000FCCF8093C6003196F5CF4AE050E061EF32
:10D520007FEF83EE9FE00E945AA3E091780CF0E039
:10D53000EE0FFF1FE45EFD4F0190F081E02DE458F7
:10D54000FE4F0190F081E02D8491882341F090916D
:10D55000C00095FFFCCF8093C6003196F5CF4AE01E
:10D5600050E06BEF7FEF83EE9FE00E945AA3809123
:10D57000C00085FFFCCF8AE08093C600E4C4E5E3E9
:10D58000F2E28491882341F09091C00095FFFCCF96
:10D590008093C6003196F5CFE091780CF0E0EE0F65
:10D5A000FF1FE45EFD4F0190F081E02DE851FF4F39
:10D5B00064E171E2808191810E944333FC012491F6
:10D5C000222341F03091C00035FFFCCF2093C600EC
:10D5D0000196F4CF8091C00085FFFCCF8AE0809354
:10D5E000C6004091540C5091550C6091560C7091AE
:10D5F000570C705822E030E083EE9FE00E9430A488
:10D600008091C00085FFFCCF8AE08093C6009BC458
:10D610008091DD059091DE059093D8058093D70524
:10D62000C090670CD090680CE090690CF0906A0C88
:10D63000CF8ED8A2E9A2FAA200916B0C10916C0CCB
:10D6400020916D0C30916E0C0BA31CA32DA33EA357
:10D6500040916F0C5091700C6091710C7091720C34
:10D660004FA358A769A77AA78091730C9091740C67
:10D67000A091750CB091760C8BA79CA7ADA7BEA707
:10D68000C982DA82EB82FC820D831E832F83388766
:10D6900049875A876B877C878D879E87AF87B88B32
:10D6A00085E40E94C24B882359F00E94AE4B9B0137
:10D6B000AC016BA57CA58DA59EA50E94ACC70AC038
:10D6C00020E030E040E050E46BA57CA58DA59EA550
:10D6D0000E94ABC76BA77CA78DA79EA793E5C92E19
:10D6E0009CE0D92EE12CF12C08EC13E49E01255D81
:10D6F0003F4FAE01495D5F4FBE016D5D7F4FCE0173
:10D700004F960E9441B48AE50E94C24B882349F09B
:10D710000E94AE4B9B01AC016FA178A589A59AA58B
:10D720001EC020E030E040E050E46FA178A589A55C
:10D730009AA50E94ACC76B017C016FA378A789A74B
:10D740009AA720E030E040E251E40E9485C887FFBC
:10D750000CC020E030E040E251E4C701B6010E9475
:10D76000ACC76FA378A789A79AA7B3E5CB2EBCE077
:10D77000DB2EE12CF12C06E913E49E01255D3F4FE1
:10D78000AE01495D5F4FBE016D5D7F4FCE014F968B
:10D790000E9441B488E50E94C24B882379F00E9420
:10D7A000AE4B9B01AC016F8D78A189A19AA10E941B
:10D7B000ACC76F8F78A389A39AA308C080E090E0DC
:10D7C000A3E5B3E48F8F98A3A9A3BAA389E50E9428
:10D7D000C24B882339F00E94AE4B6BA37CA38DA370
:10D7E0009EA304C01BA21CA21DA21EA2F3E5CF2E65
:10D7F000FCE0DF2EE12CF12C0CE812E49E01255D0B
:10D800003F4FAE01495D5F4FBE016D5D7F4FCE0161
:10D810004F960E9441B48CE40E94C24B882359F079
:10D820000E94AE4B9B01AC016BA57CA58DA59EA56E
:10D830000E94ACC70AC020E030E040EA52E46BA589
:10D840007CA58DA59EA50E94ABC76BA77CA78DA7C5
:10D850009EA773E5C72E7CE0D72EE12CF12C08ECB7
:10D8600013E49E01255D3F4FAE01495D5F4FBE0150
:10D870006D5D7F4FCE014F960E9441B40E94AEACC9
:10D88000149A64E670E080E090E00E9445C30E9434
:10D890001F9000E010E0F12C0E947B8581112AC0CE
:10D8A000F3940E945A2781E00E944055F110F4CF72
:10D8B000043FF1E01F0711F400E010E08091010146
:10D8C0008460809301010115110531F49FB7F8942C
:10D8D00080910201846008C00431110541F49FB7B2
:10D8E000F894809102018B7F809302019FBF0F5FAC
:10D8F0001F4FD2CF9FB7F894809102018B7F809306
:10D9000002019FBF20E030E04CE852E46BA57CA50B
:10D910008DA59EA50E94ACC76BA77CA78DA79EA7CF
:10D9200043E5C42E4CE0D42EE12CF12C00EA11E4A6
:10D930009E01255D3F4FAE01495D5F4FBE016D5DAC
:10D940007F4FCE014F960E9441B420E030E048E482
:10D9500052E46BA57CA58DA59EA50E94ACC76BA7C4
:10D960007CA78DA79EA7E12CF12C00E010E49E017E
:10D97000255D3F4FAE01495D5F4FBE016D5D7F4F3D
:10D98000CE014F960E9441B410927A0C1092790CFD
:10D990000E94B5908091790C90917A0C019709F4CE
:10D9A0007CC010927A0C1092790C0E9408918091A0
:10D9B000790C90917A0C8230910549F1039709F026
:10D9C00069C020E030E048E452E46BA57CA58DA559
:10D9D0009EA50E94ACC76BA77CA78DA79EA7B3E5A9
:10D9E000CB2EBCE0DB2EE12CF12C00E010E49E01FC
:10D9F000255D3F4FAE01495D5F4FBE016D5D7F4FBD
:10DA0000CE014F960E9441B40E946290C3CF20E0A5
:10DA100030E04CE852E46BA57CA58DA59EA50E9444
:10DA2000ACC76BA77CA78DA79EA793E5C92E9CE0EA
:10DA3000D92EE12CF12C00EA11E49E01255D3F4F27
:10DA4000AE01495D5F4FBE016D5D7F4FCE014F96C8
:10DA50000E9441B420E030E048E452E46BA57CA58C
:10DA60008DA59EA50E94ACC76BA77CA78DA79EA77E
:10DA7000E12CF12C00E010E49E01255D3F4FAE014A
:10DA8000495D5F4FBE016D5D7F4FCE014F960E9495
:10DA900041B47ECF0E944B907DCF20E030E040EA41
:10DAA00050E46BA57CA58DA59EA50E94ACC76BA775
:10DAB0007CA78DA79EA753E5C52E5CE0D52EE12C53
:10DAC000F12C00E010E49E01255D3F4FAE01495D61
:10DAD0005F4FBE016D5D7F4FCE014F960E9441B4F6
:10DAE000A80197016BA57CA58DA59EA50E94ABC73B
:10DAF0006BA77CA78DA79EA7E12CF12C08EC13E463
:10DB00009E01255D3F4FAE01495D5F4FBE016D5DDA
:10DB10007F4FCE014F960E9441B4E12CF12C0CE8CE
:10DB200012E49E01255D3F4FAE01495D5F4FBE018E
:10DB30006B5F7F4FCE0101960E9441B4E12CF12C26
:10DB400006E913E49E01255D3F4FAE01475F5F4F3D
:10DB5000BE016B5F7F4FCE0101960E9441B420E071
:10DB600030E040E050E46BA57CA58DA59EA50E9409
:10DB7000ACC76BA77CA78DA79EA7E12CF12C08EC66
:10DB800013E49E01255D3F4FAE01475F5F4FBE012D
:10DB90006B5F7F4FCE0101960E9441B4CE010D967E
:10DBA0000E94C8BE8091D7059091D8058093DD056D
:10DBB0009093DE059F938F938BE091E29F938F93D9
:10DBC0008E01015D1F4F1F930F930E9449D0C80122
:10DBD0000E948A480F900F900F900F900F900F9017
:10DBE000B2C188E50E94C24B882339F00E94AE4B37
:10DBF0000E94F4C880E00E94D8AD8AE50E94C24B22
:10DC0000882339F00E94AE4B0E94F4C881E00E9444
:10DC1000D8AD85E40E94C24B882309F494C10E94C8
:10DC2000AE4B0E94F4C882E00E94D8AD8CC183E55F
:10DC30000E94C24B811104C005EA17E0F12C10C00C
:10DC400010E00E94AE4B0E94F9C8812F0E94AEAE38
:10DC50001F5F1530B1F7F0CFF394F4E0FF1679F0C1
:10DC6000F80181918F010E94C24B8823A9F30E9481
:10DC7000AE4B0E94F9C88F2D0E94AEAEEDCF82E46C
:10DC80000E94C24B882339F00E94AE4B0E94F9C813
:10DC900084E00E94AEAE0E9474AF55C183E50E943D
:10DCA000C24B882309F453C00E94AE4B0E94F4C8B3
:10DCB0006130710541F06230710509F048C005EA34
:10DCC00017E0F12C25C005EA17E0F12CF80181914D
:10DCD0008F010E94C24B882341F00E94AE4B0E94EC
:10DCE000F4C84FEF8F2D0E9470AEF394F4E0FF1252
:10DCF000EDCF82E40E94C24B882349F10E94AE4BD3
:10DD00000E94F4C84FEF20C0F394F4E0FF1689F0AE
:10DD1000F80181918F010E94C24B8823A9F30E94D0
:10DD2000AE4B0E94F4C8462F6FEF8F2D0E9470AE4D
:10DD3000EBCF82E40E94C24B882349F00E94AE4B95
:10DD40000E94F4C8462F6FEF84E00E9470AE0E94DC
:10DD500074AFF9C084E50E94C24B882309F4A2C0C5
:10DD60000E94AE4B0E94F9C86093700A662309F4C2
:10DD700042C0E5E3F2E28491882341F09091C00033
:10DD800095FFFCCF8093C6003196F5CFEBE6F7E028
:10DD90008191882339F09091C00095FFFCCF80934A
:10DDA000C600F6CF40E050E06091700A83EE9FE03D
:10DDB0000E9491A3E091780CF0E0EE0FFF1FE45E6B
:10DDC000FD4F0190F081E02DE059FE4F0190F08170
:10DDD000E02D8191882339F09091C00095FFFCCF10
:10DDE0008093C600F6CF8091C00085FFFCCF8AE00B
:10DDF0008093C600A8C086E40E94C24B8823D9F055
:10DE00000E94AE4B6B017C016093220C7093230C3B
:10DE10008093240C9093250C20E030E0A9010E940F
:10DE200088CA181644F4C092A105D092A205E092C7
:10DE3000A305F092A405E5E3F2E28491882341F082
:10DE40009091C00095FFFCCF8093C6003196F5CF2E
:10DE5000E091780CF0E0EE0FFF1FE45EFD4F0190C3
:10DE6000F081E02DE259FE4F0190F081E02D81918B
:10DE7000882339F09091C00095FFFCCF8093C600B5
:10DE8000F6CF6091530C70E04AE050E083EE9FE0E3
:10DE90000E945AA38091C00085FFFCCF8AE0809346
:10DEA000C60051C0E5E3F2E28491882341F09091ED
:10DEB000C00095FFFCCF8093C6003196F5CFE0916E
:10DEC000780CF0E0EE0FFF1FE45EFD4F0190F08153
:10DED000E02DE459FE4F0190F081E02D84918823DC
:10DEE00041F09091C00095FFFCCF8093C600319621
:10DEF000F5CF80918B0A90918C0A20E6289FF00143
:10DF0000299FF00D1124EF56F54F8191882339F0A8
:10DF10009091C00095FFFCCF8093C600F6CFE9E05A
:10DF2000F1E28491882341F09091C00095FFFCCFED
:10DF30008093C6003196F5CF8091C00085FFFCCF5D
:10DF40008AE08093C6000E94E94BBCC1C0903E0CA1
:10DF5000D0903F0CE090400CF090410C2091730C5D
:10DF60003091740C4091750C5091760CC701B6013C
:10DF70000E94ABC72DEC3CEC4CEC5DE30E9488CAE0
:10DF8000181614F00C94D657C092730CD092740CDF
:10DF9000E092750CF092760C83E79CE00E94C8BE7C
:10DFA00060E080E00E945B4E8DC180E090E00E94C6
:10DFB000F8460C94DF5881E090E00E94F8460C94FB
:10DFC000EA5882E090E00E94F8460C9433590E948F
:10DFD000B74BAB01BC014093240F5093250F6093C6
:10DFE000260F7093270F8FE69EE00E94911BABCF08
:10DFF0000E94AE4B0E94F4C88B010C946F5EE091BE
:10E00000780CF0E0EE0FFF1FE45EFD4F0190F08111
:10E01000E02DE45AFE4F808191810E94E883809137
:10E02000890C882321F08CE097E00E94B8830E943D
:10E0300016C36093750A7093760A8093770A90935B
:10E04000780A0E9416C360937D0A70937E0A8093BB
:10E050007F0A9093800A77CF0E9416C368197909C6
:10E060008A099B09693E73408105910508F479C0CE
:10E07000E9E5F1E28491882341F09091C00095FF99
:10E08000FCCF8093C6003196F5CFE091700A24E072
:10E09000E29FF0011124E25BF54F408151816281E2
:10E0A000738121E030E083EE9FE00E9430A4E5E53B
:10E0B000F1E28491882341F09091C00095FFFCCF5C
:10E0C0008093C6003196F5CF6091700A70E04AE007
:10E0D00050E083EE9FE00E945AA3E1E5F1E28491D3
:10E0E000882341F09091C00095FFFCCF8093C6003B
:10E0F0003196F5CFF7FE03C0E0E5F7E025C00E94BA
:10E1000016C38B019C01C701B6016854744F8F4F31
:10E110009F4F601B710B820B930BA30192010E9416
:10E1200063CCBA01A9012AE030E083EE9FE00E94AF
:10E1300086A38091C00085FFFCCF0DC09091C000E8
:10E1400095FFFCCF8093C60081918111F7CF80911C
:10E15000C00085FFFCCF3092C6000E9416C34B0161
:10E160005C010E945A2780E00E9440550E949784DB
:10E17000FFEFCF16DF06EF06FF0609F046C08091DD
:10E180006E0AE091700AF0E08F01000F111F000F7E
:10E19000111F025B154FEE0FFF1FEA5AF54F60810A
:10E1A00071818823C9F0882777FD8095982F0E9478
:10E1B00027C920E030E040E85FE30E94ABC79B0145
:10E1C000AC01F80160817181828193810E9488CACB
:10E1D00087FF50C00C945160882777FD8095982F59
:10E1E0000E9427C920E030E040E85FE30E94ACC70E
:10E1F0009B01AC01F80160817181828193810E9451
:10E2000085C81816BCF50C945160F7FE02C00C943A
:10E210005160E091700AF0E08F01000F111F000FB4
:10E22000111F025B154FEE0FFF1FEA5AF54F608179
:10E230007181882777FD8095982F0E9427C99B01BF
:10E24000AC01F80160817181828193810E94ABC72A
:10E250000E94F4C897FF07C09095809570956195CE
:10E260007F4F8F4F9F4F663071058105910514F4E4
:10E270000C9451600E9416C36B017C010C94516098
:10E280000E94AEAC88E50E94C24B882319F0179A11
:10E290001092580C89E50E94C24B882319F0169AF7
:10E2A0001092590C8AE50E94C24B882319F0159AE6
:10E2B00010925A0C85E40E94C24B882309F443CE85
:10E2C000149A41CEE9960FB6F894DEBF0FBECDBFCB
:10E2D000DF91CF911F910F91FF90EF90DF90CF9042
:10E2E000BF90AF909F908F907F906F905F904F9076
:10E2F0003F900895CF93DF938091870A9091880A89
:10E30000039714F40E941B5160E087E89CE00E9490
:10E31000E83D8091870A9091880A892B09F47EC094
:10E320008091870C8823E1F080918B0A90918C0A70
:10E3300020E6289FE001299FD00D1124CF56D54F0C
:10E3400065EA71E2CE010E94BCCF892B59F5BE016E
:10E3500087E89CE00E946A3D8091880C882319F030
:10E360000E941D5745C0E091780CF0E0EE0FFF1FB2
:10E37000E45EFD4F0190F081E02DE65CFE4F0190E0
:10E38000F081E02D8491882341F09091C00095FFA9
:10E39000FCCF8093C6003196F5CF8091C00085FFF9
:10E3A000FCCF23C060E087E89CE00E94DE3EE09165
:10E3B000780CF0E0EE0FFF1FE45EFD4F0190F0815E
:10E3C000E02DE45CFE4F0190F081E02D84918823E4
:10E3D00041F09091C00095FFFCCF8093C60031962C
:10E3E000F5CF8091C00085FFFCCF8AE08093C60006
:10E3F0008091870A9091880A01979093880A809368
:10E40000870A80918B0A90918C0A019664E070E0F3
:10E410000E9450CC90938C0A80938B0A0E945A27BA
:10E4200080E00E9440550E944FA4DF91CF910C9450
:10E4300097848F929F92AF92BF92CF92DF92EF928A
:10E44000FF920F931F93CF93DF938C018C519E4FBC
:10E450000E942F37680189E8C80ED11C21F178018C
:10E4600081E4E81A8EEFF80AE70157018FE1A81A54
:10E47000B1086CED862E67E0962ECC15DD0599F07F
:10E48000FE01EE19FF09EA0DFB1D91828082FE015B
:10E4900078978081811102C06F97EFCFCE014B97A3
:10E4A0000E94741CF9CFC80186599F4F0E942F37D4
:10E4B000C801875B9F4FDF91CF911F910F91FF9014
:10E4C000EF90DF90CF90BF90AF909F908F900C9483
:10E4D0002F3787E89CE00C943B3787E89CE0A9CF76
:10E4E000FB016091F0057091F1057093570F6093F7
:10E4F000560F6091600F7091610F7093550F60938C
:10E50000540F62E06093EF0563EC7DE87093F105D2
:10E510006093F0059093530F8093520FF093510F37
:10E52000E093500F662757FD6095762F40934C0F70
:10E5300050934D0F60934E0F70934F0FC901AA2750
:10E5400097FDA095BA2F841B950BA60BB70B809354
:10E55000480F9093490FA0934A0FB0934B0F8081BF
:10E560009181AA2797FDA095BA2F841B950BA60B26
:10E57000B70B8093600F9093610FA093620FB093DD
:10E58000630F0895CF93DF93CDB7DEB7C054D109A1
:10E590000FB6F894DEBF0FBECDBF88E0E7E2F6E02D
:10E5A000DE01D99601900D928A95E1F788E0EFE2BD
:10E5B000F6E0DE01D19601900D928A95E1F788E0B0
:10E5C000E7E3F6E0DE01999601900D928A95E1F776
:10E5D00088E0EFE3F6E0DE01919601900D928A95D6
:10E5E000E1F788E0E7E4F6E0DE01599601900D924C
:10E5F0008A95E1F788E0EFE4F6E0DE0151960190BC
:10E600000D928A95E1F788E0E7E5F6E0DE011996DC
:10E6100001900D928A95E1F788E0EFE5F6E0DE01E2
:10E62000119601900D928A95E1F7AE01475C5F4F1C
:10E6300060E08BE69FE00E940433AE014F5C5F4FC9
:10E6400061E08BE69FE00E940433AE01475D5F4FBF
:10E6500062E08BE69FE00E940433AE014F5D5F4FA6
:10E6600063E08BE69FE00E940433AE01475E5F4F9C
:10E6700064E08BE69FE00E940433AE014F5E5F4F83
:10E6800065E08BE69FE00E940433AE01475F5F4F79
:10E6900066E08BE69FE00E940433AE014F5F5F4F60
:10E6A00067E08BE69FE00E940433C05CDF4F0FB64B
:10E6B000F894DEBF0FBECDBFDF91CF9108950F93C9
:10E6C0001F93CF93DF93EB01142F022F482F60E0AD
:10E6D0008BE69FE00E946631612F8BE69FE00E94EF
:10E6E000A4C711E1FE016491662311F0111117C056
:10E6F000112339F060E28BE69FE00E94A4C711501D
:10E70000F7CF602F8BE69FE00E94A4C760E28BE604
:10E710009FE0DF91CF911F910F910C94A4C78BE6DE
:10E720009FE00E94A4C721961150DCCFEF92FF9288
:10E730000F931F93CF93DF93EB01E42E8901F9012F
:10E7400001900020E9F7F22EFE1A92E1F90E482F0F
:10E7500060E08BE69FE00E9466316E2D8BE69FE0C5
:10E760000E94A4C7FE016491662311F0F11019C044
:10E770006AE38BE69FE00E94A4C7FF2039F060E2C5
:10E780008BE69FE00E94A4C7FA94F7CFB8018BE60E
:10E790009FE0DF91CF911F910F91FF90EF900C942C
:10E7A000A3C78BE69FE00E94A4C72196FA94DACF14
:10E7B0008093780C91E09093F205682F88EF9FE0AA
:10E7C0000E946DD280913F0F813019F482E08093D6
:10E7D0003F0F08951092DA0F87E89CE00E94F14302
:10E7E0001092690F089587E89CE00C94D03A87E86E
:10E7F0009CE00C94D73ACF9382E08093EF050E947F
:10E8000016C36C507E4F8F4F9F4F6093650F709370
:10E81000660F8093670F9093680F80910101846069
:10E8200080930101CAE09FB7F8948091020184604F
:10E83000809302019FBF84E690E00E9469C39FB766
:10E84000F894809102018B7F809302019FBF84E640
:10E8500090E00E9469C3C15031F7CF910895E091D3
:10E86000F005F091F105E817F90771F09093F105C3
:10E870008093F0054093600F5093610F6093620F97
:10E880007093630F2111B7CF089521E040E050E06D
:10E89000BA01E5CF21E040E050E0BA01E0CFCF92ED
:10E8A000DF92EF92FF920F931F93CF93DF938091AC
:10E8B000600F9091610FA091620FB091630F813052
:10E8C0009048A105B10540F01092600F1092610FC1
:10E8D0001092620F1092630F8091600F9091610F00
:10E8E000A091620FB091630FB695A7959795879504
:10E8F0004091690F50E060E070E084179507A6072B
:10E90000B70710F48093690FD091690F10916A0FC7
:10E9100012FB112710F9C0E0B1E1CB2ED12CE12C74
:10E92000F12C01E04091600F5091610F6091620FF6
:10E930007091630FD11138C08091EF058823C1F029
:10E94000E091780CF0E0EE0FFF1FE45EFD4F0190C8
:10E95000F081E02D8681978123E0423051056105E9
:10E96000710510F443E001C040E2BC018C2FA7DE2A
:10E97000112309F49CC18091600F9091610FA091C7
:10E98000620FB091630F0297A105B10508F08FC126
:10E9900032DF88E492E9DF91CF911F910F91FF90D0
:10E9A000EF90DF90CF9071CFD13051F58091EF058E
:10E9B000882389F0769567955795479523E04130F0
:10E9C00051056105710511F443E001C040E260E4C6
:10E9D00073E28C2F74DE112309F469C18091600FFA
:10E9E0009091610FA091620FB091630FB695A795BA
:10E9F000979587950197A105B10509F058C1C8CF32
:10EA0000D230B9F58091EF058823F1F0E091780CD0
:10EA1000F0E0EE0FFF1FE45EFD4F0190F081E02D6E
:10EA2000E854FE4F8081918176956795579547957B
:10EA300023E0423051056105710511F443E001C046
:10EA400040E2BC018C2F3BDE112309F430C18091E0
:10EA5000600F9091610FA091620FB091630FB69516
:10EA6000A795979587950297A105B10509F01FC154
:10EA70008FCFD330B9F58091EF058823F1F0E09185
:10EA8000780CF0E0EE0FFF1FE45EFD4F0190F08187
:10EA9000E02DE654FE4F80819181769567955795DC
:10EAA000479523E0433051056105710511F443E0BA
:10EAB00001C040E2BC018C2F02DE112309F4F7C033
:10EAC0008091600F9091610FA091620FB091630FE0
:10EAD000B695A795979587950397A105B10509F078
:10EAE000E6C056CFD430B9F58091EF058823F1F018
:10EAF000E091780CF0E0EE0FFF1FE45EFD4F019017
:10EB0000F081E02DE454FE4F8081918176956795E8
:10EB10005795479523E0443051056105710511F47F
:10EB200043E001C040E2BC018C2FC9DD112309F490
:10EB3000BEC08091600F9091610FA091620FB09163
:10EB4000630FB695A795979587950497A105B1058D
:10EB500009F0ADC01DCFD53051F58091EF05882368
:10EB600089F0769567955795479523E0453051058F
:10EB70006105710511F443E001C040E263E373E213
:10EB80008C2F9DDD112309F492C08091600F90912C
:10EB9000610FA091620FB091630FB695A7959795FD
:10EBA00087950597A105B10509F081C0F1CED63052
:10EBB00051F58091EF05882389F0769567955795F3
:10EBC000479523E0463051056105710511F443E096
:10EBD00001C040E26FE273E28C2F71DD112309F472
:10EBE00066C08091600F9091610FA091620FB0910B
:10EBF000630FB695A795979587950697A105B105DB
:10EC000009F055C0C5CED73041F58091EF05882376
:10EC100089F0769567955795479523E047305105DC
:10EC20006105710511F443E001C040E266E273E260
:10EC30008C2F45DD1123D9F18091600F9091610FE8
:10EC4000A091620FB091630FB695A79597958795A0
:10EC50000797A105B10559F59BCED83041F58091B4
:10EC6000EF05882389F0769567955795479523E0BA
:10EC7000483051056105710511F443E001C040E2DF
:10EC80006CE173E28C2F1BDD112389F08091600F02
:10EC90009091610FA091620FB091630FB695A79507
:10ECA000979587950897A105B10509F471CE8091D4
:10ECB000600F9091610FA091620FB091630F429726
:10ECC000A105B10540F0C092600FD092610FE092B3
:10ECD000620FF092630F4091600F5091610F60914D
:10ECE000620F7091630F7695679557954795809160
:10ECF000690F90E00396242F30E0821793074CF4BD
:10ED00008DEF840F8093690F0093EF05DCEFD40F34
:10ED1000CFEFCF5FDF5FC43008F404CEDF91CF9137
:10ED20001F910F91FF90EF90DF90CF9008957F9209
:10ED30008F929F92AF92BF92CF92DF92EF92FF920B
:10ED40000F931F93CF93DF938091600F9091610F8A
:10ED5000A091620FB091630F81309048A105B10579
:10ED600040F01092600F1092610F1092620F10929B
:10ED7000630F8091600F9091610FA091620FB0912D
:10ED8000630FB695A795979587954091690F50E0C9
:10ED900060E070E084179507A607B70710F480932A
:10EDA000690FE090690FD0906A0FD2FADD24D0F895
:10EDB000F12CCC24C39480913F0F81113BC0EE20F5
:10EDC00019F07724739437C08091EF05882301F1FF
:10EDD000E091780CF0E0EE0FFF1FE45EFD4F019034
:10EDE000F081E02DEA50FF4F608171818091600FCA
:10EDF0009091610FA091620FB091630F23E0029791
:10EE0000A105B10510F443E001C040E28F2D57DCAD
:10EE1000DD20B9F28091600F9091610FA091620F97
:10EE2000B091630F0297A105B10558F6E4DC86EEB8
:10EE300090E851C0712C80913F0F823009F05AC088
:10EE40007E1057C08091EF05882359F1E091780C2E
:10EE5000F0E0EE0FFF1FE45EFD4F0190F081E02D2A
:10EE6000E055FF4F0190F081E02D8091600F90916F
:10EE7000610FA091620FB091630FB695A79597951A
:10EE80008795472D50E060E070E023E084179507F8
:10EE9000A607B70711F443E001C040E2BF018F2D80
:10EEA0000EDCDD2031F18091600F9091610FA09117
:10EEB000620FB091630FB695A79597958795472DEB
:10EEC00050E060E070E084179507A607B70789F463
:10EED00092DC84EF98E9DF91CF911F910F91FF9021
:10EEE000EF90DF90CF90BF90AF909F908F907F90EA
:10EEF000CCCC73940CE112E0C0E0D0E08E2C912CCD
:10EF0000A12CB12C7E104AC08091EF05882319F105
:10EF1000D801ED91FC91EC54FE4F6081718180919C
:10EF2000600F9091610FA091620FB091630FB69541
:10EF3000A79597958795272D30E040E050E0821700
:10EF40009307A407B50719F420E24EE302C020E2BC
:10EF500040E28F2DB4DBDD2009F18091600F9091AC
:10EF6000610FA091620FB091630FB695A795979529
:10EF7000879588159905AA05BB0581F43CDC8C2F83
:10EF8000DF91CF911F910F91FF90EF90DF90CF9085
:10EF9000BF90AF909F908F907F900ACC73942196F2
:10EFA0000E5F1F4FC230D10509F0ACCF4091600F0A
:10EFB0005091610F6091620F7091630F7695679524
:10EFC00057954795872D90E0A0E0B0E04817590786
:10EFD0006A077B0788F0872D90E0880F991F0197BB
:10EFE000AA2797FDA095BA2F8093600F9093610F89
:10EFF000A093620FB093630F4091600F5091610F27
:10F000006091620F7091630F76956795579547955C
:10F010008091690F90E00396242F30E082179307C8
:10F020005CF48DEF840F8093690FC092EF05DCEFE5
:10F03000ED2EE40EFF24FA94F394E394B3E0BF15AD
:10F0400008F0B9CEDF91CF911F910F91FF90EF9013
:10F05000DF90CF90BF90AF909F908F907F9008955A
:10F060000F931F93CF93DF938091600F9091610F67
:10F07000A091620FB091630F81309048A105B10556
:10F0800040F01092600F1092610F1092620F109278
:10F09000630F8091600F9091610FA091620FB0910A
:10F0A000630FB695A795979587954091690F50E0A6
:10F0B00060E070E084179507A607B70710F4809307
:10F0C000690FD091690F10916A0F12FB112710F987
:10F0D000C0E001E08091600F9091610FA091620FFC
:10F0E000B091630FD11134C02091EF052223C1F0FC
:10F0F000E091780CF0E0EE0FFF1FE45EFD4F019011
:10F10000F081E02DEA50FF4F6081718123E002978A
:10F11000A105B10510F443E001C040E28C2FCFDA25
:10F12000112309F482C08091600F9091610FA0912A
:10F13000620FB091630F0297A105B10508F075C089
:10F140005ADB86EE90E8DF91CF911F910F919DCB16
:10F15000D130A9F52091EF052223D1F0E091780C70
:10F16000F0E0EE0FFF1FE45EFD4F0190F081E02D17
:10F1700062AD73ADB695A795979587952EE70197E4
:10F18000A105B10511F44EE301C040E28C2F97DADE
:10F19000112309F44AC08091600F9091610FA091F2
:10F1A000620FB091630FB695A795979587950197D4
:10F1B000A105B105D1F51FDB8FE09FE8BFC0D230BC
:10F1C000A1F52091EF052223D1F0E091780CF0E039
:10F1D000EE0FFF1FE45EFD4F0190F081E02D64AD66
:10F1E00075ADB695A795979587952EE70297A105DA
:10F1F000B10511F44EE301C040E28C2F60DA112317
:10F20000A1F08091600F9091610FA091620FB09179
:10F21000630FB695A795979587950297A105B105B8
:10F2200021F4E9DA86E19FE889C020E030E040E29D
:10F2300051E460913B0F70913C0F80913D0F909194
:10F240003E0F0E9485C887FF7EC08091600F90911D
:10F25000610FA091620FB091630FD330B1F520918F
:10F26000EF052223D1F0E091780CF0E0EE0FFF1FC4
:10F27000E45EFD4F0190F081E02D66AD77ADB6956F
:10F28000A795979587952EE70397A105B10511F4EA
:10F290004EE301C040E28C2F12DA111102C025E0CA
:10F2A00053C08091600F9091610FA091620FB09157
:10F2B000630FB695A795979587950397A105B10517
:10F2C00071F799DA8DE19FE839C0D43041F7209188
:10F2D000EF052223E1F0E091780CF0E0EE0FFF1F44
:10F2E000E45EFD4F0190F081E02DE05CFF4F608116
:10F2F0007181B695A795979587952EE70497A105F7
:10F30000B10511F44EE301C040E28C2FD8D911238E
:10F3100031F24091600F5091610F6091620F7091D6
:10F32000630F76956795579547954430510561056C
:10F33000710509F0B4CF5FDA89E49DE8DF91CF91E0
:10F340001F910F91A7CA23E04091600F5091610F68
:10F350006091620F7091630F769567955795479509
:10F36000822F90E0A0E0B0E0481759076A077B07BA
:10F3700088F0822F90E0880F991F0197AA2797FDA8
:10F38000A095BA2F8093600F9093610FA093620FA6
:10F39000B093630F4091600F5091610F6091620FC5
:10F3A0007091630F76956795579547958091690F92
:10F3B00090E00396242F30E0821793074CF48DEFF2
:10F3C000840F8093690F0093EF05DCEFD40FCFEF2C
:10F3D000CF5FDF5FC43008F47DCEDF91CF911F9106
:10F3E0000F91089580E090E0A0E8BFE380933B0F89
:10F3F00090933C0FA0933D0FB0933E0F31CE20E091
:10F4000044E064E18BE69FE00E949931BBD88BE633
:10F410009FE00C945A31F3DF20E040E050E0BA0165
:10F4200084EF98E91CCA1092570A1092560A10925B
:10F43000550A1092540A1092520C1092510CEBCFB4
:10F440008BE69FE00C945A318091D70F9091D80FA2
:10F450009093570A8093560A8091D50F9091D60FBA
:10F460009093550A8093540A1092520C1092510CAA
:10F47000D2DF0C942C2A8091D10F9091D20F9093CF
:10F48000570A8093560A8091CF0F9091D00F909396
:10F49000550A8093540A1092520C1092510CBBDF03
:10F4A0000C942C2A80910106909102069093570AA1
:10F4B0008093560A8091FF05909100069093550A1B
:10F4C0008093540A1092520C1092510CA4DF0C94A9
:10F4D0002C2A8091FD059091FE059093570A809308
:10F4E000560A8091FB059091FC059093550A8093F4
:10F4F000540A1092520C1092510C8DDF0C942C2A4D
:10F500008091F9059091FA059093570A8093560AD5
:10F510008091F7059091F8059093550A8093540ACD
:10F520001092520C1092510C76DF0C942C2A809180
:10F53000F5059091F6059093570A8093560A8091AD
:10F54000F3059091F4059093550A8093540A109214
:10F55000520C1092510C5FDF0C942C2A2F923F9288
:10F560004F925F926F927F928F929F92AF92BF92D3
:10F57000CF92DF92EF92FF920F931F93CF93DF937F
:10F58000CDB7DEB7A2970FB6F894DEBF0FBECDBFE2
:10F590008091EF05811104C080916A0F82FFB6C28D
:10F5A00087E89CE00E94D8424091600F5091610F23
:10F5B0006091620F7091630F413050486105710591
:10F5C00040F01092600F1092610F1092620F109233
:10F5D000630F4091600F5091610F6091620F7091C5
:10F5E000630F76956795579547950091690F10E0E1
:10F5F00020E030E0401751076207730710F4409392
:10F60000690F4090690F30906A0F32FA332430F856
:10F61000512C9C012150310939A328A3411035C038
:10F620008091EF058823F1F0E091780CF0E0EE0F87
:10F63000FF1FE45EFD4F0190F081E02D6681778130
:10F640008091600F9091610FA091620FB091630F54
:10F6500023E00297A105B10510F443E001C040E2A8
:10F66000852D2DD8332089F08091600F9091610F06
:10F67000A091620FB091630F0297A105B10528F424
:10F68000BAD888E492E901D941C26BE87CE085EF01
:10F690009CE00E94281980918B0C8F3229F031E078
:10F6A000431669F022E001C021E0A8A0B9A0C42C53
:10F6B000D12CE12CF12C22242394240C4AC08091DB
:10F6C000EF058823C9F08091600F9091610FA091A0
:10F6D000620FB091630FB695A7959795879520E235
:10F6E0000197A105B10511F44EE301C040E269EABA
:10F6F00077E0852D0E945F733320A1F28091600F27
:10F700009091610FA091620FB091630FB695A7958C
:10F71000979587950197A105B10521F66CD85AD820
:10F72000F5C1241161C140E050E0B50187E89CE0DB
:10F730000E94F33E9091CD0C8091EF05992309F43E
:10F740009BC081110BC0311074C0222DF1E0AF1AA3
:10F75000B1083FEFA316B30621F748C18091600FAF
:10F760009091610FA091620FB091630FB695A7952C
:10F7700097958795452D60E08C159D05AE05BF05D5
:10F7800061F58BE69FE00E9466316EE38BE69FE0B9
:10F790000E94A4C765E08BE69FE00E94A4C7809109
:10F7A000980C882329F01092AA0C08E91CE002C0EA
:10F7B0000BE81CE092E1992EF80161918F0166231C
:10F7C00011F0911062C1992009F4BDCF60E28BE67F
:10F7D0009FE00E94A4C79A94F6CF8BE69FE00E9418
:10F7E000663160E28BE69FE00E94A4C765E08BE68D
:10F7F0009FE00E94A4C78091980C882329F0109262
:10F80000AA0C08E91CE002C00BE81CE082E1982E7B
:10F81000F80161918F01662311F091103CC199208C
:10F8200009F491CF60E28BE69FE00E94A4C79A940E
:10F83000F6CF8091600F9091610FA091620FB0910F
:10F84000630FB695A795979587958C159D05AE0581
:10F85000BF0509F07ACF0E94FB736BE87CE087E874
:10F860009CE00E943B431092600F1092610F109237
:10F87000620F1092630F4AC1811103C0311071C031
:10F8800064CF8091600F9091610FA091620FB09151
:10F89000630FB695A795979587958C159D05AE0531
:10F8A000BF05B1F52091E20F2F8F10E0412F60E0EE
:10F8B0008BE69FE00E94663160E28BE69FE00E944B
:10F8C000A4C71F5F143091F7452D60E08BE69FE0E1
:10F8D0000E9466316EE38BE69FE00E94A4C7A9E90F
:10F8E0008A2EACE09A2EB8E96B2EBCE07B2E01E0AC
:10F8F00010E0F30121913F012111D3C014E1101B4D
:10F9000060E28BE69FE00E94A4C71150C9F7B6CF12
:10F91000452D60E08BE69FE00E94663160E28BE659
:10F920009FE00E94A4C78091980C882329F0109230
:10F93000AB0C08E91CE002C00BE81CE0F3E19F2ED1
:10F94000F80161918F01662311F09110D9C09920BF
:10F9500009F494CF60E28BE69FE00E94A4C79A94DA
:10F96000F6CF8091600F9091610FA091620FB091DE
:10F97000630FB695A795979587958C159D05AE0550
:10F98000BF0509F0E2CE0E94FB738BE89CE09F93D9
:10F990008F9388EF92E29F938F938E010F5F1F4F9B
:10F9A0001F930F930E9449D00F900F900F900F90CC
:10F9B0000F900F907E01F5E0EF0EF11CF7018081B2
:10F9C000882349F0992787FD90950E947DCFF70104
:10F9D00081937F01F3CFC8010E948A4884EF92E2AD
:10F9E0000E940A4918DD92C02F5FB0CE8091600F4F
:10F9F0009091610FA091620FB091630FB695A7959A
:10FA000097958795422F50E060E070E08417950746
:10FA1000A607B70788F0822F90E0880F991F0197FB
:10FA2000AA2797FDA095BA2F8093600F9093610F3E
:10FA3000A093620FB093630F8091600F9091610F5C
:10FA4000A091620FB091630FB695A7959795879592
:10FA50002091690F30E02D5F3F4F482F50E0241771
:10FA6000350764F42DEF280F2093690F21E02093D0
:10FA7000EF054CEF442E480E55245A94539443946A
:10FA800083E0851508F0CACD41C08BE69FE00E9457
:10FA9000A4C79A9491CE8BE69FE00E94A4C79A9443
:10FAA000B7CE452D602F8BE69FE02AA30E946631DA
:10FAB0002AA1622F8BE69FE00E94A4C70F5F1F4F11
:10FAC0000431110509F015CF34010CE211E08091E9
:10FAD0006A0F82FD05C08091E20F3F8D381749F013
:10FAE000015011090115110591F78FEF881A980A35
:10FAF000FECE61E070E080E090E00E9445C3F0CF70
:10FB00008BE69FE00E94A4C79A941ACFA2960FB6E4
:10FB1000F894DEBF0FBECDBFDF91CF911F910F9143
:10FB2000FF90EF90DF90CF90BF90AF909F908F901D
:10FB30007F906F905F904F903F902F900895CF925D
:10FB4000DF92EF92FF920F931F93CF93DF938091F9
:10FB5000600F9091610FA091620FB091630F81309F
:10FB60009048A105B10540F01092600F1092610F0E
:10FB70001092620F1092630F8091600F9091610F4D
:10FB8000A091620FB091630FB695A7959795879551
:10FB90004091690F50E060E070E084179507A60778
:10FBA000B70710F48093690FD091690F10916A0F15
:10FBB00012FB112710F9C0E0BFE0CB2ED12CE12CB5
:10FBC000F12C01E04091600F5091610F6091620F44
:10FBD0007091630FD1113BC08091EF058823C9F06C
:10FBE000E091780CF0E0EE0FFF1FE45EFD4F019016
:10FBF000F081E02D8681978123E042305105610537
:10FC0000710510F443E001C040E2BC018C2F0E945A
:10FC10005F73112309F4A6C18091600F9091610F69
:10FC2000A091620FB091630F0297A105B10508F092
:10FC300099C10E94FB7388E492E9DF91CF911F91F3
:10FC40000F91FF90EF90DF90CF900C944574D130DE
:10FC5000A9F58091EF05882391F0769567955795E2
:10FC6000479520E2413051056105710511F44EE3DD
:10FC700001C040E264ED72E28C2F0E945F73112399
:10FC800009F470C18091600F9091610FA091620F93
:10FC9000B091630FB695A795979587950197A105A4
:10FCA000B10509F05FC10E94FB73DF91CF911F91F5
:10FCB0000F91FF90EF90DF90CF90DDCBD230A9F580
:10FCC0008091EF05882391F0769567955795479534
:10FCD00020E2423051056105710511F44EE301C087
:10FCE00040E265EC72E28C2F0E945F73112309F4ED
:10FCF00039C18091600F9091610FA091620FB09116
:10FD0000630FB695A795979587950297A105B105BD
:10FD100009F028C10E94FB73DF91CF911F910F91D1
:10FD2000FF90EF90DF90CF908FCBD330A9F58091EB
:10FD3000EF05882391F0769567955795479520E2D2
:10FD4000433051056105710511F44EE301C040E2F5
:10FD500066EB72E28C2F0E945F73112309F402C1DB
:10FD60008091600F9091610FA091620FB091630F2D
:10FD7000B695A795979587950397A105B10509F0C5
:10FD8000F1C00E94FB73DF91CF911F910F91FF9003
:10FD9000EF90DF90CF909DCBD430A9F58091EF0507
:10FDA000882391F0769567955795479520E24430E2
:10FDB00051056105710511F44EE301C040E266EAA8
:10FDC00072E28C2F0E945F73112309F4CBC08091E3
:10FDD000600F9091610FA091620FB091630FB69583
:10FDE000A795979587950497A105B10509F0BAC025
:10FDF0000E94FB73DF91CF911F910F91FF90EF90C5
:10FE0000DF90CF907DCBD530A9F58091EF05882389
:10FE100091F0769567955795479520E245305105C5
:10FE20006105710511F44EE301C040E266E972E23A
:10FE30008C2F0E945F73112309F494C08091600F8E
:10FE40009091610FA091620FB091630FB695A79545
:10FE5000979587950597A105B10509F083C00E9484
:10FE6000FB73DF91CF911F910F91FF90EF90DF9087
:10FE7000CF9018CBD630A9F58091EF05882391F06B
:10FE8000769567955795479520E24630510561056F
:10FE9000710511F44EE301C040E267E872E28C2F75
:10FEA0000E945F73112309F45DC08091600F9091EF
:10FEB000610FA091620FB091630FB695A7959795CA
:10FEC00087950697A105B10509F04CC00E94FB7308
:10FED000DF91CF911F910F91FF90EF90DF90CF9026
:10FEE00026CBD73009F03EC08091EF058823E9F09A
:10FEF000E091780CF0E0EE0FFF1FE45EFD4F019003
:10FF0000F081E02D86A597A576956795579547953D
:10FF100020E2473051056105710511F44EE301C03F
:10FF200040E2BC018C2F0E945F731123D9F08091B5
:10FF3000600F9091610FA091620FB091630FB69521
:10FF4000A795979587950797A105B10559F40E9444
:10FF5000FB73DF91CF911F910F91FF90EF90DF9096
:10FF6000CF9061CA8091600F9091610FA091620F54
:10FF7000B091630F4097A105B10540F0C092600FAA
:10FF8000D092610FE092620FF092630F4091600F88
:10FF90005091610F6091620F7091630F7695679534
:10FFA000579547958091690F90E00396242F30E094
:10FFB000821793074CF48DEF840F8093690F0093A1
:10FFC000EF05DCEFD40FCFEFCF5FDF5FC43008F475
:10FFD000F9CDDF91CF911F910F91FF90EF90DF90BE
:10FFE000CF900895CF93DF93CDB7DEB728970FB6A4
:10FFF000F894DEBF0FBECDBF88E0E7E6F6E0DE0195
:020000021000EC
:10000000119601900D928A95E1F7AE014F5F5F4F17
:1000100061E08BE69FE00E94043328960FB6F894C7
:10002000DEBF0FBECDBFDF91CF910895CF93DF9399
:10003000CDB7DEB728970FB6F894DEBF0FBECDBFA1
:1000400088E0EFE2F6E0DE01119601900D928A95CC
:10005000E1F7AE014F5F5F4F61E08BE69FE00E94EA
:10006000043328960FB6F894DEBF0FBECDBFDF91E4
:10007000CF91089588EF9FE00E9465D2823028F4E6
:100080008093780C10923F0F089581E08093780C54
:1000900080933F0F08951F93CF93DF93EC01FB01F3
:1000A000608111810E946DD2612FCE010196DF9196
:1000B000CF911F910C946DD2FF920F931F93CF930A
:1000C000DF938C01EB010E9465D2F82EC8010196E6
:1000D0000E9465D2F8828983DF91CF911F910F91A1
:1000E000FF900895EF92FF920F931F93CF93DF93AA
:1000F0001F92CDB7DEB77B018C01061B170B460F95
:10010000C701800F911FF70161917F0149830E9410
:100110006DD249814E11F4CF0F90DF91CF911F9195
:100120000F91FF90EF90089581E09091D90F911178
:1001300080E08093D90F41E069ED7FE08FEF9FE091
:10014000D1DF0E9408AE21E047E050E060E070E0BF
:1001500086EE90E80C942F7481E09091D90F911164
:1001600080E08093D90F41E069ED7FE08FEF9FE061
:10017000B9DF0E9408AE21E049E050E060E070E0A5
:1001800083EF98E80C942F74EF92FF920F931F93D4
:10019000CF93DF931F92CDB7DEB77B018C01061B97
:1001A000170B460FC701800F911F49830E9465D22C
:1001B000F70181937F0149814E13F4CF0F90DF91B6
:1001C000CF911F910F91FF90EF900895CF92DF9202
:1001D000EF92FF920F931F93CF93DF9341E069ED6E
:1001E0007FE08FEF9FE0D0DF8091600F9091610FF3
:1001F000A091620FB091630F81309048A105B105C5
:1002000040F01092600F1092610F1092620F1092E6
:10021000630F8091600F9091610FA091620FB09178
:10022000630FB695A795979587954091690F50E014
:1002300060E070E084179507A607B70710F4809375
:10024000690FD091690F10916A0F12FB112710F9F5
:10025000C0E09FE0C92ED12CE12CF12C01E04091AF
:10026000600F5091610F6091620F7091630FD11117
:100270003BC08091EF058823C9F0E091780CF0E055
:10028000EE0FFF1FE45EFD4F0190F081E02D8681AF
:10029000978123E0423051056105710510F443E078
:1002A00001C040E2BC018C2F0E945F73112309F44E
:1002B00053C18091600F9091610FA091620FB09136
:1002C000630F0297A105B10508F046C10E94FB73B8
:1002D00088E492E9DF91CF911F910F91FF90EF9009
:1002E000DF90CF900C944574D130E1F58091EF050B
:1002F0008823F9F0E091780CF0E0EE0FFF1FE45E48
:10030000FD4F0190F081E02DE856FF4F80819181F3
:1003100076956795579547952EE7413051056105CC
:10032000710511F44EE301C040E2BC018C2F0E9424
:100330005F73112309F410C18091600F9091610FD8
:10034000A091620FB091630FB695A7959795879589
:100350000197A105B10509F0FFC00E94FB7386EF6C
:1003600096E897C1D230D1F58091EF058823E9F066
:10037000E091780CF0E0EE0FFF1FE45EFD4F01907E
:10038000F081E02D80AD91AD7695679557954795B5
:100390002EE7423051056105710511F44EE301C0AD
:1003A00040E2BC018C2F0E945F73112309F4D4C07A
:1003B0008091600F9091610FA091620FB091630FD7
:1003C000B695A795979587950297A105B10509F070
:1003D000C3C00E94FB7382EF99E75BC1D330E1F5A4
:1003E0008091EF058823F9F0E091780CF0E0EE0FB2
:1003F000FF1FE45EFD4F0190F081E02DEC50FF4FB8
:1004000080819181769567955795479520E2433095
:1004100051056105710511F44EE301C040E2BC01D4
:100420008C2F0E945F73112309F496C08091600F96
:100430009091610FA091620FB091630FB695A7954F
:10044000979587950397A105B10509F085C00E948E
:10045000FB7386E193E23CC0D43009F043C0809145
:10046000EF058823E9F0E091780CF0E0EE0FFF1F34
:10047000E45EFD4F0190F081E02D828593857695B5
:1004800067955795479520E2443051056105710500
:1004900011F44EE301C040E2BC018C2F0E945F7357
:1004A000112309F459C08091600F9091610FA091C0
:1004B000620FB091630FB695A795979587950497AE
:1004C000A105B10509F048C00E94FB7382E193E2E7
:1004D000DF91CF911F910F91FF90EF90DF90CF9020
:1004E0000C940A49D530C1F58091EF058823E9F0D5
:1004F000E091780CF0E0EE0FFF1FE45EFD4F0190FD
:10050000F081E02D8485958576956795579547957B
:1005100020E2453051056105710511F44EE301C03B
:1005200040E2BC018C2F0E945F731123A9F08091DF
:10053000600F9091610FA091620FB091630FB6951B
:10054000A795979587950597A105B10529F40E9470
:10055000FB738EE093E2BCCF2091D90F8091600FA6
:100560009091610FA091620FB091630F211114C09F
:10057000D63009F054C02091EF05222379F1E091A3
:10058000780CF0E0EE0FFF1FE45EFD4F0190F0816C
:10059000E02DE05EFE4F13C0D63009F040C0209140
:1005A000EF052223D9F0E091780CF0E0EE0FFF1F69
:1005B000E45EFD4F0190F081E02DE25EFE4F608130
:1005C0007181B695A7959795879520E20697A10525
:1005D000B10519F140E28C2F0E945F73112309F4D9
:1005E00062C08091600F9091610FA091620FB091F5
:1005F000630FB695A795979587950697A105B105C1
:1006000009F051C00E94FB73DF91CF911F910F91B0
:10061000FF90EF90DF90CF9087CD4EE3DCCFD730C7
:1006200009F041C02091EF052223E9F0E091780C18
:10063000F0E0EE0FFF1FE45EFD4F0190F081E02D32
:10064000EA54FE4F60817181B695A795979587957D
:100650002EE70797A105B10511F44EE301C040E272
:100660008C2F0E945F731123F1F08091600F9091A5
:10067000610FA091620FB091630FB695A795979502
:1006800087950797A105B10571F40E94FB7387E96F
:1006900096E7DF91CF911F910F91FF90EF90DF9040
:1006A000CF900C944A748091600F9091610FA0914B
:1006B000620FB091630F4097A105B10540F0C09261
:1006C000600FD092610FE092620FF092630F409141
:1006D000600F5091610F6091620F7091630F76957A
:1006E0006795579547958091690F90E00396242F61
:1006F00030E0821793074CF48DEF840F8093690FDD
:100700000093EF05DCEFD40FCFEFCF5FDF5FC43096
:1007100008F4A5CDDF91CF911F910F91FF90EF903D
:10072000DF90CF9008956FEF88EF9FE00C946DD22B
:100730008093590F1092580F0895E7EBFFE0019056
:100740000020E9F73197E75BFF401E161F0634F0E3
:100750001092CB0F82E08093EF05089580E2E431A0
:10076000F105B4F7DF01A954B04F8C933196F7CF60
:100770002091CC0F211108C044E150E0BC0187EB6F
:100780009FE00E943AD0D9CF08951092890C60E082
:1007900087E89CE00E94DE3E0E9424AD88EE92E253
:1007A0000E940A4981E08093420CE091780CF0E0CD
:1007B000EE0FFF1FE45EFD4F0190F081E02DEA5344
:1007C000FF4F80819181D4DF84EE92E20C940A493C
:1007D0002091CC0F211108C044E150E0BC0187EB0F
:1007E0009FE00E94ADCFA9CF0895F2DF81E0809312
:1007F000CC0F0C940B7A1092CC0F0895CF92DF920D
:10080000EF92FF92CF93C0910301C2FBCC27C0F9B6
:1008100081E0C8278091030181FFC260C090650F0D
:10082000D090660FE090670FF090680F0E9416C39B
:10083000C616D706E806F90620F48091000186FF67
:1008400039C0C0936A0F80916A0F817090916A0FCE
:1008500091FD82609091640F891721F18130F1F050
:1008600028F0823089F08330A1F01CC0913021F44F
:100870009091E20F9F5F05C09230A1F49091E20F3A
:1008800091509093E20F0EC0992391F3933051F45D
:10089000F5CF923069F3913029F4F0CF933041F3E2
:1008A000992361F38093640FCF91FF90EF90DF90D5
:1008B000CF900895C460C5CF0E94FF79E4E0F1E0D5
:1008C00080818B7F808380818D7F80839FB7F89428
:1008D000E5E0F1E08081846080839FBF9FB7F8945A
:1008E0008081826080839FBFE1E0F1E080818F7B27
:1008F00080839FB7F894E2E0F1E080818064808398
:100900009FBF60E08FE00E9436C29FB7F894E5E099
:10091000F1E08081816080839FBF80910301809599
:10092000817080935F0F6ADF1092E20F0895CF927B
:10093000DF92EF92FF9262DF80910301817091E07C
:10094000892720915F0F821709F182E08093EF05DC
:10095000809103018170892780935F0F0E94FF7946
:1009600080915F0F882309F4A8C087E89CE00E946B
:10097000CD39E091780CF0E0EE0FFF1FE45EFD4F03
:100980000190F081E02D8281938122DFC0905B0F86
:10099000D0905C0FE0905D0FF0905E0F0E9416C348
:1009A000C616D706E806F90608F09EC08091E20F49
:1009B000482F552747FD509557FF03C05195419546
:1009C00051094230510584F191E09093EF0587FD84
:1009D0008F5F482F4595552747FD5095652F752FFB
:1009E0008091600F9091610FA091620FB091630FA1
:1009F000840F951FA61FB71F8093600F9093610F00
:100A0000A093620FB093630F1092E20F0E9416C37F
:100A10006856754C8F4F9F4F60932F0F7093300F18
:100A20008093310F9093320F80916A0F82FF0EC036
:100A30000E9416C36856754C8F4F9F4F60932F0FBF
:100A40007093300F8093310F9093320FE091F00547
:100A5000F091F1051995C0902F0FD090300FE090D4
:100A6000310FF090320F0E9416C3C616D706E80663
:100A7000F90638F48091F0059091F105845F98496A
:100A800069F58091EF05823011F40E94207A8091FF
:100A9000EF05882319F081508093EF050E9416C35B
:100AA0006C597F4F8F4F9F4F60935B0F70935C0F1C
:100AB00080935D0F90935E0F17C087E89CE00E94C3
:100AC000CC3AE091780CF0E0EE0FFF1FE45EFD4FB2
:100AD0000190F081E02D8481958157CF0E940B7A9F
:100AE00082E08093EF05CDCFFF90EF90DF90CF9025
:100AF000089581E0089580916A0F82FB882780F92C
:100B00000895FC01808190E02AE030E0B9010E9464
:100B100050CC482FCB01B9010E9450CC805D80930E
:100B2000330F405D4093340F1092350F83E39FE005
:100B3000089520E030E040E251E4FC0160817181E1
:100B4000828193810E945ACB0E94F4C877FD02C033
:100B50002BE201C02DE22093330F9B0177FF04C0ED
:100B600022273327261B370BC90168EE73E00E944A
:100B700050CCCB01EAE0F0E0BF010E9450CC805D98
:100B80008093340FC90164E670E00E9450CCCB0121
:100B9000BF010E9450CC805D8093350FC901BF0119
:100BA0000E9450CC282FCB01BF010E9450CC805D09
:100BB0008093360F8EE28093370F205D2093380F9D
:100BC0001092390F83E39FE008958F929F92AF9226
:100BD000BF92CF92DF92EF92FF92FC0180809180D2
:100BE000A280B38020E030E048EC52E4C501B401BB
:100BF0000E945ACB6B017C0120E030E0A9010E94E9
:100C000088CA18161CF4C701B60103C0C701B60193
:100C100090580E94F4C86B017C0120E030E0A901EB
:100C2000C501B4010E9485C887FF12C08DE2809380
:100C3000330FC701B60128EE33E040E050E00E94D8
:100C400085CCCA01B9012AE030E040E050E036C06E
:100C5000C701B60120E137E240E050E00E9485CCB8
:100C6000AAE08A2E912CA12CB12CCA01B901A501B0
:100C700094010E9485CC662391F0605D6093330FF0
:100C8000C701B60128EE33E040E050E00E9485CC79
:100C9000CA01B901A50194010E9485CC13C080E26C
:100CA0008093330FC701B60128EE33E040E050E0F7
:100CB0000E9485CCCA01B901A50194010E9485CC8E
:100CC000662311F0605D01C060E26093340FC701DC
:100CD000B60124E630E040E050E00E9485CCFAE026
:100CE0008F2E912CA12CB12CCA01B901A501940120
:100CF0000E9485CC605D6093350FC701B601A501E8
:100D000094010E9485CC662381F0605D6093380F6A
:100D1000CA01B901A50194010E9485CC605D609370
:100D2000370F8EE28093360F15C0CA01B901A501B5
:100D300094010E9485CC662329F0605D6093370F93
:100D40008EE203C080E28093370F8093360F80E2FB
:100D50008093380F1092390F83E39FE0FF90EF905C
:100D6000DF90CF90BF90AF909F908F900895FC013F
:100D70002081318137FF07C08DE28093330F319599
:100D80002195310914C02436310574F0C90164E697
:100D900070E00E9450CCCB016AE070E00E9450CC21
:100DA000805D8093330F06C080E28093330F2A303A
:100DB000310564F0EAE0F0E0C901BF010E9450CCC7
:100DC000CB01BF010E9450CC805D01C080E28093C6
:100DD000340FC9016AE070E00E9450CC805D8093BE
:100DE000350F1092360F83E39FE00895AF92BF92C4
:100DF000CF92DF92EF92FF920F931F93CF93DF93E7
:100E00006091140270911502809116029091170260
:100E10000E94A5306093440F7093450F8093460F56
:100E20009093470F6091100270911102809112020D
:100E3000909113020E94B1306093400F7093410F64
:100E40008093420F9093430F8091600F9091610FB8
:100E5000A091620FB091630F81309048A105B10558
:100E600040F01092600F1092610F1092620F10927A
:100E7000630F8091600F9091610FA091620FB0910C
:100E8000630FB695A795979587954091690F50E0A8
:100E900060E070E084179507A607B70710F4809309
:100EA000690F0091690FB0906A0FB2FABB24B0F8D5
:100EB00010E047E0C42ED12CE12CF12CAA24A394FD
:100EC0008091600F9091610FA091620FB091630FBC
:100ED00001113DC02091EF052223C9F0E091780C6B
:100EE000F0E0EE0FFF1FE45EFD4F0190F081E02D7A
:100EF000EA50FF4F6081718123E00297A105B1059F
:100F000010F443E001C040E2812F0E945F73BB20D8
:100F100009F427C18091600F9091610FA091620F39
:100F2000B091630F0297A105B10508F01AC10E94A4
:100F3000FB7386EE90E8DF91CF911F910F91FF90A8
:100F4000EF90DF90CF90BF90AF900C94457401303C
:100F500009F052C02091EF05222329F1E091780C8D
:100F6000F0E0EE0FFF1FE45EFD4F0190F081E02DF9
:100F7000E25BFF4FC081D181B695A7959795879584
:100F80000197A105B10531F486E59AE0F0DE9C01F8
:100F90004EE305C086E59AE0EADE9C0140E2BE0130
:100FA000812F0E949673BB2009F4DBC08091600FF3
:100FB0009091610FA091620FB091630FB695A795C4
:100FC000979587950197A105B10509F0CAC00E94C0
:100FD000FB73E091780CF0E0EE0FFF1FE45EFD4F35
:100FE0000190F081E02DE25BFF4F21E331E040E032
:100FF00050E066E57AE0A7C0023009F052C02091C7
:10100000EF05222329F1E091780CF0E0EE0FFF1FAD
:10101000E45EFD4F0190F081E02DEC5AFF4FC0815E
:10102000D181B695A795979587950297A105B105AA
:1010300031F484E59AE09BDE9C014EE305C084E533
:101040009AE095DE9C0140E2BE01812F0E949673DA
:10105000BB2009F486C08091600F9091610FA09130
:10106000620FB091630FB695A795979587950297F4
:10107000A105B10509F075C00E94FB73E091780CE1
:10108000F0E0EE0FFF1FE45EFD4F0190F081E02DD8
:10109000EC5AFF4F23E930E040E050E064E57AE0AD
:1010A00052C0033009F05DC02091EF05222329F1E1
:1010B000E091780CF0E0EE0FFF1FE45EFD4F019031
:1010C000F081E02DEA5AFF4FC081D181B695A795F6
:1010D000979587950397A105B10531F481E59CE0CB
:1010E00046DE9C014EE305C081E59CE040DE9C01AC
:1010F00040E2BE01812F0E949673BB2091F1809146
:10110000600F9091610FA091620FB091630FB6953F
:10111000A795979587950397A105B10511F50E94AD
:10112000FB73E091780CF0E0EE0FFF1FE45EFD4FE3
:101130000190F081E02DEA5AFF4F2FEF30E040E0C0
:1011400050E061E57CE080819181DF91CF911F913A
:101150000F91FF90EF90DF90CF90BF90AF900C94E5
:1011600070728091600F9091610FA091620FB091A9
:10117000630F0897A105B10540F0C092600FD092AF
:10118000610FE092620FF092630F4091600F5091F7
:10119000610F6091620F7091630F76956795579517
:1011A00047958091690F90E00396242F30E08217D5
:1011B00093074CF48DEF840F8093690FA092EF0595
:1011C0000CEF040F1FEF1F5F0F5F143008F478CE91
:1011D000DF91CF911F910F91FF90EF90DF90CF9013
:1011E000BF90AF900895AF92BF92CF92DF92EF92EF
:1011F000FF920F931F93CF93DF9341E069ED7FE060
:101200008FEF9FE00E94C4808091600F9091610FEA
:10121000A091620FB091630F81309048A105B10594
:1012200040F01092600F1092610F1092620F1092B6
:10123000630F8091600F9091610FA091620FB09148
:10124000630FB695A795979587954091690F50E0E4
:1012500060E070E084179507A607B70710F4809345
:10126000690F0091690FB0906A0FB2FABB24B0F811
:1012700010E04FE0C42ED12CE12CF12CAA24A39431
:101280008091600F9091610FA091620FB091630FF8
:1012900001113BC02091EF052223B9F0E091780CB9
:1012A000F0E0EE0FFF1FE45EFD4F0190F081E02DB6
:1012B0006681778123E00297A105B10510F443E030
:1012C00001C040E2812F0E945F73BB2009F419C264
:1012D0008091600F9091610FA091620FB091630FA8
:1012E0000297A105B10508F00CC20E94FB7388E4C7
:1012F00092E9DF91CF911F910F91FF90EF90DF90D6
:10130000CF90BF90AF900C944574013009F052C05B
:101310002091EF05222329F1E091780CF0E0EE0F07
:10132000FF1FE45EFD4F0190F081E02DE45BFF4F75
:10133000C081D181B695A795979587950197A1050D
:10134000B10531F48DED95E012DD9C014EE305C051
:101350008DED95E00CDD9C0140E2BE01812F0E94E5
:101360009673BB2009F4CDC18091600F9091610FFD
:10137000A091620FB091630FB695A7959795879549
:101380000197A105B10509F0BCC10E94FB73E09172
:10139000780CF0E0EE0FFF1FE45EFD4F0190F0814E
:1013A000E02DE45BFF4F27EE33E04AE050E06DEDC7
:1013B00075E054C0023009F05FC02091EF05222390
:1013C00029F1E091780CF0E0EE0FFF1FE45EFD4F95
:1013D0000190F081E02DE25BFF4FC081D181B69595
:1013E000A795979587950297A105B10531F486E5F4
:1013F0009AE0BDDC9C014EE305C086E59AE0B7DCCF
:101400009C0140E2BE01812F0E949673BB2009F42B
:1014100078C18091600F9091610FA091620FB0919F
:10142000630FB695A795979587950297A105B10586
:1014300009F067C10E94FB73E091780CF0E0EE0FB9
:10144000FF1FE45EFD4F0190F081E02DE25BFF4F56
:1014500021E331E040E050E066E57AE0808191816F
:10146000DF91CF911F910F91FF90EF90DF90CF9080
:10147000BF90AF900C947072033009F052C020916D
:10148000EF05222329F1E091780CF0E0EE0FFF1F29
:10149000E45EFD4F0190F081E02DEC5AFF4FC081DA
:1014A000D181B695A795979587950397A105B10525
:1014B00031F484E59AE05BDC9C014EE305C084E5F1
:1014C0009AE055DC9C0140E2BE01812F0E94967398
:1014D000BB2009F416C18091600F9091610FA0911B
:1014E000620FB091630FB695A7959795879503976F
:1014F000A105B10509F005C10E94FB73E091780CCC
:10150000F0E0EE0FFF1FE45EFD4F0190F081E02D53
:10151000EC5AFF4F2CE830E040E050E064E57AE020
:101520009DCF043009F052C02091EF05222329F10C
:10153000E091780CF0E0EE0FFF1FE45EFD4F0190AC
:10154000F081E02DEA5AFF4FC081D181B695A79571
:10155000979587950497A105B10531F481E59CE045
:1015600006DC9C014EE305C081E59CE000DC9C01AB
:1015700040E2BE01812F0E949673BB2009F4C1C0D6
:101580008091600F9091610FA091620FB091630FF5
:10159000B695A795979587950497A105B10509F08C
:1015A000B0C00E94FB73E091780CF0E0EE0FFF1FDB
:1015B000E45EFD4F0190F081E02DEA5AFF4F2FEFDE
:1015C00030E040E050E061E57CE048CF053009F0D4
:1015D00052C02091EF05222329F1E091780CF0E030
:1015E000EE0FFF1FE45EFD4F0190F081E02DE85A01
:1015F000FF4FC081D181B695A7959795879505979F
:10160000A105B10531F48BED95E0B1DB9C014EE312
:1016100005C08BED95E0ABDB9C0140E2BE01812F64
:101620000E949673BB2009F46CC08091600F90916A
:10163000610FA091620FB091630FB695A795979532
:1016400087950597A105B10509F05BC00E94FB7362
:10165000E091780CF0E0EE0FFF1FE45EFD4F01908B
:10166000F081E02DE85AFF4F27EE33E04AE050E0EA
:101670006BED75E0F3CE063009F043C02091EF0525
:101680002223E9F0E091780CF0E0EE0FFF1FE45E1A
:10169000FD4F0190F081E02DE252FF4F608171819A
:1016A000B695A7959795879520E20697A105B10570
:1016B00011F44EE301C040E2812F0E945F73BB2012
:1016C00001F18091600F9091610FA091620FB09134
:1016D000630FB695A795979587950697A105B105D0
:1016E00081F40E94FB7382E892E2DF91CF911F9117
:1016F0000F91FF90EF90DF90CF90BF90AF900C9440
:101700000A492091D90F8091600F9091610FA091AB
:10171000620FB091630F211114C0073009F055C05A
:101720002091EF05222379F1E091780CF0E0EE0FA3
:10173000FF1FE45EFD4F0190F081E02DE05EFE4F63
:1017400013C0073009F041C02091EF052223D9F0E2
:10175000E091780CF0E0EE0FFF1FE45EFD4F01908A
:10176000F081E02DE25EFE4F60817181B695A79514
:101770009795879520E20797A105B10521F140E2F1
:10178000812F0E945F73BB2001F18091600F9091C7
:10179000610FA091620FB091630FB695A7959795D1
:1017A00087950797A105B10581F40E94FB73DF912E
:1017B000CF911F910F91FF90EF90DF90CF90BF904E
:1017C000AF900C94AC804EE3DBCF8091600F909192
:1017D000610FA091620FB091630F4097A105B10511
:1017E00040F0C092600FD092610FE092620FF092D1
:1017F000630F8091600F9091610FA091620FB09183
:10180000630FB695A795979587952091690F30E05E
:101810002D5F3F4F482F50E0241735074CF42DEF34
:10182000280F2093690FA092EF050CEF080F1FEF10
:101830001F5F0F5F143008F423CDDF91CF911F910C
:101840000F91FF90EF90DF90CF90BF90AF900895F1
:10185000FC01808191818436910524F164E670E079
:101860000E9450CCCB012AE030E0B9010E9450CC5C
:10187000805D8093330F80819181B9010E9450CCAB
:10188000CB01B9010E9450CC805D8093340F8081E0
:101890009181B9010E9450CC805D8093350F1092E8
:1018A000360F23C08A309105BCF02AE030E0B90140
:1018B0000E9450CCCB01B9010E9450CC805D809336
:1018C000330F80819181B9010E9450CC805D80935B
:1018D000340F1092350F09C06AE070E00E9450CCBE
:1018E000805D8093330F1092340F83E39FE008955F
:1018F0008F929F92AF92BF92CF92DF92EF92FF9220
:10190000CF9320E030E040E251E4FC01608171813E
:10191000828193810E945ACB0E94F4C897FD02C035
:101920002BE201C02DE22093330F6B017C0197FF66
:1019300008C0F094E094D094C094C11CD11CE11C68
:10194000F11CC701B60120E137E240E050E00E94FF
:1019500085CC7AE0872E912CA12CB12CCA01B9013B
:10196000A50194010E9485CC605D6093340FC7018E
:10197000B60128EE33E040E050E00E9485CCCA0179
:10198000B901A50194010E9485CC605D6093350F7B
:10199000C701B60124E630E040E050E00E9485CC6B
:1019A000CA01B901A50194010E9485CC605D6093D4
:1019B000360FC701B601A50194010E9485CCC62F40
:1019C000CA01B901A50194010E9485CC605D6093B4
:1019D000370F8EE28093380FC05DC093390F10929D
:1019E0003A0F83E39FE0CF91FF90EF90DF90CF908D
:1019F000BF90AF909F908F900895CF92EF920F93EA
:101A0000F7E4CF2EA5E5EA2E06E423E142E162E504
:101A10008BE69FE00E9451320F91EF90CF90089596
:101A2000CF93DF93FC016491EC012196662331F0A2
:101A30008BE69FE00E943E33CE01F4CFDF91CF9141
:101A400008950F931F93CF93DF938C01EB0141E037
:101A500061E08BE69FE00E946631C801E1DF6AE346
:101A60008BE69FE00E94A4C7FE0101900020E9F7E9
:101A70006C2F6E1B6C5E41E08BE69FE00E9466312E
:101A8000BE018BE69FE0DF91CF911F910F910C94E7
:101A9000A3C7CF92DF92EF92FF920F931F93809193
:101AA000600F9091610FA091620FB091630F00974A
:101AB000A105B10509F442C0BC01882777FD8095D6
:101AC000982F0E9427C920913B0F30913C0F4091E5
:101AD0003D0F50913E0F0E945ACB9B01AC0160918B
:101AE000730C7091740C8091750C9091760C0E941F
:101AF000ACC76093730C7093740C8093750C9093C7
:101B0000760C1092600F1092610F1092620F10927B
:101B1000630FB3E5CB2EBCE0DB2EE12CF12C00E80B
:101B20001FE323E73CE04FE65CE06BE67CE087E602
:101B30009CE00E9441B481E08093EF058091EF0525
:101B4000882341F083E79CE00E949985BC0185E0F1
:101B500093E277DF80916A0F82FF0EC021E040E0C0
:101B600050E0BA0180E398E71F910F91FF90EF904A
:101B7000DF90CF900C942F741F910F91FF90EF90F6
:101B8000DF90CF900895CF93DF931F921F92CDB730
:101B9000DEB78091600F9091610FA091620FB091BC
:101BA000630FB7FF08C01092600F1092610F109280
:101BB000620F1092630F8091480F9091490FA0918E
:101BC0004A0FB0914B0F4091600F5091610F60919F
:101BD000620F7091630F84179507A607B70744F447
:101BE0008093600F9093610FA093620FB093630F87
:101BF0008091EF058823A9F080914C0F90914D0FB3
:101C00002091600F3091610F820F931F9A83898317
